:0800000C32322E332E302E3764
:1000000A3D585E4084795F3A7F8B8F6E496E744C9F
:1000000A8C777B505E5659585E5A5F605BA2968821
:1000000A53A89BA58A62808365A59281846A7975C3
:1000000A737575767B7B7F7A777C7E7E808081862E
:1000000A868A8582A587A97AB09FA288A2A68BCB69
:0F00000AA98ED7CBBD88BEADB096C0C499BEBE7F
:020000040800F2
:40800000C0D90120E1BD0008F3BD000835FB0308F7BD0008F9BD0008FBBD00080000000000000000000000000000000021830008FFBD000800000000E583000859840008EE
:4080400005BE000805BE000805BE000805BE000805BE000805BE000805BE000805BE000805BE000805BE000805BE000805BE000805BE000805BE000805BE000805BE000850
:4080800005BE000805BE000809620308676703087B68030805BE000805BE000805BE00080FCB03081BCB030827CB03089FCA0308C1CA0308CFCA0308DBCA0308A592030819
:4080C000B5920308C5920308CF92030805BE0008D99B0308A5720308AF720308B972030805BE000805BE000805BE000833CB03083FCB03084BCB030803CB030805BE00084E
:4081000005BE000805BE0008E5CA030805BE000805BE000805BE0008F1CA0308FBCA030805BE000805BE000805BE000805BE000805BE000805BE000805BE000821680308D7
:40814000EF6803086569030805BE000805BE000805BE000805BE000805BE0008D7720308D9920308E992030805BE000805BE000805BE000805BE000805BE00080000000086
:4081800005BE000805BE0008E1720308EB72030805BE000805BE0008E39B030805BE0008000000000000000005BE000800F002F800F073F80AA090E8000C82448344AAF113
:4081C0000107DA4501D100F068F8AFF2090EBAE80F0013F0010F18BFFB1A43F00103184728070400480704000A444FF0000C10F8013B13F0070408BF10F8014B1D1108BFB7
:4082000010F8015B641E05D010F8016B641E01F8016BF9D113F0080F1EBF10F8014BAD1C0C1B09D16D1E58BF01F801CBFAD505E014F8016B01F8016B6D1EF9D59142D6D37C
:40824000704700000023002400250026103A28BF78C1FBD8520728BF30C148BF0B607047632937F0E682732937F0EB82002070471FB53CF00CF89DE8030037F070FA37F0B8
:408280001AF937F0DFFB0400002000213BF030F9401C60601FBD10B510BD37F0AEFB1146FFF7E6FF12F079FE37F0DFFB03B4FFF7F2FF03BC37F010FC80F309887047EFF3DE
:4082C00009807047684680F3098804480078C00714BF0220032080F31488704750780408DFF818C0EFF305831B0618BF6047EFF31483DB0708BF604700DF7047772604088F
:40830000DFF818C0EFF305831B0618BF6047EFF31483DB0708BF604700DF70477D280408EFF30980816911F8021C01B142E010B590E80F10E047BDE81040EFF3098C254BC6
:4083400093E80600914232D041B91EF0100F16D12149086820F00100086010E00CB41EF0100F06BF2CED108A0323012381F826302CE9F00FC1F82CC03AF016FE0CBC1A609F
:40838000D2F82CC0BCE8F00F92F8263013F0020F1ABFBCEC108A6FF0120E6FF0020E8CF3098813F0010F08BF704792F82500CCF80000704710B5094A1268914209D8084C02
:4083C00054F8214090E80F10A047EFF3098C8CE80F0010BD0808002034EF00E024FB030824FB030810B53AF093FCBDE81040194B93E80600914208BF70470CB4EFF3098C24
:408400001EF0100F06BF2CED108A0223002381F826302CE9F00FC1F82CC03AF0C5FD0CBC1A60D2F82CC0BCE8F00F92F8263013F0020F1ABFBCEC108A6FF0120E6FF0020E43
:408440008CF3098813F0010F1CBF92F82530CCF8003070470808002010B53AF075FEC4E710B53AF007F93AF06FFEBEE70B49D1F800C04A685CF8043B1068184442F8040BCD
:408480008C4528BFA1F1DC0C8A4228BFA1F1DC02C1F800C04A6020F0004070470CFC00200146FB48B0F8AA0000EE100AB8EE400A81ED080AF64890ED800A81ED010A90ED86
:4084C000810A81ED020A90ED820A81ED030A90F8AF0000EE100AB8EE400A81ED050AEC4890F8AE000877EA4890ED7D0A81ED000A90F8B00000EE100AB8EE400A81ED060A02
:40850000B7EE000A81ED040A012070474FF6FF76DFF880C300DF074639460120DFF878C300DF0421DD4880F8D0110021DC4880F8441000BF002231460120DFF868C300DF99
:408540000446012C17D100BFD44890F8D10140F00101D24880F8D111B0F8DC014FF6FF71884207DACD48B0F8DC01401C81B2CB48A0F8DC11DEE7022CDCD1DFF82CC300DFD6
:40858000054605F001000028D4D0C548FFF788FFD0E7C34880ED0C0ADFEDC40AC0ED0D0ADFEDC20AC0ED0F0ADFEDC00AC0ED0E0A80ED0A0A704710B52DED0C8BB0EE409AA2
:4085C000B0EE608AF0EE419A9FEDB80AF0EE408A2422B349243101F1240037F002F89FEDB40AC9EE000AAE48C0ED090AB5EEC08AF1EE10FA04D1B0EE480AFFF7CAFF10E16A
:40860000B5EEC08AF1EE10FA07DDA54890ED130AB5EEC00AF1EE10FA0CD9B5EEC08AF1EE10FA0FD29E4890ED130AB5EEC00AF1EE10FA07DBB0EE480AFFF7ABFF31F094FB0F
:4086400097490867964A92ED080ABCEEC00A10EE101A106F31F08EFB50BBB5EEC08AF1EE10FA0ADD9FED930A8D4880ED0A0A9FED8F0A914880ED000A11E09FED900A8848D2
:4086800080ED0A0AD0ED050AB7EE001A81EE200AF0EE000A80EE201A874880ED001A804890ED0A0A80ED0C0A012085490870B8E09FED800AB4EEC08AF1EE10FA07DB9FEDFB
:4086C000810A774880ED0A0AF0EE488A80E09FED7B0AB4EEC08AF1EE10FA07D89FED7A0A6F4880ED0A0AF0EE488A71E0724890ED000A30EE290A80ED000A694890ED050A4B
:40870000DFED720A20EE200A6B48D0ED000A20EE200A10EE101A08463BF048FD41EC1D0BB0EE4D0AF0EE6D0A38F0DAFFB0EE40BAF0EE60BA5A4890ED060A10EE101A08464C
:408740003BF034FD41EC1C0B53EC1B2B3BF038FA41EC1A0B3AF0EEFE08EE900AF5EEC08AF1EE10FA05DD4E4890ED060AF0EE408A06E04B4890ED060AB1EE400AF0EE408A15
:4087800038EE880AF0EE408AB5EEC08AF1EE10FA09DDF5EEC08AF1EE10FA04D89FED4C0AF0EE408A0DE0B5EEC08AF1EE10FA08D2F5EEC08AF1EE10FA03DB9FED460AF0EED6
:4087C000408A374890ED000A20EE280A80ED0A0A3B48007870B13248C0ED0C8A90ED0A0AD0ED090A30EE600A80ED0D0A00203449087016E09FED2D0A2949243101F12400F7
:4088000016F0A7FF26493431A1F1300016F0C0FBF0EE408A224890ED0C0A30EE280A80ED0C0A1F4890ED0A0AB5EEC00AF1EE10FA0BDD90ED0C0AB5EEC00AF1EE10FA04D2C8
:408840009FED1A0A80ED0C0A54E0154890ED0A0AB5EEC00AF1EE10FA0BD290ED0C0AB5EEC00AF1EE10FA04DD9FED100A80ED0C0A40E00B4890ED0C0ADFED0E0AB4EEE00A07
:40888000F1EE10FA28DD9FED0B0A80ED0C0A31E02021002021340408E127040868520020CC16002041280408892704080000000000007A440000C842940300200000C8C2A9
:4088C0009003002066662640666626C0DB0FC9400AD7233C0AD723BCF74890ED0C0A5FED090AB4EEE00AF1EE10FA03D21FED0D0A80ED0C0AF04890ED0C0ABDEC0C8B10BDF5
:4089000001B500BF01226946EC480068B03012F0FFFD20B99DF80000E94981F8B00000BFE848D0F8CC110120DFF89CC300DF08BD10B52DED020B00BF04226946DF4800680F
:4089400000F5FA7012F0E4FD20B99DED000ADC4880ED7D0A00BFDB48D0F8CC110120DFF868C300DF1CBD01B500BF01226946D3480068AE3012F0CCFD20B99DF80000D049D4
:4089800081F8AE0000BFCF48D0F8CC110120DFF838C300DF08BD01B500BF01226946C7480068AF3012F0B4FD20B99DF80000C44981F8AF0000BFC348D0F8CC110120DFF824
:4089C00008C300DF08BD10B52DED020B00BF04226946BA48006800F5027012F099FD20B99DED000AB64880ED820A00BFB548D0F8CC110120DFF8D0C200DF1CBD10B52DED39
:408A0000020B00BF04226946AC48006800F5017012F07EFD20B99DED000AA94880ED810A00BFA848D0F8CC110120DFF89CC200DF1CBD10B52DED020B00BF042269469F4837
:408A4000006800F5007012F063FD20B99DED000A9B4880ED800A00BF9A48D0F8CC110120DFF864C200DF1CBD01B500BF0222694692480068AA3012F04BFD20B9BDF8000028
:408A80008F49A1F8AA0000BF8E48D0F8CC110120DFF834C200DF302004F062FD08BD10B58AB00446022C1FD1B2EE040A8DED090A9FED860A8DED020A1FED840A8DED030AC7
:408AC0009FED820A8DED040A9FED810A8DED060A01208DF820009FED7F0A8DED010AB1EE080A8DED070AA8E0042C1FD1B3EE080A8DED090A1FED910A8DED020A1FED950AD9
:408B00008DED030A1FED950A8DED040A1FED970A8DED060A01208DF820009FED6F0A8DED010AB1EE040A8DED070A86E0052C01D01A2C1FD1B2EE060A8DED090A9FED670AE4
:408B40008DED020A1FEDA70A8DED030A9FED630A8DED040A1FEDA90A8DED060A01208DF820009FED5F0A8DED010AB2EE020A8DED070A62E00E2C1FD1B2EE040A8DED090A43
:408B80009FED520A8DED020A1FEDB80A8DED030A9FED520A8DED040A9FED4D0A8DED060A01208DF820009FED4E0A8DED010AB2EE040A8DED070A40E0152C1FD1B2EE040AAE
:408BC0008DED090A9FED470A8DED020A1FEDC90A8DED030A9FED430A8DED040A9FED3C0A8DED060A01208DF820009FED3A0A8DED010AB1EE080A8DED070A1EE01FEDD50A22
:408C00008DED090A1FEDD70A8DED020A1FEDD90A8DED030A1FEDDB0A8DED040A1FEDDD0A8DED060A00208DF820001FEDE00A8DED010A1FEDE20A8DED070A9DED090ABDEEBD
:408C4000C00A10EE101A08B2FFF70EFFDDED020AB0EE600AFFF7EDFEDDED030AB0EE600AFFF7CCFEDDED040AB0EE600AFFF7ABFE9DED060ABCEEC00A10EE101AC8B2FFF7C2
:408C80008AFE9DF82000FFF76EFEDDED010AB0EE600AFFF74DFE9DED070ABCEEC00A10EE101AC8B2FFF72CFE302004F059FC552004F056FC0AB010BDCC160020F003002036
:408CC0002021002068520020E1270408000048420000A042F3FDD43CA69B443C0000484396438B3C0000F042204890ED0A0ABDEEC00A10EE100A00B270471C4890ED090AB8
:408D0000BDEEC00A10EE100A00B2704780220270164A92ED010ADFED160A20EE200ABCEEC00A10EE102A91B241700A0A82700F4A92ED020ADFED0E0A20EE200ABCEEC00A01
:408D400010EE102A91B2C1700A0A0271074A92ED030ADFED070A20EE200ABCEEC00A10EE102A91B241710A0A82717047CC1600200000C84270B5054601249148DFF844C218
:408D800000DF204670BD9049097801708F49416001218160002181764176704700B5A1B06846FFF7F0FF01208DF8180006219DF81920501CC0B28DF819000DF14B0081548E
:408DC00000208DF819006846019930F099FC002021B000BD00B5A1B06846FFF7D4FF02208DF8180005219DF81920501CC0B28DF819000DF14B00815400208DF819006846D4
:408E0000019930F07DFC9DF81800401E0DF11B01085C21B000BD2DE9F74F814615464FF000081FFA89F7E8191FFA80FBBBF5005F02DD4FF0080855E02D2D02DD4FF04008C3
:408E400050E04FF47A615E48DFF884C100DF012802D14FF0100845E0842036F0C7F90446002C3FD0FFF79AFFFFF7B4FF82462046FFF789FFE81C20760221627E501C6076B9
:408E800004F14B008154390A627E501C607604F14B008154627E501C607604F14B008754627E014650182A46019936F055FB002060762046616830F023FC94F8800001283E
:408EC0000BD1FFF787FF06460AF0020010B106F0020020B14FF0800801E04FF02008204636F0BFF93648DFF8ECC000DFB8F1000F05D03948007840EA0800374908704046DF
:408F0000BDE8FE8F2DE9F043A1B080460F4614460026BDB260191FFA80F9B9F5005F01DD082642E02D2C01DD40263EE06846FFF72AFFE01CC0B28DF8180003219DF8192090
:408F4000501CC0B28DF819000DF14B008154290A9DF81920501CC0B28DF819000DF14B0081549DF81920501CC0B28DF819000DF14B0085549DF819200146501855222146F5
:408F800036F061FB00208DF819006846019930F0B7FB9DF88000012806D122460DF11E01404636F0D9FA00E0202626B10A480078304309490870304621B0BDE8F0830000DB
:408FC000D8560020B52B04083E07002000380040A92C0408C52B0408ED03002000487047D0FA0020401ECAB210F8011F8A4202D00029F9D100207047FFFFFFFFFFFFFFFF22
:40900000FE4890ED0A0A704710B52DED048BB0EE408A0446F94890ED720ADFEDF90A80EE201AB0EE419AF74890F8AE0058B1FFF7E7FFF0EE409A9FEDF41AF0EE480AFFF786
:40904000BAFAB0EE408AEF4890F89C00012803D1B1EE480AB0EE408A9FEDEC0AB4EEC08AF1EE10FA04D29FEDE90AB0EE408A0AE09FEDE70AB4EEC08AF1EE10FA03DD9FED67
:40908000E40AB0EE408A0E2C14D008DCA4F10200052866D2DFE800F0111410124B00A4F1120009285DD2DFE800F0430C5C065C5C0D5C0A0000BF00BF00BF00BF00BF00BFFF
:4090C00000BF00BFB5EEC08AF1EE10FA0ED2B1EE480AB0EE408A0021CE4800782EF0ACFA0121CD4800782EF0A7FA19E0B5EEC08AF1EE10FA0ADD0121C64800782EF09CFAF0
:409100000021C54800782EF097FA09E00021C14800782EF091FA0021BF4800782EF08CFAB0EE480ABD48007832F08AFE1AE000BFF0EE000A89EE200A9FEDB51AC8EE010AED
:4091400060EE890AB1EE001AC0EE811A70EE218ADFEDB30AB0EE680AB24800782EF0E6FA00E000BF00BFBDEC048B10BDAE480078704710B50446AD480078A04205D0AB484C
:4091800004700C2028F066F80DE0A948006830F013FEB0F5FA7F06D930F0E6FDA44908600C2028F057F810BD10B50446954991F830000FF0F7FE90B12046FFF7DAFF2146F6
:4091C0009C4800782EF038FA21469B4800782EF033FA2146994800782EF02EFA1CE02FF054F850B12146934800782EF025FA2146914800782EF020FA0EE021468D480078BF
:409200002EF01AFA21468C4800782EF015FA21468A4800782EF010FA10BD10B52FF035F8C8B127F0C1FADFED860AB4EEE00AF1EE10FA10D24FF47A718248006830F09AFD50
:40924000E0B101217D4800782EF0F6F930F08CFD7D49086012E02FF018F878B140F6B8317948006830F086FD40B10021734800782EF0E2F930F078FD7249086010BD6A496F
:409280000870704770B52DED048B04460D466F48007848B10120207001216D4880F8291030F062FD6A490862207830B1012845D0022857D003287ED168E0654890F82900EF
:4092C00001280ED16248016A284630F084FDFA2807D2012020705E4890ED090A84ED010A2BE05B4890F8350001280ED15848C16A284630F070FDFA2807D202202070544862
:4093000090ED0C0A84ED010A17E0514890F8410001280ED14E48816B284630F05CFDFA2807D2032020704A4890ED0F0A84ED010A03E09FED480A84ED010A3FE0444890F892
:40934000290030B14248016A284630F044FDFA2802D90020207004E03D4890ED090A84ED010A2BE03A4890F8350030B13848C16A284630F030FDFA2802D90020207004E0DB
:40938000334890ED0C0A84ED010A17E0304890F8410030B12E48816B284630F01CFDFA2803D90020207005E005E0294890ED0F0A84ED010A02E00020207000BF00BF94ED75
:4093C000020A84ED030A2078B0B194ED050AB5EEC00AF1EE10FA6ED094ED010A10EE101A08463AF0E3FE41EC190BB0EE490AF0EE690A37F0B5FA2FE086E00000EC080020C7
:4094000000007A44202100206F12833A0000C8C20000C84231070020320700208F070020030058415707002038000020400000203C000020700700208807002090070020A9
:409440003D0A0F4030000020340000202D0000204008002000000000B0EE408AF0EE608A9FEDFA0B53EC102B51EC180B3AF06CFB3DD894ED010AB5EEC00AF1EE10FA04D105
:409480001FED0C0A84ED020A35E094ED010AD4ED050A30EE600AD4ED020AB4EEE00AF1EE10FA09DD94ED020AD4ED050A30EE200A84ED020A1FE01AE094ED010AD4ED050A75
:4094C00030EE200AD4ED020AB4EEE00AF1EE10FA08D294ED020AD4ED050A30EE600A84ED020A08E094ED010A84ED020A03E094ED010A84ED020A94ED020A84ED040A01209C
:40950000D44981F8480013E01FED2E0A84ED020A1FED300A84ED010A1FED320A84ED030A1FED340A84ED040A0020CA4981F8480094ED040AC74880ED110ABDEC048B70BDC9
:4095400070B52DED088B044603F066FFB0EE408A94ED090AD4ED0B0A30EE200AF0EE000A80EE201AF0EE418A94ED080AD4ED0A0A30EE200AF0EE000A80EE201AB0EE419A6B
:4095800094ED020AB4EEE80AF1EE10FA33DD94F84400022825D1B2EE040A03F000F8E0B994ED120A38EE400AF0EE040AB4EEE00AF1EE10FA11D20FF01DFD10B141F2883059
:4095C00001E04FF47A7005462946E06C30F0D2FB30B101215020015502E000215020015508E0022084F8440084ED128A30F0BCFBE06400BF5EE094ED020AB4EEC90AF1EE08
:4096000010FA33D294F84400012825D1B2EE040A02F081FFE0B994ED120A38EE400AF8EE040AB4EEE00AF1EE10FA11DD0FF0E2FC10B141F2883001E04FF47A7005462946BE
:40964000E06C30F097FB30B101215020015502E000215020015508E0012084F8440084ED128A30F081FBE06400BF23E0002084F8440094ED120A30EE480A10EE101A08467F
:409680003AF094FD41EC1B0BB0EE4B0AF0EE6B0A37F066F9B0EE40AAF0EE60AA9FED6E0B53EC102B51EC1A0B3AF088FB02D2002150200155BDEC088B70BD70B52DED0C8BD8
:4096C00004460D4694ED0A0AF2EE040AB4EEE00AF1EE10FA0CD294ED0A0AFAEE040AB4EEE00AF1EE10FA03DD1FEDA60A84ED0A0A94ED0A0A5FEDBE0AC0EE208A95ED020A47
:40970000D5ED080AB4EEE00AF1EE10FA18D895ED0C0AD5ED020A20EE200A1FEDC31AC0EE010A94ED780A20EE800A1FEDCB1AC0EE010A95ED0D0A30EEC00A84ED620A25E008
:4097400095ED020AD5ED090AB4EEE00AF1EE10FA18DB95ED0C0AD5ED020A60EE200A1FEDD41A80EE810AD4ED780A60EE200A1FEDDC1A80EE810AD5ED0D0A30EE200A84ED05
:40978000620A03E01FEDCD0A84ED620A95ED020AB5EEC00AF1EE10FA02D11FEDE78A18E094ED620A10EE101A08463AF0FFFC41EC1B0BB0EE4B0AF0EE6B0A37F0D1F8B0EEBF
:4097C00040AAF0EE60AA51EC1A0B39F0B3FE08EE100A94ED620A10EE101A08463AF0E6FC41EC1D0BB0EE4D0AF0EE6D0A37F0B8F8B0EE40BAF0EE60BA18EE900A3AF0D6FC3A
:4098000041EC1D0BB0EE4D0AF0EE6D0A37F0A8F8B0EE40CAF0EE60CA53EC1B2B51EC1C0B3AF0DAFB41EC1A0B39F084FE09EE100A89EE080AB0EE409A1E210948B0EE490A9A
:409840001DF07FFFBDEC0C8B70BD0000000000000000594040080020000000000000F83F2C0800202DE9F0412DED028B04460D46FA4890F8BD010A287DD14FF43270015992
:40988000001D0151001FD4F8C4120151F448007832F031FAC4F8C4024FF432700059D4F8C412081A00EE100AB8EEC00ADFEDED0A80EE201A84EDB41A94EDB40AB2EE041A82
:4098C000C0EE010A9FEDE80A20EE800A84EDC40A95ED020AD5ED080AB4EEE00AF1EE10FA23D895ED0E0AD5ED020A20EE200A9FEDDF1AC0EE010A94ED780A20EE800A9FED83
:40990000DC1AC0EE010A95ED0F0A30EEC00A84EDDA0A94EDDA0AB5EEC00AF1EE10FA37DD9FEDD40A84EDDA0A32E095ED020AD5ED090AB4EEE00AF1EE10FA25DB95ED0E0A8E
:40994000D5ED020A20EE200A9FEDC81AC0EE010A94ED780A20EE800A9FEDC51AC0EE010A95ED0F0A30EE800A84EDDA0A94EDDA0AB5EEC00A00E08CE0F1EE10FA08D29FEDF6
:40998000BD0A84EDDA0A03E09FEDBA0A84EDDA0AB24890F8300091280ED0B04890F83000922809D0AD4890F83000712804D0AB4890F83000B82803D132274FF0480802E034
:4099C00032274FF04108D4EDC40AB0EE600A394604F53E701DF0B5FED4EDDA0AB0EE600A414604F554701DF0ACFE94EDD40AD4EDBE0A30EE600AF2EE040A20EE208A9FEDBF
:409A00009C0AB4EEC08AF1EE10FA04DD9FED980AB0EE408A0AE09FED980AB4EEC08AF1EE10FA03D29FED940AB0EE408A012104F53970B0EE480A1DF084FE94EDD40A84EDCD
:409A4000DD0A94EDBE0A84EDC70A04261AE0711E04F55D7000EB810090ED000A04F55D7000EB860080ED000A04F5477000EB810090ED000A04F5477000EB860080ED000A1F
:409A8000701EC6B2002EE2DC94EDB90A7B4880ED150ABDEC028BBDE8F081704991F84A10062904D06D4991F84A10122901D1012000E00020704710B52DED020B00BF0422E7
:409AC00069466F48006800F5587011F021FD20B99DED000A614880EDD80A00BF1CBD10B52DED020B00BF042269466548006800F5577011F00DFD20B99DED000A574880EDEA
:409B0000D70A00BF1CBD10B52DED020B00BF042269465B48006800F5567011F0F9FC20B99DED000A4D4880EDD60A00BF1CBD10B52DED020B00BF042269465148006800F513
:409B4000557011F0E5FC20B99DED000A434880EDD50A00BF1CBD414991F84A10032901D1012000E00020704710B52DED020B00BF042269464248006800F55C7011F0C8FC27
:409B800020B99DED000A354880EDDC0A00BF1CBD10B52DED020B00BF042269463848006800F55B7011F0B4FC20B99DED000A2B4880EDDB0A00BF1CBD10B52DED020B00BF82
:409BC000042269462E48006800F55A7011F0A0FC20B99DED000A214880EDDA0A00BF1CBD10B52DED020B00BF042269462448006800F5597011F08CFC20B99DED000A174830
:409C000080EDD90A00BF1CBD144991F84A10042922D0124991F84A1002291DD00F4991F84A10052918D00D4991F84A100E2913D00A4991F84A1015290ED0084991F84A105D
:409C4000132909D0054991F84A10182904D0034991F84A101A2915D1012014E020210020540700208DED244800606A470000C84200007A440000000000007AC440080020DB
:409C8000F00300200020704710B52DED028B84B00446FFF760FF10B1B2EE048A01E0B7EE008AFE4890ED280A20EE080A84ED000AB0F8A80000EE100AB8EE400A84ED020A27
:409CC0001FED140A84ED010AF44890F89C0084F82C00F24890F842106C3000EB810090ED000A84ED030AED4890F84210743000EB810090ED000A84ED040AE84890F8421066
:409D00007C3000EB810090ED000A84ED050AE34890F84210843000EB810090ED000A84ED060ADE4890ED700A84ED070A90ED710A84ED080A90ED720A84ED090A90ED730A46
:409D400084ED0A0A2DF04EFC002876D0FFF7A5FE78B30121D24800782DF06EFC0021D14800782DF069FC0021CF4800782DF064FCB2EE040AFFF7DBFE9FEDCC0AFFF7C3FE93
:409D8000B7EE000AFFF7ABFE1FED460AFFF793FE9FEDC70AFFF724FF9FEDC60AFFF70CFF9FEDC50AFFF7F4FE1FED4F0AFFF7DCFE95E0FFE7FFF728FFF0B3C048009094EDF3
:409DC000020AF0EE400A9FEDBE0A01231A46BD49BD48007831F096FC0021B14800782DF02BFC0121AF4800782DF026FC0121AE4800782DF021FC9FEDB50AFFF798FE9FED4E
:409E0000AD0AFFF780FE9FEDAC0AFFF768FE1FED680AFFF750FE9FEDAE0AFFF7E1FE9FEDA50AFFF7C9FE9FEDA40AFFF7B1FE1FED700AFFF799FE52E000E041E0FFF78BFEE2
:409E400070B39E48009094ED020AF0EE400A9FED9C0A01231A469B499B48007831F052FC00218F4800782DF0E7FB01218D4800782DF0E2FB01218C4800782DF0DDFB9FED69
:409E8000930AFFF754FE9FED8B0AFFF73CFE9FED8A0AFFF724FE1FED8A0AFFF70CFE1EE000217F4800782DF0C7FB01217D4800782DF0C2FB01217C4800782DF0BDFB0EE0FD
:409EC0007E48009094ED020AF0EE400A9FED7C0A012300227F497C48007831F013FC94F82C00B0B90020009001900290034603227949039055202DF076FC002000900190CF
:409F00000290034603227549039056202DF06BFC15E00020009001900290034603226F49039055202DF05FFC0020009001900290034603226849039056202DF054FC0120DF
:409F400004B0BDEC028B10BD2DED028B5421644835F081FB4FF46771624835F07CFB5821614835F078FB5E48604908605E4848305F4908605B485F49086000F5F0705E4912
:409F80000860A0F5DC705D49086000F5B0705C49086000F59E705B4908604C305A490860514854305949086059485A4908604C481430594908601FEDD30A143880ED030A2E
:409FC0001FEDD60A484880ED130A9FED540A80ED140AFFF7C0FD40B1DFF844C100DF06460A2202212FF0CAFF0AE02DF0FBFA38B1DFF82CC100DF0646012202212FF0BEFF0E
:40A00000DFF81CC100DF064602212FF0FDFFDFF810C100DF064631460120DFF808C100DF0321414880F8541000BF00224FF6FF710320DFF8F8C000DF044604F00100002802
:40A04000F3D104F002000028EFD0DFF8E4C000DF054605F0010030B121481430FFF714FE1D2027F0F7F805F002000028DDD03148007818F0F3FA1B4880ED780AD0ED780A88
:40A08000B0EE600A142100F5E4701DF05AFB2DF091FA08B1284851E05FE00000202100206C0700208D0700208C0700206F12833A00401C45000048420000FA4370EC0020FA
:40A0C000A037A04B001800408F070020000048450080544500000140A1070020A207002098080020EC080020400800200000002004000020080000200C0000201000002014
:40A100001400002018000020200000201C000020540C002024000020280000200000C8C221340408E12704086852002041280408892704080F07002060070020007818F0E4
:40A140004AFCFE4880ED0A0AD0ED0A0AB0EE600A1E2110301DF0F5FA87E02DF043FA002823D0FFF79AFC08B3F548007818F033FCF24880ED8E0AF348007818F06FFAEF48D5
:40A1800080EDA40AD0EDA40AB0EE600A142100F51E701DF0D6FAE948D0ED8E0AB0EE600A142100F508701DF0CCFA5EE0E648007818F011FCE14880ED0A0AD0ED0A0AB0EE67
:40A1C000600A1E2110301DF0BCFADC4890ED0A0AD0ED040A30EE600A20EE000AB0EE408A1E212030B0EE480A1DF0ABFAD748007818F0F1FBD14880ED200AD0ED200AB0EE3A
:40A20000600A1E2168301DF09CFACC4890ED200AD0ED1A0A30EE600A20EE000AB0EE408A1E217830B0EE480A1DF08BFAC848007818F0D1FBC14880ED360AD0ED360AB0EE80
:40A24000600A1E21C0301DF07CFAC248007818F0C2FBBA4880ED4C0AD0ED4C0AB0EE600A1E2100F58C701DF06CFABB49B348FFF7F9FAB949B148FFF720FAB748FFF760F9B7
:40A280002FF072FD06463146B348FEF7FBFFB248007818B1B14890F84800A0BB2DF08AF990B19FEDAF0AAC4880ED020A0020A34908700021AB4800782DF0BEF90021AA487A
:40A2C00000782DF0B9F950E02DF08CF900284CD09FEDA30AA04880ED020A0020974908700021A14800782DF0A7F900219D4800782DF0A2F900219D4800782DF09DF9002029
:40A30000FEF7BDFF31E0FFE7944890F8480001282BD18A48007840BB2DF04CF968B10120864908700121904800782DF085F901218C4800782DF080F917E02DF053F9A0B1BA
:40A3400001207E4908700121874800782DF074F90121844800782DF06FF90121834800782DF06AF90120FEF78AFFFEF756FFFEF7FDFE0646FEF718FF7D4991F84A00764931
:40A38000D1ED020AB0EE600AFEF73EFE4DE601B50DF0E4FA70B900BF01226946754800689C3011F0B5F820B99DF80000704981F89C0000BF7048016D0120DFF8C0C100DF04
:40A3C000142003F0CDF808BD10B52DED020B00249DED000AF2EE040AB4EEE00AF1EE10FA05DDB2EE040A8DED000A02240BE09DED000AB5EEC00AF1EE10FA04D29FED580AD2
:40A400008DED000A032400BF0422694659480068A03011F07DF820B99DED000A544880ED280A00BF5448016D0120DFF850C100DF192003F095F820461CBD01B500BF0222A4
:40A4400069464C480068A83011F062F820B9BDF800004749A1F8A80000BF4748016D0120DFF818C100DF08BD10B5FFF774FB58B144F62060FFF7E1FFB6EE000AFFF7A4FF64
:40A480000020FFF784FF1BE0FFF707FB50B12820FFF7D3FF9FED320AFFF796FF0020FFF776FF0DE0FFF7B0FB50B144F62060FFF7C4FF9FED2B0AFFF787FF0020FFF767FF66
:40A4C0002B4991F84A00FEF7EAFA012010BD70B52DED028BB0EE408A04460D460026012C04D0022C03D0032C6DD101E000BF00BF1A4890ED140AB4EEC80AF1EE10FA05DD4D
:40A5000090ED140AB0EE408A03260CE0134890ED130AB4EEC80AF1EE10FA04D290ED130AB0EE408A022610210C48DFF854C000DF012846D004EB4401084823E0EC08002088
:40A54000580700205D0700206007002063070020A1070020A207002098080020400800200000000071070020720700207307002020210020F003002068520020E1270408E1
:40A58000A92C0408143000EB810080ED018A2FF0EBFB04EB4402F84941F82200012104EB4402F54800EB8200017204EB4401F24800EB81004572F0481438DFF8C0C300DF7A
:40A5C00000E0062601E0062600BF00BF3046BDEC028B70BDE848143890ED110A7047E84890F85000012800D170470020FCE7E248143890ED150A70470020DF49143991F87D
:40A600004810012904D1DF490978012900D10120704701B500BF01226946DB4800684A3010F076FF20B99DF80000D84981F84A0000BFFFF719FFD648016D0120DFF854C3CC
:40A6400000DF272002F08CFF08BDCE4890ED780A7047CC4890ED8E0A7047CA4890ED040A7047C84890ED1A0A7047C64890ED080A7047C44890ED300A7047C24890ED460A65
:40A68000704700B5FFF767FA30B1C348007808B1012000BD0020FCE70020FAE700207047BD480078022804D1BC48007D012800D170470020FCE710B5FFF7EFF930B1B848CC
:40A6C00000782DF0BBFB08B1012010BD0020FCE7AE4890F84A00182801D1012070470020FCE700B50121FFF7F3FF00B900E00021084600BD70B52DED068B0024FFF77CFFC7
:40A7000080B32CF08BFF68B3FFF7EBFF50B3FFF77BFA38B39D4890EDD50A10EE101A084639F044FD41EC180BFEF76AFC10EE105A284639F03BFD41EC1A0BB0EE4A0AF0EEC7
:40A740006A0A36F00DF9B0EE409AF0EE609A53EC182B51EC190B39F031FB01D2012000E0002004462046BDEC068B70BD0020844991ED020A854991F84220743101EB820162
:40A78000D1ED000AB4EEE00AF1EE10FA10DB7C4991ED020A7D4991F84220843101EB8201D1ED000AB4EEE00AF1EE10FA00D8012070470020724991ED020A744991F8422053
:40A7C0006C3101EB8201D1ED000AB4EEE00AF1EE10FA10D86A4991ED020A6C4991F842207C3101EB8201D1ED000AB4EEE00AF1EE10FA00DB0120704700B50023FFF7D9FF99
:40A8000010B9FFF7B3FF00B10123184600BD70B52DED068B0024FFF7EFFE88B32CF0FEFE70B3FFF7E9FF58B3FFF75BFF40B3FFF7EBF928B3554890EDD60A10EE101A084619
:40A8400039F0B4FC41EC180BFEF7DAFB10EE105A284639F0ABFC41EC1A0BB0EE4A0AF0EE6A0A36F07DF8B0EE409AF0EE609A53EC182B51EC190B39F067F902D2012001E07C
:40A8800001E0002004462046BDEC068B70BD70B52DED068B0024FFF7AFFE70BB2CF0BEFE58B3FFF71EFF40B3FFF7AEF928B3374890EDD70A10EE101A084639F077FC41EC41
:40A8C000180BFEF79DFB10EE105A284639F06EFC41EC1A0BB0EE4A0AF0EE6A0A36F040F8B0EE409AF0EE609A53EC182B51EC190B39F064FA02D2012001E001E00020044670
:40A900002046BDEC068B70BD70B52DED068B0024FFF77AF970B3FFF76FFE58B32CF07EFE40B3FFF7DEFE28B3184890EDD50A10EE101A084639F03AFC41EC180BFFF799FEB6
:40A9400010EE105A284639F031FC41EC1A0BB0EE4A0AF0EE6A0A36F003F8B0EE409AF0EE609A53EC182B51EC190B39F027FA19D2012018E018E0000054080020C52B040803
:40A9800098080020EC080020F00300202021002068520020E12704082C000020842A002094070020002004462046BDEC068B70BD70B52DED068B0024FFF726F988B3FFF71B
:40A9C0001BFE70B3FFF7F5FE58B32CF027FE40B3FFF787FE28B3F74890EDD60A10EE101A084639F0E3FB41EC180BFFF742FE10EE105A284639F0DAFB41EC1A0BB0EE4A0AE6
:40AA0000F0EE6A0A35F0ACFFB0EE409AF0EE609A53EC182B51EC190B39F096F802D2012001E001E0002004462046BDEC068B70BD70B52DED068B0024FFF7E6F880B3FFF72B
:40AA4000DBFD68BB2CF0EAFD50B3FFF74AFE38B3D84890EDD70A10EE101A084639F0A6FB41EC180BFFF705FE10EE105A284639F09DFB41EC1A0BB0EE4A0AF0EE6A0A35F053
:40AA80006FFFB0EE409AF0EE609A53EC182B51EC190B39F093F901D2012000E0002004462046BDEC068B70BD70B52DED068B0024FFF7AAF880B3FFF79FFD68B32CF0AEFD02
:40AAC00050B3FFF70EFE38B3BA4890EDD50A10EE101A084639F06AFB41EC180BFFF7CDFD10EE105A284639F061FB41EC1A0BB0EE4A0AF0EE6A0A35F033FFB0EE409AF0EE56
:40AB0000609A53EC182B51EC190B39F057F901D2012000E0002004462046BDEC068B70BD70B52DED068B0024FFF76EF888B3FFF763FD70B3FFF71AFE58B32CF06FFD40B31C
:40AB4000FFF7CFFD28B39B4890EDD60A10EE101A084639F02BFB41EC180BFFF78EFD10EE105A284639F022FB41EC1A0BB0EE4A0AF0EE6A0A35F0F4FEB0EE409AF0EE609A49
:40AB800053EC182B51EC190B38F0DEFF02D2012001E001E0002004462046BDEC068B70BD70B52DED068B0024FFF72EF880B3FFF723FD68BB2CF032FD50B3FFF792FD38B385
:40ABC0007C4890EDD70A10EE101A084639F0EEFA41EC180BFFF751FD10EE105A284639F0E5FA41EC1A0BB0EE4A0AF0EE6A0A35F0B7FEB0EE409AF0EE609A53EC182B51ECBB
:40AC0000190B39F0DBF801D2012000E0002004462046BDEC068B70BD70B52DED088B0024FEF7F2FFB8B32CF0F9FCA0B3FFF759FD88B3FFF71EFDF0EE400AFFF71EFD30EE4F
:40AC4000800AB0EE408A5B4890EDD80A10EE101A084639F0ABFA41EC190BFFF7FEFC30EE480A10EE105A284639F0A0FA41EC1B0BB0EE4B0AF0EE6B0A35F072FEB0EE40AA9C
:40AC8000F0EE60AA53EC192B51EC1A0B39F096F802D2012001E002E00020044600BF2046BDEC088B70BD444890ED030A704710B50124404890F84A000E281BD03D4890F821
:40ACC0004A00022816D03B4890F84A00152811D0384890F84A001A280CD0364890F84A00032802D12CF07EFC20B9324890F84A00182800D100240CB1012010BD0020FCE72B
:40AD000010B50024FFF778FCB0B12CF087FC98B1FFF7CDFF80B1FFF7E4FC68B1FFF7C3FF2448D0EDD90AB4EEE00AF1EE10FA01DD012000E000200446204610BD10B50024F7
:40AD4000FFF75AFCB0B12CF069FC98B1FFF7AFFF80B1FFF7A8FF1748D0EDDA0AB4EEE00AF1EE10FA04D2FFF7BCFC08B1012000E000200446204610BD10B50024FFF73CFC83
:40AD8000B0B92CF04BFC98B1FFF791FF80B1FFF78AFF0848D0EDDB0AB4EEE00AF1EE10FA04DDFFF79EFC08B1012000E000200446204610BD20210020880C00209B4890EDA4
:40ADC000030A704710B50024FFF716FCB0B12CF025FC98B1FFF76BFF80B1FFF782FC68B1FFF7ECFF9248D0EDD90AB4EEE00AF1EE10FA01DD012000E000200446204610BD4D
:40AE000010B50024FFF7F8FBB0B12CF007FC98B1FFF74DFF80B1FFF764FC68B1FFF7CEFF8348D0EDDA0AB4EEE00AF1EE10FA01D2012000E000200446204610BD10B5002497
:40AE4000FFF7DAFBB0B92CF0E9FB98B1FFF72FFF80B1FFF746FC68B1FFF7B0FF7448D0EDDB0AB4EEE00AF1EE10FA01DD012000E000200446204610BD70B52DED068B0024C7
:40AE80002CF0CCFB88B3FFF712FF70B3FFF729FC58B3674890EDDC0A10EE101A084639F085F941EC180BFFF7FEFEF0EE400AFFF785FF30EEC00A10EE105A284639F076F9BB
:40AEC00041EC1A0BB0EE4A0AF0EE6A0A35F048FDB0EE409AF0EE609A53EC182B51EC190B38F06CFF02D2012001E001E0002004462046BDEC068B70BD10B52DED028B9FEDA6
:40AF00004D0AB0EE408A2CF055FB28B14A4890ED030AB0EE408A11E02CF064FB70B1FFF7C2FEB0EE408AB3EE040AB4EEC08AF1EE10FA03D89FED3F0AB0EE408AB0EE480A52
:40AF4000BDEC028B10BD3D4890EDA40A704710B52DED068BFEF7A1FD20B1FFF7A4FEB0EE408A0CE0324890F84A00032803D1344890ED038A03E0FFF770FBB0EE408A18EE24
:40AF8000100A39F013F941EC1A0BB0EE4A0AF0EE6A0A35F0E5FCB0EE409AF0EE609A9FED290B53EC102B51EC190B38F0CDFD03D89FED200AB0EE408AB0EE480ABDEC068BA6
:40AFC00010BD00B50022FFF717FB90B1FEF765FD78B1FFF7B8FFF0EE400AFFF736FB9FED1B1A20EE010AF4EEC00AF1EE10FA00DD0122104600BD00B50022FFF7FDFA90B161
:40B00000FEF74BFD78B1FFF79EFFF0EE400AFFF71CFB9FED0F1A20EE010AF4EEC00AF1EE10FA00D20122104600BD0000E00C00202021002000000000380D0020EC08002091
:40B04000900D002000000000000034406666663FCDCCCC3D10B501F004FF292002F080FA2A2002F07DFA0EF090F870B1DFF8F0C300DF044604212EF0C7FFDFF8E4C300DFAB
:40B08000044602212EF0C0FF0DE0DFF8D4C300DF044604212EF0D5FFDFF8C4C300DF044602212EF0CEFF10BD10B5EE48C16B01202EF0E4FFEB48C16B0120DFF8ACC300DF5B
:40B0C00010BD10B52DED0C8BB0EE408AE74890ED630AB0EE409AB4EEC98AF1EE10FA02DD01F0A9FE38B9B4EEC98AF1EE10FA2CD201F0A1FE48BBDD4890ED6A0A10EE101A21
:40B10000084639F053F841EC1B0B38EE490A10EE101A084639F04AF841EC1D0BB0EE4D0AF0EE6D0A35F01CFCB0EE40CAF0EE60CA53EC1B2B51EC1C0B38F042FD41EC1A0B72
:40B1400038F0F8F908EE900A3BE0B4EEC98AF1EE10FA02DD01F06FFE38B1B4EEC98AF1EE10FA2CD201F067FE48B3C04890ED6B0A10EE101A084639F019F841EC1B0B38EEB7
:40B18000490A10EE101A084639F010F841EC1D0BB0EE4D0AF0EE6D0A35F0E2FBB0EE40CAF0EE60CA53EC1B2B51EC1C0B38F008FD41EC1A0B38F0BEF908EE900A01E0DFEDC0
:40B1C000AC8A9FEDAC0AF4EEC08AF1EE10FA03DD9FEDA80AF0EE408A9FEDA70AF4EEC08AF1EE10FA03D29FEDA40AF0EE408AB0EE680ABDEC0C8B10BD10B52DED028B2EF04C
:40B20000B3FD9E490860002001F072F9B0EE408AFFF757FF994880ED030A01F03BFBBDEC028B10BD2821954834F015FA01218D4880F82012DFF828C200DF0646012204212C
:40B240002EF09CFEDFF818C200DF0646192202212EF094FEDFF808C200DF064631460120DFF804C200DF03217E4880F8201200BF00224FF6FF710720DFF804C200DF85B248
:40B28000012DF5D0022DF3D1DFF8F8C100DF044604F0040008B101F0D9FB04F0020018B1FFF7AAFFFFF700FF04F001000028DFD0FFF7D0FEDCE710B504466A48D0F81C121C
:40B2C0002046DFF8A4C100DF10BD10B52DED088B664890ED630AD0ED610A30EE600ADFED660A80EE801A11EE104A204638F05EFF41EC1B0BB0EE4B0AF0EE6B0A35F030FBD5
:40B30000B0EE40AAF0EE60AA51EC1A0B38F006F941EC190B38F00EF908EE900A534890ED620AD0ED630A30EE600ADFED520A80EE801A11EE104A204638F038FF41EC1A0B2E
:40B34000B0EE4A0AF0EE6A0A35F00AFBB0EE409AF0EE609A51EC190B38F0ECF808EE100A002001F066FA414890F8300091280ED03E4890F83000922809D03C4890F830003C
:40B38000712804D0394890F83000B8280CD1374890F8B201032807D19FED3B0AB0EE408AB1EE480AF0EE408AB0EE680A01F0B9FAB0EE480A01F0C9FABDEC088B10BD70B515
:40B3C00005460C4601F0F0F9284600F019FE204600F02EFEFFF779FF64201BF04AFB0120FFF769FF70BD2548D0ED030AB0EE600A7047224890F82400042801D00120704710
:40B400000020FCE70220704710B52DED088BB0EE408A18EE100A38F0C9FE41EC190BFFF7E2FF10EE104A204638F0C0FE41EC1B0BB0EE4B0AF0EE6B0A35F092FAB0EE40AAA9
:40B44000F0EE60AA53EC192B51EC1A0B38F07CFB03D20120BDEC088B10BD0020FAE700002134040868520020E127040820210020000000000000C8420000C8C2D01C002010
:40B480004128040889270408D051863910B501F0E8FC292002F064F82A2002F061F80DF0ADFE70B1DFF828C400DF044604212EF0ABFDDFF81CC400DF044602212EF0A4FD53
:40B4C0000DE0DFF80CC400DF044604212EF0B9FDDFF8FCC300DF044602212EF0B2FD10BD10B5FC48C16B01202EF0C8FDF948C16B0120DFF8E4C300DF10BDF0EE400AF748C2
:40B50000D0ED631AB0EE611AD0ED611AF4EEC11AF1EE10FA1FD2F4EEC10AF1EE10FA08D2D0ED671A90ED6A2AB0EE610A02EE200A31E0F4EEC10AF1EE10FA09DBE748D0ED90
:40B54000691A90ED6B2AB0EE610A02EE200A22E09FEDE30A1FE0F4EEC10AF1EE10FA09D2DE48D0ED691A90ED6B2AB0EE610A02EE200A10E0F4EEC10AF1EE10FA09DBD74804
:40B58000D0ED671A90ED6A2AB0EE610A02EE200A01E09FEDD30A7047D048B0F9A0037047CE48B0F9A2037047CE49097D31B1012906D0022906D0032906D106E0002006E073
:40B5C000012004E0022002E000BF032000BF00BF704710B52DED028BFFF7E6FF10B9FFF7DFFF01E0FFF7D8FF08EE100A2EF0BCFBBD490860002000F07BFFF0EE408AFFF71E
:40B600007CFFB94880ED030A90ED030AF8EEC80A30EE600A80ED030A01F03CF9BDEC028B10BD2C21B04834F016F80121A94880F83412DFF89CC200DF0646012204212EF099
:40B640009DFCDFF88CC200DF0646192202212EF095FCDFF87CC200DF064631460120DFF878C200DF03219B4880F8341200BF00224FF6FF710720DFF874C200DF85B2012D39
:40B68000F5D0022DF3D1DFF868C200DF044604F0040008B101F0DAF904F0020018B1FFF798FFFFF71DFF04F001000028DFD0FFF7EDFEDCE710B504468648D0F83012204618
:40B6C000DFF814C200DF10BD8448B0F8900370478248B0F88E0370478048B0F88C03704710B52DED048BFFF7EFFF0146FFF7F4FF081A00EE100AB8EEC00A7848D0ED630ABD
:40B7000090ED611A70EEC10A80EE201AB0EE418AFFF7DEFF0146FFF7D7FF081A00EE100AB8EEC00A6D48D0ED620A90ED631A70EEC10A80EE201AF0EE418AFFF7C5FF00EE5D
:40B74000100AB8EE400A6548D0ED630A08EE600AB0EE409AFFF7B8FF00EE100AB8EE400A5E48D0ED630A08EEE00AF0EE409A002001F05FF8B0EE480A01F0D3F8B0EE680ADF
:40B7800001F0E3F8B0EE490A01F0F3F8B0EE690A01F003F9BDEC048B10BD70B505460C4601F002F8284600F02BFC204600F040FCFFF796FF0120FFF77DFF70BD4A48D0ED8F
:40B7C000030AB0EE600A7047474890F82400042801D0012070470020FCE70220704773B50D46002400BF022269464248006800F563700FF08DFE20B9BDF800003749A1F875
:40B800008C0300BF5C2001F0ABFE20467CBD73B50D46002400BF022269463648006800F28E300FF075FE20B9BDF800002B49A1F88E0300BF5D2001F093FE20467CBD31B55D
:40B84000002400BF022269462A48006800F564700FF05EFE20B9BDF800002049A1F8900300BF5E2001F07CFE204638BD31B5002400BF022269461F48006800F292300FF0D0
:40B8800047FE20B9BDF800001449A1F8920300BF622001F065FE204638BD1048B0F89203704731B5002400BF022269461148006800F565700FF02CFE20B9BDF800000749C0
:40B8C000A1F8940300BF682001F04AFE204638BD2134040868520020E12704082021002000000000CC2A0020282A00204128040889270408F00300205648B0F8940370472D
:40B9000031B5002400BF012269465348006800F567700FF0FDFD20B9BDF800004D4981F89C0300BF692001F01BFE204638BD494890F89C03704731B5002400BF01226946B1
:40B940004548006800F29E300FF0E2FD20B9BDF80000404981F89E0300BF632001F000FE204638BD3B4890F89E03704731B5002400BF022269463848006800F568700FF0C4
:40B98000C7FD20B9BDF900003249A1F8A00300BF6D2001F0E5FD204638BD31B5002400BF022269462C48006800F2A2300FF0B0FD20B9BDF900002749A1F8A20300BF6C2093
:40B9C00001F0CEFD204638BD10B52DED0C8BB0EE408AFFF779FE044638F0A2F841EC1A0BFFF772FE00EE100AB8EE401AFFF7E6FE31EE400A10EE104A204638F0D7FB41ECF1
:40BA00001D0BB0EE4D0AF0EE6D0A34F0A9FFB0EE40CAF0EE60CA9FED110B53EC102B51EC1C0B38F0CDF841EC1B0B53EC1A2B37F06FFE41EC190B37F07DFD08EE900AF4EED6
:40BA4000C88AF1EE10FA03D20120BDEC0C8B10BD0020FAE720210020F0030020000000000000594010B52DED028BB0EE408ABE4880ED008A2EF078F9BC490860BDEC028B77
:40BA800010BD10B52DED088BB0EE408A9FEDB80AF0EE408AB3EE040AB0EE40BA18EE100A38F084FB41EC1A0BB0EE4A0AF0EE6A0A34F056FFB0EE409AF0EE609A9FEDAD0B38
:40BAC00053EC102B51EC190B38F078F90ED2B3EE040A38EE400ADFEDA90A80EE201AB3EE040A21EE000AF0EE408A03E09FEDA00AF0EE408AB0EE680ABDEC088B10BD10B59D
:40BB00002DED048B04469FED9A0AB0EE408A9FED980AF0EE408A9A4890F83000922804D0974890F83000932875D1954890F8FF0102280ED0924890F8FF01032809D0904839
:40BB400090F8300092280BD08D4890F83000932806D0864800682EF02FF9B0F57A7F03D300208849087001E086480470864800682EF022F9C8284ED3814890F830001D2898
:40BB80004AD18048007828B1774890ED000AB0EE408A15E07D4800782BF014FF00EE100AB8EE400ADFED7A0A30EE600ADFED790A80EE201AB2EE0E0A21EE000AB0EE408A43
:40BBC000754890ED000A78EE400A744890ED000A9FED731A01EE200A80ED000A062025F039FB44B114F0F4FFB0EE409AFFF749FFF0EE408A03E001F088FCF0EE408A6948FB
:40BC000090ED000A30EE280A674880ED000A052025F020FB2CE049E05A48007828B1524890ED000AB0EE408A15E0584800782BF0C9FE00EE100AB8EE400AF3EE040A70EECD
:40BC4000600A9FED541A80EE810AF2EE0E0A20EE200AB0EE408A504890ED000A78EE400A90ED000A9FED4E1A01EE200A80ED000A2EF07AF844490860414890F8FF01022835
:40BC800004D03F4890F8FF0103280CD13C4890F83000922804D03A4890F83000932802D1042025F0D7FA072025F0D4FABDEC048B10BD394890ED000A704701B500BF012297
:40BCC00069463A48006800F2FF100FF021FC20B99DF800002A4981F8FF0100BF08BD224890ED000A70472D4890ED000A70472E4890ED000A70472B4890ED000A7047F0B54B
:40BD00000546059C0E78022E02D0042E28D113E08F78487867F31F2000EE100AB8EE400ADFED230A30EE600ADFED220A80EE201A1C4E86ED001A14E08F78487867F31F20AD
:40BD400000EE100AB8EE400ADFED190A30EE600ADFED180A80EE201A0F4E86ED001A00E000BF00BFF0BD000000040020180400200000000000000000000034400000A04213
:40BD800020210020140400201C0400205507002000004842000080450C040020040400209A99993E1004002008040020F00300200000FB4600007A4488B001680791416829
:40BDC000069181680591C1680491016903914169029181690191C169009108B0704700000C48016841F4700101600B4880470B480047FEE7FEE7FEE7FEE7FEE7FEE7FEE7D3
:40BE0000FEE7FEE7FEE7000005480649064A074B7047000088ED00E0E9E70308AD81000818FC0020C0D9012018FE0020C0D501207047704770471DF0D5BE704700000000A2
:40BE40000000000000000000000000000000000000000000000000000000000000000000000000000000000000000000526176656E20496E647573747269657320496E6342
:40BE80000000000000000000000000004175672D31382D32303138000000000032322E332E302E3700000000000000005374656572696E6720436F6E74726F6C20556E69C1
:40BEC0007400000000000000000000003037373031373135303200000000000000000000000000000000000000000000FFFFFFFFFFFFFFFFFFFFFFFFFFFFFFFFFFFFFFFFE4
:40BF0000FFFFFFFFFFFFFFFFFFFFFFFFFFFFFFFFFFFFFFFFFFFFFFFFFFFFFFFFFFFFFFFFFFFFFFFFFFFFFFFFFFFFFFFFFFFFFFFFFFFFFFFFFFFFFFFFFFFFFFFFFFFFFFFF41
:40BF4000FFFFFFFFFFFFFFFFFFFFFFFFFFFFFFFFFFFFFFFFFFFFFFFFFFFFFFFFFFFFFFFFFFFFFFFFFFFFFFFFFFFFFFFFFFFFFFFFFFFFFFFFFFFFFFFFFFFFFFFFFFFFFFFF01
:40BF8000FFFFFFFFFFFFFFFFFFFFFFFFFFFFFFFFFFFFFFFFFFFFFFFFFFFFFFFFFFFFFFFFFFFFFFFFFFFFFFFFFFFFFFFFFFFFFFFFFFFFFFFFFFFFFFFFFFFFFFFFFFFFFFFFC1
:40BFC000FFFFFFFFFFFFFFFFFFFFFFFFFFFFFFFFFFFFFFFFFFFFFFFFFFFFFFFFFFFFFFFFFFFFFFFFFFFFFFFFFFFFFFFF00C00008FFFF030800800008FBBF0008622B1BA406
:40C0000001B500BF01226946FE48006800F5D9700FF07EFA20B99DF80000FB4981F8B20100BF02201AF051FB0120FFF744F908BD01B500BF01226946F248006800F2B3108A
:40C040000FF066FA20B99DF80000EF4981F8B30100BF02201AF039FB0120FFF72CF908BD70B52DED068BB0EE408AF0EE608A04460425E54890F8B201E4490978884206D144
:40C08000E14890F8B301E249097888427ED0DE4890F8B2010C287CD2DFE800F05D213E06595A5B5C073C3D5E00BF9FEDDA0ADA4880ED000A9FEDD70AD84880ED000A9FED5B
:40C0C000D50AD74880ED000A9FEDD20AD54880ED000A0120D4490870D449087059E0B6EE000ACD4880ED000A9FEDD10ACB4880ED000A9FEDC80ACA4880ED000A9FEDC50ADE
:40C10000C84880ED000A0120C74908700020C74908703EE000BF00BF9FEDC60ABE4880ED000A9FEDC50ABD4880ED000A9FEDB90ABB4880ED000A9FEDB70ABA4880ED000A4C
:40C140000120B94908700020B849087021E000BF00BF00BF00BF00BF9FEDAE0AAE4880ED000A9FEDAC0AAD4880ED000A9FEDA90AAB4880ED000A9FEDA70AAA4880ED000A21
:40C180000120A94908700020A84900E002E0087000BF00BFA448007808B900254CE0A3480078012804D1FEF76CFA50B3002543E03CB99A4890ED000AB4EEC08AF1EE10FA7B
:40C1C00009DC012C09D1974890ED000AB4EEC08AF1EE10FA01DD01252EE03CB98E4890ED000AB4EEC08AF1EE10FA09D3012C09D18B4890ED000AB4EEC08AF1EE10FA01D2FA
:40C20000002519E018EE900A37F0D0FF41EC1A0BB0EE4A0AF0EE6A0A34F0A2FBB0EE409AF0EE609A9FED850B53EC102B51EC190B37F0C4FD00D203252846BDEC068B70BDF5
:40C2400031B52DED020B044600BF042269466D48006800F5C2700FF05BF920B99DED000A694880ED610A00BF0CF08FFF10B1FFF72CF808E00CF0C2FF10B1FFF731FA02E0B9
:40C2800001201AF01BFB212024F0E4FF01203EBD31B52DED020B2DED088B044694B300209FED680A19F0BAF810EE105A284637F07DFF41EC1B0BB0EE4B0AF0EE6B0A34F08F
:40C2C0004FFBB0EE40AAF0EE60AA51EC1A0B37F031F908EE100A4C4890EDE20A30EE480AF0EE408A90EDE20A30EE080AB0EE409A9DED080AB4EEC90AF1EE10FA03DD8DED47
:40C30000089A09E009E09DED080AB4EEE80AF1EE10FA01D2CDED088A0FE000BF042208A93848006800F562700FF0F2F820B99DED080A354880EDE20A00BF00BF042208A994
:40C340003048006800F5C6700FF0E2F820B99DED080A2D4880ED630A00BF0CF016FF10B1FEF7B3FF08E00CF049FF10B1FFF7B8F902E002201AF0A2FA212024F06BFF0120BF
:40C38000BDEC088B3EBD31B52DED020B044600BF042269461B48006800F5C4700FF0B8F820B99DED000A184880ED620A00BF0CF0ECFE10B1FEF789FF08E00CF01FFF10B16C
:40C3C000FFF78EF902E003201AF078FA212024F041FF01203EBD014600200B2955D2DFE801F054494A06474854543B4546009FED161AC0EE010A9FED151A70EE810AFCEE27
:40C40000E00A25E0F0030020202100205800002059000020000000005C0000206000002064000020680000206C0000206D00002066664640CDCCCC3C33339F40000000004F
:40C4400000406F4035FA0E3D0000AF4300401C4510EE902A90B21AE05FED040A70EE200AFCEEE00A10EE902A90B210E000BF00BF00BF00BF00BFDFEDFC0A60EE200AFCEE3D
:40C48000E00A10EE902A90B201E0002000BF00BF7047014600200B2926D2DFE801F0251A1B0618192525101617005FED190A80EE201AFDEEC10A10EE902A10B216E0FCEED8
:40C4C000C00A10EE902A10B210E000BF00BF00BF00BF00BFDFEDE40A60EE200AFDEEE00A10EE902A10B201E0002000BF00BF70475FED380AB0EE600A28B9DC49D1ED560ADC
:40C50000B0EE600A06E0012804D1D849D1ED990AB0EE600A704770B52DED0A8BB0EE408A9FEDD30AC8EE000A10EE905AD14890ED610AF0EE408A90ED630AB0EE409A002056
:40C54000FFF7D6FFF0EE409A284637F02FFE41EC1A0B38EEE90A78EEC90A80EE201A11EE106A304637F022FE41EC1C0BB0EE4C0AF0EE6C0A34F0F4F9B0EE40BAF0EE60BAB7
:40C5800053EC1A2B51EC1B0B37F0DEFA01D2012000E0002004462046BDEC0A8B70BD70B52DED0A8BB0EE408A9FEDB10AC8EE000A10EE905AAF4890ED620AF0EE408A90ED56
:40C5C000630AB0EE409A0020FFF792FFF0EE409A284637F0EBFD41EC1A0B38EEE90A78EEC90A80EE201A11EE106A304637F0DEFD41EC1C0BB0EE4C0AF0EE6C0A34F0B0F9D4
:40C60000B0EE40BAF0EE60BA53EC1A2B51EC1B0B37F09AFA01D2012000E0002004462046BDEC0A8B70BD70B52DED0C8BF0EE408A9FED8F0AC8EE800A10EE904A8D4890EDAC
:40C64000620AF0EE409A90ED610AB0EE40AA90ED630AB0EE408A0020FFF74AFFB0EE409A204637F0A3FD41EC1B0B39EE480A7AEE480A80EE201A11EE106A304637F096FDF9
:40C6800041EC1D0BB0EE4D0AF0EE6D0A34F068F9B0EE40CAF0EE60CA53EC1B2B51EC1C0B37F052FA24D2204637F080FD41EC1B0B39EE480A79EEC80A80EE201A11EE106A24
:40C6C000304637F073FD41EC1D0BB0EE4D0AF0EE6D0A34F045F9B0EE40CAF0EE60CA53EC1B2B51EC1C0B37F02FFA01D2012000E0002005462846BDEC0C8B70BD5B4890F8FE
:40C700005000042801D0012070470020FCE710B50124FFF7F3FF28B95449C86A64212DF029FB00B10024204610BD504890F82800042801D0012070470020FCE710B5012477
:40C74000FFF7F3FF28B94949486864212DF012FB00B10024204610BD10B5FFF7EFFF10B1FFF7D5FF08B9022411E0424890ED6A0AB5EEC00AF1EE10FA08D090ED6B0AB5EEAD
:40C78000C00AF1EE10FA01D0012400E00024204610BD18B9354991ED080A04E0012802D1324991ED120A704710B50021324800782FF034FB0021314800782FF02FFB2D4818
:40C7C00090F8B201032802D0082820D10FE000209FED2B0AFFF734FD00201FEDF20AFFF757FD00209FED270AFFF7CDFD1FE000209FED250AFFF724FD00201FEDFA0AFFF7C3
:40C8000047FD00209FED210AFFF7BDFD0FE00020B6EE000AFFF714FD0020B0EE040AFFF737FD0020B1EE020AFFF7ADFD00BF00BF10BD01B50F4890F8410001280FD000BF20
:40C84000012269461248006800F2B5100EF060FE20B99DF80000074981F8B50100BF212024F0F8FC08BD000000007A44E80D00200000C84220210020540700205307002024
:40C8800090ED24C990ED244900803BC500803B45F003002010B52DED028B044694ED030AD4ED040A30EE600A84ED060A94ED030A84ED040A2DF058FA2060D4E90001401A61
:40C8C000A06094ED020AB8EE400A5FED190A80EE201AB0EE418A20686060B5EEC08AF1EE10FA1BDD94ED060AC0EE080AC4ED050A0CF080FB48B1D4ED050AB0EE600AC821E3
:40C9000004F11C001AF01DFF08E0D4ED050AB0EE600A042104F11C001AF013FFBDEC028B10BD10B52DED020B00BF04226946FA48006800F5D4700EF0EBFD20B99DED000AF5
:40C94000F64880ED6A0A00BF1CBD10B52DED020B00BF04226946F048006800F5D6700EF0D7FD20B99DED000AEC4880ED6B0A00BF1CBD10B52DED020B00BF04226946E6480A
:40C98000006800F5CE700EF0C3FD20B99DED000AE24880ED670A00BF1CBD10B52DED020B00BF04226946DC48006800F5D2700EF0AFFD20B99DED000AD84880ED690A00BFF8
:40C9C0001CBD19B9D64A82F8280004E0012902D1D34A82F85000704710B52DED088BB0EE408A9FEDD00AF0EE408AB3EE040AB0EE40BA18EE100A37F0D9FB41EC1A0BB0EE11
:40CA00004A0AF0EE6A0A33F0ABFFB0EE409AF0EE609A9FEDC50B53EC102B51EC190B37F0CDF90AD21FED6E0AC8EE000A9FEDC00A20EE800AF0EE408A03E09FEDBA0AF0EE48
:40CA4000408AB0EE680ABDEC088B10BD10B52DED028BB34890F86D02012816D0AF4890F84B00AF4981F86C02084690F86C1254301AF056FEAA4890F86C1200F5B0701AF070
:40CA80004FFE0120A64981F86D02A44890F8B2010B287DD2DFE800F0FE06162AFDFCFBFA2B3BB400A34800782AF08CFF00EE100AB8EE400ADFEDA00A20EE200A984880ED8A
:40CAC000040A03E19B4800782AF07CFF00EE100AB8EE400ADFED980A20EE200ADFED970A80EE201A8E4880ED041AEFE000BF914800782FF000F900EE100AB8EEC00A884801
:40CB0000D0ED000A30EE200A80ED040ADEE00AF025FF10B90AF0D7FD18B3FDF75BFDB0EE408AFFF759FF864880ED000A854800682DF042F900EE100AB8EE400A5FEDB60A55
:40CB400080EE201A804880ED001A7D4890ED000A7D48D0ED000A20EE200A7C4880ED000A20E0744800782FF0C6F800EE100AB8EEC00A7748D0ED000A30EE600A5FEDC60AC0
:40CB800080EE201A714880ED001A6A48007800E094E02FF0B0F800EE100AB8EEC00A6C4880ED000A2DF0E0F8664908605C4890ED040A6648D0ED000A30EE200AF6EE000ABF
:40CBC000B4EEE00AF1EE10FA19DD554890ED040A5E48D0ED000A30EE200AF1EE020AB4EEE00AF1EE10FA0AD24D4890ED040A5748D0ED000A30EE200A494880ED040A65E092
:40CC0000FFF779F8B2EE041AC0EE010AB0EE040A30EE800A424880ED040A464800782FF06AF800EE100AB8EEC00A4948D0ED000A30EE600A5FEDF40A80EE201A404880EDF7
:40CC4000001A3C4800782FF056F800EE100AB8EEC00A3F4880ED000A3A4800682DF0ACF800EE100AB8EE400ADFED3A0A80EE201A354880ED001A324890ED000A3248D0ED24
:40CC8000000A20EE200AF1EE040A04E018E00FE008E006E013E020EE200A2F4880ED000A14E000BF9FED1F0A1D4880ED040A0DE09FED1C0A1A4880ED040A07E000BF00BF6A
:40CCC0009FED180A164880ED040A00BF00BF144890F86C12D0ED040AB0EE600A54301AF0CBFC0F48001DFFF7D5FD0D4890ED081AF0EE410A90ED041AB0EE410A0020FFF7B2
:40CD0000AFF904460021FFF75CFE044890F8B3010B2866D222E00000F003002020210020E80D0020000000000000000000003440713DAA3F540700203333533A0CAC233F7F
:40CD400070000020800000207C000020780000207400002000007A4454000020DFE800F0420616312A2B3B3532333400FE4800782AF028FE00EE100AB8EE400A5FED120A87
:40CD800020EE200AF94880ED0E0A31E0F64800782AF018FE00EE100AB8EE400A5FED1A0A20EE200A5FED1B0A80EE201AEF4880ED0E1A1DE000BF1FED250AEC4880ED0E0A49
:40CDC00016E000BF00BF00BF00BF1FED2A0AE74880ED0E0A0CE01FED2D0AE44880ED0E0A06E000BF1FED310AE04880ED0E0A00BF00BFDE4890F86C12D0ED0E0AB0EE600A4D
:40CE000000F5B0701AF038FCD8482C30FFF742FDD64890ED121AF0EE410A90ED0E1AB0EE410A0120FFF71CF904460121FFF7C9FDBDEC028B10BDCE4890ED610AD0ED630AF1
:40CE400030EE600AB5EEC00AF1EE10FA01DD012070470020FCE7B0EE040AC44880ED040A704730B589B02AF0D0FB40B10021084619F011FD0121002019F00DFD2AE0BC4854
:40CE800090F8B201032804D0B94890F8B201082808D10021032019F0FEFC0121032019F0FAFC17E0B24890F8B20109280AD10021032019F0F0FC0121032019F0ECFCFFF7CB
:40CEC000CAFF07E00021032019F0E5FC0121002019F0E1FCA64890F8B25190F8B3410B2D7ED2DFE805F08C06182A8E8F608D2B2C2D000020009001900290034603229D496A
:40CF00000390084600782AF06EFC0321994800782BF017F888E000200090019002900346032294490390084600782AF05CFC0021904800782BF005F876E000BF00BF00BF00
:40CF400000200090019002900346022289490390084600782AF047FC0221864800782AF0F0FF2AF027FB68B183485FED920A9FED830A04230022824900907E4800782EF056
:40CF8000C1FB0FE02AF02EFB60B17B485FED9B0A9FED7A0A0423002219070090754800782EF0B0FB40E000200090019002900346022270490390084600782AF014FC0621F4
:40CFC0006C4800782AF0BDFF002000900190022314220121029004A82EF0ACFC04A800E00DE05FEDB00A9FED670A032300224FF0804100905F4800782EF084FB14E000BFAA
:40D0000000BF00BF00200090019002900346032258490390084600782AF0E5FB0121554800782AF08EFF00BF00BF0B2C7ED2DFE804F08B06182A8D8E608C2B2C2D00002021
:40D040000090019002900346032247490390084600782AF0C8FB0321434800782AF071FF9AE00020009001900290034603223E490390084600782AF0B6FB00213A48007897
:40D080002AF05FFF88E000BF00BF00BF00200090019002900346022233490390084600782AF0A1FB0221304800782AF04AFF2AF081FA68B130485FEDE50A9FED300A0423C4
:40D0C00001222F490090284800782EF01BFB0FE02AF088FA60B128485FEDEE0A9FED270A04230122910700901F4800782EF00AFB52E00020009001900290034602221A4993
:40D100000390084600782AF06EFB0621164800782AF017FF002000900190034614220121029004A82EF006FC04A800E00CE0DFED160A9FED120A02230122910700900A48D8
:40D1400000782EF0DFFA27E000BF00BF00BF00200090019002900346032203490390084600782AF040FB11E053070020E80D0020202100205407002070EC0020809FD54AAB
:40D1800000040140A037A04C000000000121E14800782AF0D6FE00BF00BF09B030BD10B5DD4988684FF496712CF0E4FD10BDDB4890ED000A704710B52DED048B19F01EFBB2
:40D1C00010EE104A204636F0F1FF41EC190BB0EE490AF0EE690A33F0C3FBB0EE408AF0EE608A9FEDCF0B53EC102B51EC180B36F0ABFC03D20120BDEC048B10BD0020FAE7AE
:40D20000C94991F84110012901D1012007E0C64991F8B51109B1012100E000210846704710B52DED068BB0EE408AC048007838B91FED2B0ABE4880ED000A0120BB4908701A
:40D24000FFF7DEFF00287ED0FFF7B5FF18B90AF085FB002877D0FFF7AAFF10EE104A204636F0A4FF41EC1A0BB0EE4A0AF0EE6A0A33F076FBB0EE409AF0EE609A9FEDAD0B1D
:40D2800053EC102B51EC190B36F05EFC5BD2FFF786FF002857D123F08BFADFEDA80AB4EEE00AF1EE10FA4EDBFFF756FA01284AD19D4890F83000912845D09B4890F83000D7
:40D2C000922840D0984890F8300071283BD0964890F83000B82836D0934890F8B2010B282AD2DFE800F029121306141529290708160000BF00BF8E4890ED000ADFED900A7B
:40D3000008EE200A80ED000A1CE000BF00BF00BF00BF8548D0ED630A9FED891A48EE410AB0EE600A0120FEF7B3FF1FED690A804880ED000A06E006E01FED6D0A7C4880EDA9
:40D34000000A00BF00BFBDEC068B10BD784890F8280008B9012070470020FCE7744890F82800012800D170470020FCE7704890F82800032801D1012070470020FCE76C48FE
:40D3800090F8500008B9012070470020FCE7684890F85000012800D170470020FCE7644890F85000032801D1012070470020FCE700B50021FFF7CAFF08B13D2103E0FFF7DC
:40D3C000CDFF00B13C21084600BD00B50021FFF7CDFF08B1082117E0FFF7B8FF08B1072112E0FFF7BBFF08B106210DE0FFF7D7FF08B10B2108E0FFF7A9FF08B10A2103E0DC
:40D40000FFF7ACFF00B10921084600BD10B519F018FB0446204610BD10B52DED028B0BF0B4FE20B1FDF7DFFFB0EE408A16E019F0E1F93D48D0ED640A30EE600ADFED410ABB
:40D4400020EE200AD0ED650A90ED641A70EEC10A80EE201A9FED3C0A31EE008AB0EE480ABDEC028B10BD01B59DF80000202801DD2020009000BF01226946344800684B30DD
:40D480000EF046F820B99DF80000274981F84B0000BF0020264981F86D0208BD10B54FF41C71234832F0D7F810BD29490870704727480078704710B52DED028BB0EE408AC2
:40D4C0002448007830B9154800210160416001202049087023F068F9F0EE408AF0EE680AB0EE480A19F07DF81B4880ED000A28210A48194A92ED000A1AF023F9BDEC028B46
:40D5000010BD154890ED000A7047144890ED000A70470000530700209C5500204C000020000000A046DF913F2021002084000020E80D0020000000A046DF813F2FDDE43E90
:40D540000AD7A33B000048430000C8C2F00300204400002085000020480000205400002010B50446204625F029FA10BD07B586B000200490002108980170069800786F28E0
:40D5800081F0AF82DFE810F06F007100ED000D013B01AD0AB10050075B0766076901CF01E1014702BC0211036603B303080470045D048200BD042F059D05E3053206B00637
:40D5C0000D09CA0671079B097D07C307D20710081E082C0872087E088E089808A808AD0AAD0AAD0AB808C908E308890795079F07B707AB07AD0AAD0AAD0AAD0AAD0AAD0A7D
:40D60000AD0AAD0AAD0AAD0AAD0AD404AD0AAD0AAD0A1109390956097E09AD0AAD0AAD0AAD0AAD0AAD0AAD0AAD0AAD0AAD0AAD0AAD0AAD0AAD0AAD0AAD0AAD0AAD0AAD0A83
:40D64000AB09DC090D0AAD0AAD0AAD0A1F0A670AAD0AAD0AAD0AAD0A310A430AAD0A550A790A8B0A9D0A01F040BAF94890F841000390069890ED010ABCEEC00A10EE100AC8
:40D68000C0B20290039919F006F9ECE70698007A032803D006210898017025E0069890ED010AF7EE000AB4EE600AF1EE10FA02D117F0F9F918E0069890ED010AF0EE000AC0
:40D6C000B4EE600AF1EE10FA02D117F0D4F90BE0069890ED010AF0EE080AB4EE600AF1EE10FA01D116F0CBFFBDE70698007A032809D1069890ED010A8DED030A9DED030AF1
:40D7000010F074F82AE00698007A012811D1D048B0F8BE110A22079802FB001000EE100AB8EEC00A8DED030A9DED030A10F05EF814E00698007A022810D1C548B0F8BE1162
:40D740000A22079802FB101000EE100AB8EEC00A8DED030A9DED030A10F048F80120049081E70AF0FBF8C0B90698007A032811D1069890ED010A8DED030A9DED030A0BF004
:40D7800018F9B448D0F81801014603908020DFF8C8C200DF0120049002E001210898017061E716F0DFFA30BB0698007A03281ED1069890ED010ABCEEC00A10EE100A80B2CF
:40D7C00003900BF0D4F80BF052F880B90821A348DFF88CC200DF012809D0A248406840F00100A04948609D48DFF87CC200DF182023F030FD02E001210898017033E716F05D
:40D80000B1FA30BB0BF033F818B30698007A03281BD1069890ED010ABCEEC00A10EE100AC0B203900BF07DF808218C48DFF830C200DF012809D08B48406840F001008949E6
:40D8400048608648DFF820C200DF182023F002FD02E001210898017005E70698007A032817D17B4890F842000390794890F841000290069890ED010ABCEEC00A10EE100A36
:40D88000C0B20190DDE9021213F000FA0899087046E00698007A01281FD16D4890F841105C3000EB41006A4991F84210415C0122079802FB0010C0B20190654890F8420064
:40D8C0000390634890F8410002900146039A019813F0DCF90899087022E00698007A02281ED15B4890F841105C3000EB4100584991F84210415C0122079802FB1010C0B250
:40D900000190534890F842000390514890F8410002900146039A019813F0B8F908990870012004909FE60698007A03280CD1069890ED010ABCEEC00A10EE100AC0B203900F
:40D9400013F0E0F9089908708DE60698007A032817D13F4890F8420003903D4890F841000290069890ED010ABCEEC00A10EE100AC0B20190DDE9021213F004FA08990870A7
:40D9800046E00698007A01281FD1314890F84110603000EB41002E4991F84210415C0122079802FB0010C0B20190294890F842000390274890F8410002900146039A01982C
:40D9C00013F0E0F90899087022E00698007A02281ED11F4890F84110603000EB41001C4991F84210415C0122079802FB1010C0B20190174890F842000390154890F8410062
:40DA000002900146039A019813F0BCF9089908700120049027E60698007A032826D10C4890F8420003900A4890F841000290069890ED010ABCEEC00A10EE100AC0B20190F7
:40DA4000DDE9021213F0DBF90899087055E000002021002068520020E127040848320020A92C040858320020C52B04080698007A01281FD1FB4890F84110643000EB41002A
:40DA8000F84991F84210415C0122079802FB0010C0B20190F34890F842000390F14890F8410002900146039A019813F0A8F90899087022E00698007A02281ED1E94890F889
:40DAC0004110643000EB4100E64991F84210415C0122079802FB1010C0B20190E14890F842000390DF4890F8410002900146039A019813F084F90899087001200490B2E522
:40DB00000698007A032810D1D64890F842000390069890ED010A8DED020A03989DED020A13F0CBFA089908703CE00698007A01281AD1CC4890F842107C3000EB8100D0ED7D
:40DB4000000A9DED070AB8EEC00A30EEC00A8DED020AC44890F8420003909DED020A13F0ACFA089908701DE00698007A022819D1BC4890F842107C3000EB8100D0ED000A7B
:40DB80009DED070AB8EEC00A30EE800A8DED020AB44890F8420003909DED020A13F08DFA08990870012004905DE50698007A032810D1AC4890F842000390069890ED010A08
:40DBC0008DED020A03989DED020A13F0BCF9089908703CE00698007A01281AD1A14890F842106C3000EB8100D0ED000A9DED070AB8EEC00A30EEC00A8DED020A994890F8E1
:40DC0000420003909DED020A13F09DF9089908701DE00698007A022819D1924890F842106C3000EB8100D0ED000A9DED070AB8EEC00A30EE800A8DED020A8A4890F8420046
:40DC400003909DED020A13F07EF9089908700120049008E50698007A032812D1814890F842000390069890ED010ABCEEC00A10EE100AC0B20290039913F0FFF80899087095
:40DC800032E00698007A012815D1764890F842106830415C0122079802FB0010C0B20290704890F8420001460390029813F0E5F80899087018E00698007A022814D16948CC
:40DCC00090F842106830415C0122079802FB1010C0B20290634890F8420001460390029813F0CBF80899087001200490BBE40698007A032810D15B4890F842000390069854
:40DD000090ED010A8DED020A03989DED020A13F032FA089908703CE00698007A01281AD1504890F84210843000EB8100D0ED000A9DED070AB8EEC00A30EE800A8DED020A82
:40DD4000484890F8420003909DED020A13F013FA089908701DE00698007A022819D1414890F84210843000EB8100D0ED000A9DED070AB8EEC00A30EEC00A8DED020A39488A
:40DD800090F8420003909DED020A13F0F4F9089908700120049066E40698007A032810D1304890F842000390069890ED010A8DED020A03989DED020A13F023F9089908705A
:40DDC0003CE00698007A01281AD1264890F84210743000EB8100D0ED000A9DED070AB8EEC00A30EE800A8DED020A1E4890F8420003909DED020A13F004F9089908701DE014
:40DE00000698007A022819D1164890F84210743000EB8100D0ED000A9DED070AB8EEC00A30EEC00A8DED020A0E4890F8420003909DED020A13F0E5F8089908700120049037
:40DE400011E40698007A03280AD1069890ED010ABCEEC00A10EE100AC0B20390FCF797FA13E40000202100200698007A032812D1F74890F842000390069890ED010ABCEE6A
:40DE8000C00A10EE100AC0B20290039913F028F80899087032E00698007A012815D1EC4890F842106A30415C0122079802FB0010C0B20290E64890F84200014603900298E7
:40DEC00013F00EF80899087018E00698007A022814D1DF4890F842106A30415C0122079802FB1010C0B20290D94890F8420001460390029812F0F4FF0899087001200490A4
:40DF00002EE40698007A032803D00621089801700DE0069890ED010A8DED030A9DED030A0A2009F099FB10B901210898017017E40698007A032814D1069890ED010ABCEEAA
:40DF4000C00A10EE100A80B200EE100AB8EE400A8DED030A9DED030A0FF048FC089908703EE00698007A01281BD110F000FAF0EE400AB748B0F8BE0100EE100AB8EE401A40
:40DF80009DED070AF8EE401AB0EE410A00EEA10A8DED030A9DED030A0FF028FC089908701EE00698007A02281AD110F0E0F9F0EE400AA748B0F8BE0100EE100AB8EE401A20
:40DFC0009DED070AF8EE401AB0EE410A00EEE10A8DED030A9DED030A0FF008FC08990870012004900AE40698007A032815D1984890F842000390964890F84100029006986A
:40E0000090ED010A8DED010ADDE902019DED010A12F0EBFD0899087050E00698007A012824D18B4890F842000290894890F841000190029910F092FFDDED070AF8EE600A5B
:40E040009FED841A01EE200A8DED030A804890F8420002907E4890F84100019002999DED030A12F0C2FD0899087027E00698007A022823D1764890F842000290744890F8EB
:40E0800041000190029910F069FFDDED070AF8EE600A9FED701A01EE600A8DED030A6C4890F8420002906A4890F84100019002999DED030A12F099FD0899087001200490B6
:40E0C00030E40698007A03280BD1069890ED010A8DED030A9DED030A13F0E7F80899087032E00698007A012815D15948D0ED7E0A9DED070AB8EE401ADFED571AB0EE600AAF
:40E1000001EE810A8DED030A9DED030A13F0CDF80899087018E00698007A022814D14C48D0ED7E0A9DED070AB8EE401ADFED4A1AB0EE600A01EEC10A8DED030A9DED030AC3
:40E1400013F0B3F8089908700120049062E40698007A032814D1069890ED010ABCEEC00A10EE100A80B200EE100AB8EE400A8DED030A9DED030AFCF727F90899087032E07D
:40E180000698007A012815D13148D0ED280A079800EB8000400000EE100AB8EEC00A30EE800A8DED030A9DED030AFCF70DF90899087018E00698007A022814D12448D0EDEE
:40E1C000280A079800EB8000400000EE100AB8EEC00A30EEC00A8DED030A9DED030AFCF7F3F8089908700120049039E20698007A032835D1069890ED010ADFED180AB4EE5F
:40E20000E00AF1EE10FA06DD022108980170642006F0EAFA62E0069890ED010AF2EE040AB4EEE00AF1EE10FA06D20321089801700A2006F0D9FA51E0069890ED010ABCEECA
:40E24000C00A10EE100AC0B2039006F0CDFA45E0202100200AD7233CCDCCCC3D0000C8420698007A01281BD1FE4890F8401007984000C0F1650081420BDAFA4890F8401086
:40E280000222079802FB0010C0B2039006F0ACFA24E0022108980170642006F0A5FA1DE00698007A022819D1EE4890F8401007984000093081420BDDEA4890F84010022274
:40E2C000079802FB1010C0B2039006F08DFA05E00321089801700A2006F086FA1A20FFF73FF901200490BBE10698007A032803D006210898017010E0069890ED010ABCEE5F
:40E30000C00A10EE100AC0B21FED2C0A039009F0A3F910B9012108980170E6E30698007A032803D00621089801707CE0069890ED010AF8EE000AB4EE600AF1EE10FA13D1C1
:40E34000C84890F842107C3000EB810090ED000A8DED030A9DED030A082009F07DF900BB0121089801705EE0069890ED010AFFEE000AB4EE600AF1EE10FA13D1B94890F8B4
:40E3800042106C3000EB810090ED000A8DED030A9DED030A082009F05FF910B901210898017040E0069890ED010AF7EE000AB4EE600AF1EE10FA13D1AA4890F8421074306B
:40E3C00000EB810090ED000A8DED030A9DED030A082009F041F900BB01210898017022E0069890ED010AF0EE000AB4EE600AF1EE10FA13D19B4890F84210843000EB8100FD
:40E4000090ED000A8DED030A9DED030A082009F023F910B901210898017004E09FED920A002009F019F960E30020FEF761F88DED030A00209DED030AFDF702FF55E300208B
:40E44000FEF756F88DED030A00209DED030AFDF71FFF4AE30020FEF74BF88DED030A00209DED030AFDF78FFF3FE3069890ED010ABCEEC00A10EE100AC0B203900FF0CDFD22
:40E4800033E3069890ED010ABCEEC00A10EE100AC0B20390FEF7CDF927E3069890ED010ABCEEC00A10EE100AC0B2039013F05AF81BE3069890ED010A8DED030A9DED030A7C
:40E4C00013F065F811E3069890ED010ABCEEC00A10EE100AC0B2039010F0B8FC05E3069890ED010ABCEEC00A10EE100A80B2039010F090FAF9E2069890ED010ABCEEC00AFF
:40E5000010EE100A80B2039010F099FAEDE2069890ED010ABCEEC00A10EE100AC0B2039011F02DFD2120FFF71BF8DEE20698007A032803D006210898017034E0069890ED33
:40E54000010AF7EE000AB4EE600AF1EE10FA0ED10AF050FD28B1B7EE000A112009F07CF821E0B7EE000A072009F076F81BE0069890ED010AF0EE000AB4EE600AF1EE10FA24
:40E5800005D19FED390A002009F066F80BE0069890ED010AF0EE080AB4EE600AF1EE10FA01D100F08BFCA0E2069890ED010ABCEEC00A10EE100A80B201460390022017F097
:40E5C00093FF92E2069890ED010ABCEEC00A10EE100A80B201460390012017F085FF84E20698007A03283BD1069890ED010AB5EEC00AF1EE10FA0BD11A4890F842000390DF
:40E60000184890F84100029003990AF0A9FB27E0069890ED010AF7EE000AB4EE600AF1EE10FA07D10F4890F84200012103900AF000FB15E0069890ED010AF0EE080AB4EE84
:40E64000600AF1EE10FA0BD1064890F842000390044890F841000122029003990AF068FA43E200002021002000000000069890ED010ABCEEC00A10EE100AC0B203900AF0C7
:40E6800029FA32E20698007A03280AD1069890ED010ABCEEC00A10EE100AC0B20390FBF7B8FF22E215F05EFB28B90698007A032801D10AF0B0F918E20698007A03280AD192
:40E6C000069890ED010ABCEEC00A10EE100AC0B20390FDF795FC08E20698007A03280AD1069890ED010ABCEEC00A10EE100AC0B20390FDF79DFCF8E10698007A03280BD19A
:40E70000069890ED010ABCEEC00A10EE100AC0B20121039010F0A8F9E7E10698007A032814D1069890ED010ADFEDFE0AB4EE600AF1EE10FA0AD10EF004F801200DF0A6FEE9
:40E740000021F94801720020F8490870CDE10698007A03280BD1069890ED010ABDEEC00A10EE100A00B20390FAF77EF918E00698007A012808D1EE48B0F8AA00401C00B216
:40E780000390FAF771F90BE00698007A022807D1E748B0F8AA00401E00B20390FAF764F9A3E11C20FEF7DCFE9FE10698007A03281AD1DF4890F842106C3000EB810090ED31
:40E7C000000A8DED050A9DED050AB5EEC00AF1EE10FA03D19FEDD70A8DED050A9DED050A082008F039FF07E00698007A20B91FED620A082008F030FF77E10698007A0328A2
:40E800000FD1CB4890F842107C3000EB810090ED000A8DED030A9DED030A082008F01CFF07E00698007A20B91FED710A082008F013FF5AE10698007A03281AD1BC4890F88D
:40E840004210743000EB810090ED000A8DED050A9DED050AB5EEC00AF1EE10FA03D19FEDB60A8DED050A9DED050A082008F0F4FE07E00698007A20B91FED850A082008F050
:40E88000EBFE32E10698007A03280FD1A84890F84210843000EB810090ED000A8DED030A9DED030A082008F0D7FE07E00698007A20B91FED930A082008F0CEFE15E10698B4
:40E8C000007A03280AD1069890ED010ABCEEC00A10EE100AC0B203900AF0DDF805E10698007A03280ED1069890ED010ABCEEC00A10EE100A80B201210390FCF770FF08996E
:40E9000008701CE00698007A01280AD1FCF7E4FE401C80B201210390FCF761FF089908700DE00698007A022809D1FCF7D5FE401E80B201210390FCF752FF08990870D4E09E
:40E940000698007A03280ED1069890ED010ABCEEC00A10EE100A80B201210390FCF757FF089908701CE00698007A01280AD1FCF7AFFE401C80B201210390FCF748FF0899A4
:40E9800008700DE00698007A022809D1FCF7A0FE401E80B201210390FCF739FF08990870A3E00698007A03280CD1069890ED010ABCEEC00A10EE100A80B20390FCF73FFF71
:40E9C0000899087091E00698007A03280CD1069890ED010ABCEEC00A10EE100A80B20390FCF744FF089908707FE00698007A03280CD1069890ED010ABCEEC00A10EE100A76
:40EA000080B20390FCF74DFF089908706DE00698007A03280CD1069890ED010ABCEEC00A10EE100A80B20390FCF76AFF089908705BE00698007A03280CD1069890ED010ADF
:40EA4000BCEEC00A10EE100AC0B2039018F011F80899087049E00698007A03280CD1069890ED010ABCEEC00A10EE100A80B20390FCF761FF0899087037E00698007A032855
:40EA80000CD1069890ED010ABDEEC00A10EE100A00B20390FCF781FF0899087025E00698007A03280CD1069890ED010ABDEEC00A10EE100A00B20390FCF758FF0899087075
:40EAC00013E00698007A03280AD1069890ED010ABCEEC00A10EE100AC0B20390FDF7EDF803E007210898017000BF00BF049809B000BD86B04FF6FF7438211048DFF840C053
:40EB000000DF02210F4880F808110C2284210E4833F010FD002879D103210A4880F8081100BF13E000007E43583200203C05002020210020CDCCCCBDCDCCCC3DF010002056
:40EB400069290408685200206C100020224605A98748DFF820C200DF012858D000208DF800008DF80D0001208DF80C0000208DF80E0005980078002839D004AA0121059864
:40EB8000FEF7F4FC05469DF8100068B100250599087824F081FA06460598837A427A9DF81010304624F07EFA08F0D8FE08B1002504E00598007A032800D100250DB39DF81F
:40EBC0000D00F0B90598007AD8B1059A07CA8DE8070001208DF80D008DF80C004FF47A649DF80E00401CC0B28DF80E0009E008F06AFD30B16048D0F890110120DFF87CC1FB
:40EC000000DF5F480599F9F77BFB8AE747E09DF80000002885DD9DF80E0000283CDD9DF80E00032803D102208DF80C000EE09DF80E00052803D106208DF80C0006E09DF896
:40EC40000E00072802D110208DF80C009DF80E00FF2805DA9DF80E00401CC0B28DF80E009DF80C1004AA6846FEF780FC9DF8100078B100208DF80E000599087824F00CFADF
:40EC800006460598837A427A9DF81010304624F009FA4FF4FA6444E74FF6FF7441E70521354880F808110020DFF8D8C000DF00BFFEE72DE9F0472DED028B0546B0EE408AD7
:40ECC0000E46174698464FF001092948DFF8B8C000DFD0B900BF284890F8090140F00201254880F80911B0F814014FF6FF71884207DA2148B0F81401401C81B21E48A0F851
:40ED0000141100BF4FF000092CE01D48F9F7E8FA04466CB1257084ED018A2672677284F80A800A2221461248DFF860C000DF19E000BF114890F8090140F004010E4880F88C
:40ED40000911B0F814014FF6FF71884207DA0A48B0F81401401C81B20748A0F8141100BF4FF000094846BDEC028BBDE8F0870000F0100020F92A040868520020E12704088E
:40ED80006C1000206532040861290408552A040831B52DED020B0446FE4890EDD40ADDED000AB4EEE00AF1EE10FA00D3ACB100BF04226946F848006800F554700CF0A8FBEE
:40EDC00020B99DED000AF34880EDD40A00BFF348C16B0220DFF8C8C300DF3EBD31B52DED020B0446EB4890EDD30ADDED000AB4EEE00AF1EE10FA00DCACB100BF04226946A2
:40EE0000E548006800F553700CF082FB20B99DED000AE04880EDD30A00BFE048C16B0220DFF87CC300DF3EBD31B52DED020B0446D84890ED2F0ADDED000AB4EEE00AF1EE9C
:40EE400010FA00D3A4B100BF04226946D2480068BC300CF05DFB20B99DED000ACD4880ED2F0A00BFCD48C16B0220DFF834C300DF3EBD31B52DED020B0446C64890ED2E0AFE
:40EE8000DDED000AB4EEE00AF1EE10FA00DCA4B100BF04226946C0480068B8300CF038FB20B99DED000ABB4880ED2E0A00BFBB48C16B0220DFF8E8C200DF3EBD10B54FF435
:40EEC000F671B84830F0C7FBB24890F82800B54981F8E0012AF048FFB2498860012081F8DC01002081F8DD019FEDAF0A084680ED500A002007F0EBF801209FEDAB0AFFF7E9
:40EF0000B8FF01209FEDA80AFFF78EFF01209FEDA60AFFF763FF01209FEDA30AFFF738FF10BD10B517F0C3FDA04880ED000A90ED000AF2EE000A20EE200ADFED9D0A80EEBA
:40EF4000201A9C4880ED001A984890ED000AF0EE080A20EE200ADFED960A80EE201A964880ED001A914890ED000AF3EE010A20EE200ADFED8F0A80EE201A904880ED001AF4
:40EF800010BD10B5002428F015FB40B38C4800680078012800D128E0894800680078022801D1142421E0864800680078052801D128241AE0824800680078032801D13C24EA
:40EFC00013E07F4800680078062801D150240CE07B4800680078082807D1642405E028F001FB10B16F4890F8E141204610BD10B56C4890F8DD0173490978884203D0FFF7E7
:40F00000C0FF7149087010BD70B52DED028B044614F0A8FE00287DD1002596E05D48C03000EB8400D0ED000AB0EE600A284612F078F95848C03000EB8400D0ED000AB0EE29
:40F04000600A284611F07FFF5248C83000EB8400D0ED000AB0EE600A284612F086F94D48C83000EB8400D0ED000AB0EE600A284611F0C7FF4748D03000EB8400D0ED000AB5
:40F08000B0EE600A284612F094F94248D03000EB8400D0ED000AB0EE600A284612F00DF83C48D83000EB8400D0ED000AB0EE600A284612F0A2F93748D83000EB8400D0ED86
:40F0C000000AB0EE600A284612F055F83149E031085D294612F0B5F92E49E231085D294612F0CDF928F066FA08B32A49E0310A5D891C095D501800EBD071491000EE101ADE
:40F10000B8EEC00AB0EE408ABCEEC80A10EE101AC8B200E01DE0214611F0AFFEBCEEC80A10EE101AC8B2214611F0DAFE0BE01949E031085D214611F0A0FE1649E231085DE9
:40F14000214611F0CDFE681CC5B2022DFFF666AFAFE01048C03000EB8400D0ED000AB0EE600A204612F0DDF80A48C03000EB8400D0ED000AB0EE600A204611F0E4FE0548C0
:40F18000C83000EB8400D0ED000AB0EE600A20461CE0000020210020F003002068520020E12704082811002000000000700300200000C84274030020780300207C0300208E
:40F1C00048030020800300206E03002012F0CDF8FE4800EB8400D0ED000AB0EE600A204611F00FFFF948083000EB8400D0ED000AB0EE600A204612F0DCF8F448083000EB5E
:40F200008400D0ED000AB0EE600A204611F055FFEE48103000EB8400D0ED000AB0EE600A204612F0EAF8E948103000EB8400D0ED000AB0EE600A204611F09DFFE34918319B
:40F24000085D214612F0FDF8E0491A31085D214612F015F928F0AEF9F8B1DC4918310A5D891C095D501800EBD071491000EE101AB8EEC00AB0EE408ABCEEC80A10EE101AB2
:40F28000C8B2214611F0F9FDBCEEC80A10EE101AC8B2214611F024FE0BE0CC491831085D214611F0EAFDC9491A31085D214611F017FEBDEC028B70BD01B500BF01226946E8
:40F2C000C348006800F5E9700CF022F928B99DF80000BE49C83981F8D20100BF08BD10B5032006F0F4FE1FED500A002008F0B4F90120FFF7E1FFB549C83991F84200FFF736
:40F3000083FE1C2021F0A6FF10BD01B5B8B000203590349033903290319030902F902E901FED5F0A389880ED530A1FED610A389880ED560A1FED640A389880ED540A1FEDFF
:40F34000660A389880ED580A1FED690A389880ED550A1FED6B0A389880ED590A01203790FEE3379834F0DCFB9FED9A0B53EC102BCDE926019DED260B51EC100B34F0C8F92F
:40F38000CDE92C0137983690389890ED6A0B8DED200B9DED2C0B53EC102B9DED200B51EC100B34F00DFCCDE92401389890ED680B8DED1A0B9DED2C0B53EC102B9DED1A0BD5
:40F3C00051EC100B34F0FCFBCDE91C019DED2C0B53EC102B9DED1C0B51EC100B34F0F0FBCDE92001389890ED660B8DED140B9DED2C0B53EC102B9DED140B51EC100B34F0E6
:40F40000DFFBCDE916019DED2C0B53EC102B9DED160B51EC100B34F0D3FBCDE918019DED2C0B53EC102B9DED180B51EC100B34F0C7FBCDE91C01389890ED640B8DED0E0BDE
:40F440009DED2C0B53EC102B9DED0E0B51EC100B34F0B6FBCDE910019DED2C0B53EC102B9DED100B51EC100B34F0AAFBCDE912019DED2C0B53EC102B9DED120B51EC100BB6
:40F4800034F09EFBCDE914019DED2C0B53EC102B9DED140B51EC100B34F092FBCDE91801389890ED620B8DED080B9DED2C0B53EC102B9DED080B51EC100B34F081FBCDE93B
:40F4C0000A019DED2C0B53EC102B9DED0A0B51EC100B34F075FBCDE90C019DED2C0B53EC102B9DED0C0B51EC100B34F069FBCDE90E019DED2C0B53EC102B9DED0E0B51ECDC
:40F50000100B34F05DFBCDE910019DED2C0B53EC102B9DED100B51EC100B34F051FBCDE91401389890ED600B8DED020B9DED2C0B53EC102B9DED020B51EC100B34F040FB32
:40F54000CDE904019DED2C0B53EC102B9DED040B51EC100B34F034FBCDE906019DED2C0B53EC102B9DED060B51EC100B34F028FBCDE908019DED2C0B53EC102B9DED080B88
:40F5800051EC100B34F01CFBCDE90A019DED2C0B53EC102B9DED0A0B51EC100B34F010FBCDE90C019DED2C0B53EC102B9DED0C0B51EC100B34F004FBCDE91001389890ED68
:40F5C0005E0B8DED000B9DED2C0B07E0E8210020F0030020000000000000244053EC102B9DED000B51EC100B34F0EAFACDE902019DED2C0B53EC102B9DED020B51EC100B83
:40F6000034F0DEFACDE904019DED2C0B53EC102B9DED040B51EC100B34F0D2FACDE906019DED2C0B53EC102B9DED060B51EC100B34F0C6FACDE908019DED2C0B53EC102B2E
:40F640009DED080B51EC100B34F0BAFACDE90A019DED2C0B53EC102B9DED0A0B51EC100B34F0AEFACDE90C019DED2C0B53EC102B9DED0C0B51EC100B34F0A2FACDE90E0182
:40F680009DED100B53EC102B9DED0E0B51EC100B33F082FFCDE912019DED140B53EC102B9DED120B51EC100B33F076FFCDE916019DED180B53EC102B9DED160B51EC100B12
:40F6C00033F06AFFCDE91A019DED1C0B53EC102B9DED1A0B51EC100B33F05EFFCDE91E019DED200B53EC102B9DED1E0B51EC100B33F052FFCDE922019DED240B53EC102B6C
:40F700009DED220B51EC100B33F046FFCDE92601389890ED6C0B8DED240B9DED240B53EC102B9DED260B51EC100B33F035FFCDE92A01389890ED7A0B8DED200B9DED2C0B52
:40F7400053EC102B9DED200B51EC100B34F038FACDE92401389890ED780B8DED1A0B9DED2C0B53EC102B9DED1A0B51EC100B34F027FACDE91C019DED2C0B53EC102B9DED43
:40F780001C0B51EC100B34F01BFACDE92001389890ED760B8DED140B9DED2C0B53EC102B9DED140B51EC100B34F00AFACDE916019DED2C0B53EC102B9DED160B51EC100BE4
:40F7C00034F0FEF9CDE918019DED2C0B53EC102B9DED180B51EC100B34F0F2F9CDE91C01389890ED740B8DED0E0B9DED2C0B53EC102B9DED0E0B51EC100B34F0E1F9CDE9B4
:40F8000010019DED2C0B53EC102B9DED100B51EC100B34F0D5F9CDE912019DED2C0B53EC102B9DED120B51EC100B34F0C9F9CDE914019DED2C0B53EC102B9DED140B51ECB8
:40F84000100B34F0BDF9CDE91801389890ED720B8DED080B9DED2C0B53EC102B9DED080B51EC100B34F0ACF9CDE90A019DED2C0B53EC102B9DED0A0B51EC100B34F0A0F9C4
:40F88000CDE90C019DED2C0B53EC102B9DED0C0B51EC100B34F094F9CDE90E019DED2C0B53EC102B9DED0E0B51EC100B34F088F9CDE910019DED2C0B53EC102B9DED100B59
:40F8C00051EC100B34F07CF9CDE91401389890ED700B8DED020B9DED2C0B53EC102B9DED020B51EC100B34F06BF9CDE904019DED2C0B53EC102B9DED040B51EC100B34F040
:40F900005FF9CDE906019DED2C0B53EC102B9DED060B51EC100B34F053F9CDE908019DED2C0B53EC102B9DED080B51EC100B34F047F9CDE90A019DED2C0B53EC102B9DED3B
:40F940000A0B51EC100B34F03BF9CDE90C019DED2C0B53EC102B9DED0C0B51EC100B34F02FF9CDE91001389890ED6E0B8DED000B9DED2C0B53EC102B9DED000B51EC100B45
:40F9800034F01EF9CDE902019DED2C0B53EC102B9DED020B51EC100B34F012F9CDE904019DED2C0B53EC102B9DED040B51EC100B34F006F9CDE906019DED2C0B53EC102BF8
:40F9C0009DED060B51EC100B34F0FAF8CDE908019DED2C0B53EC102B9DED080B51EC100B34F0EEF8CDE90A019DED2C0B53EC102B9DED0A0B51EC100B34F0E2F8CDE90C0151
:40FA00009DED2C0B53EC102B9DED0C0B51EC100B34F0D6F8CDE90E019DED100B53EC102B9DED0E0B51EC100B33F0B6FDCDE912019DED140B53EC102B9DED120B51EC100B00
:40FA400033F0AAFDCDE916019DED180B53EC102B9DED160B51EC100B33F09EFDCDE91A019DED1C0B53EC102B9DED1A0B51EC100B33F092FDCDE91E019DED200B53EC102B4E
:40FA80009DED1E0B51EC100B33F086FDCDE922019DED240B53EC102B9DED220B51EC100B33F07AFDCDE92601389890ED7C0B8DED240B9DED240B53EC102B9DED260B51EC5B
:40FAC000100B33F069FDCDE928016421369890FBF1F201FB120008BB9DED2A0B51EC100B33F028FD01466422369890FBF2F2521E389800F5027040F822109DED280B51EC7D
:40FB0000100B33F017FD01466422369890FBF2F2521E389800F50C7040F82210389890ED000AB1EE400A8DED250A259834F03EFBCDE926019DED2A0B53EC102B9DED260B7A
:40FB400051EC100B34F03AF92AD23598401C80B235909DED350AB8EE400ADFEDFE0A00E028E2B4EEE00AF1EE10FA1BDD389890ED530AB5EEC00AF1EE10FA13D19DED2C0B31
:40FB800051EC100B33F0D6FC00EE100AB1EE400AF3EE040A30EE200A389880ED530A01E000203590389890ED000AB1EE400A8DED250A259834F0FAFACDE926019DED2A0B16
:40FBC00053EC102B9DED260B51EC100B34F0F6F826D23498401C80B234909DED340AB8EE400ADFEDDC0AB4EEE00AF1EE10FA19DD9DED2C0B51EC100B33F09CFC00EE100A9F
:40FC0000F1EE400A9DED340AB8EE400AB2EE041AC0EE011A30EEA10A389880ED520A01E000203490389890ED010AB1EE400A8DED250A259834F0BAFACDE926019DED2A0B1A
:40FC400053EC102B9DED260B51EC100B34F0B6F828D23198401C80B231909DED310AB8EE400AF1EE040AB4EEE00AF1EE10FA1BDD389890ED540AB5EEC00AF1EE10FA13D11F
:40FC80009DED2C0B51EC100B33F054FC00EE100AB1EE400AF6EE000A30EE200A389880ED540A01E000203190389890ED030AB1EE400A8DED250A259834F078FACDE9260118
:40FCC0009DED2A0B53EC102B9DED260B51EC100B34F074F828D22F98401C80B22F909DED2F0AB8EE400AF1EE040AB4EEE00AF1EE10FA1BDD389890ED550AB5EEC00AF1EE15
:40FD000010FA13D19DED2C0B51EC100B33F012FC00EE100AB1EE400AF6EE000A30EE200A389880ED550A01E000202F9038980068259034F03BFACDE926019DED280B53ECE9
:40FD4000102B9DED260B51EC100B33F0FDFE26D23398401C80B233909DED330AB8EE400ADFED7C0AB4EEE00AF1EE10FA19DD389890ED560AB5EEC00AF1EE10FA11D19DED20
:40FD80002C0B51EC100B33F0D5FB00EE100AF3EE040A30EE600A389880ED560A01E00020339038980068259034F000FACDE926019DED280B53EC102B9DED260B51EC100BAF
:40FDC00033F0C2FE24D23298401C80B232909DED320AB8EE400ADFED5F0AB4EEE00AF1EE10FA17DD9DED2C0B51EC100B33F0A2FB00EE900A9DED320AB8EE400AB2EE041AE7
:40FE0000C0EE011A30EEE10A389880ED570A01E00020329038984068259034F0C7F9CDE926019DED280B53EC102B9DED260B51EC100B33F089FE26D23098401C80B230909F
:40FE40009DED300AB8EE400AF1EE040AB4EEE00AF1EE10FA19DD389890ED580AB5EEC00AF1EE10FA11D19DED2C0B51EC100B33F061FB00EE100AF6EE000A30EE600A3898A9
:40FE800080ED580A01E0002030903898C068259034F08CF9CDE926019DED280B53EC102B9DED260B51EC100B33F04EFE26D22E98401C80B22E909DED2E0AB8EE400AF1EE2B
:40FEC000040AB4EEE00AF1EE10FA19DD389890ED590AB5EEC00AF1EE10FA11D19DED2C0B51EC100B33F026FB00EE100AF6EE000A30EE600A389880ED590A01E000202E9067
:40FF0000389890ED5C0AB1EE400A8DED250A259834F04CF9CDE926019DED2A0B53EC102B9DED260B51EC100B33F048FF19D29DED2A0B51EC100B33F0FDFA3899C1F87001AC
:40FF40009DED2C0B51EC100B33F0F4FA00EE100A02E0000000004843B1EE400A389880ED5A0A3898D0F87401259034F01FF9CDE926019DED280B53EC102B9DED260B51EC4E
:40FF8000100B33F0E1FD11D29DED280B51EC100B33F0D0FA3899C1F874019DED2C0B51EC100B33F0C7FA3899C1F86C013798401C80B237903798B0F57A7F7FF7D2A93898FB
:40FFC00090ED540AB5EEC00AF1EE10FA0BD0389890ED540A80ED5A0A389890ED010AB1EE400A80ED5C0A389890ED580AB5EEC00AF1EE10FA09D0389890ED580A80ED5B0A06
:020000040801F1
:40000000389890ED010A80ED5D0A389890ED530AB5EEC00AF1EE10FA61D0389890ED560AB5EEC00AF1EE10FA59D0389890ED5A0AD0ED530AB7EE001A70EEC10AB4EEE00AF8
:40004000F1EE10FA4BDC389890ED5B0AD0ED560AB7EE001A70EE810AB4EEE00AF1EE10FA3DD3389890ED530AD0ED520A30EE600A8DED230A239834F099F8CDE924019DEDAD
:40008000240B30F06DFC8DED260B9FEDF80B53EC102B9DED260B51EC100B33F08FFE1ED3389890ED560AD0ED570A30EE600A8DED230A239834F07AF8CDE924019DED240B41
:4000C00030F04EFC8DED260B9FEDE80B53EC102B9DED260B51EC100B33F070FE03D22320E44981F8DA01389890ED550AB5EEC00AF1EE10FA04D19FEDE00A389880ED550ACC
:40010000389890ED590AB5EEC00AF1EE10FA04D19FEDDA0A389880ED590A39B000BD70B52DED088B064600246FE09FEDD50BB0EE408AF0EE608A9FEDD20BB0EE409AF0EE42
:40014000609A002551E006F1400000EB850090ED000A10EE101A084634F028F841EC1B0B04EB440000EBC400C74901EBC00000EBC50090ED001BB0EE410AF0EE610A53EC9D
:40018000102B51EC1B0B33F01BFD53EC182B33F003FA41EC180B06F16C0000EB850090ED000A10EE101A084634F000F841EC1B0B04EB440000EBC400B34901EBC00000EBC0
:4001C000C50090ED001BB0EE410AF0EE610A53EC102B51EC1B0B33F0F3FC53EC192B33F0DBF941EC190B681CC5B20B2DABDB06F5BC7000EBC40080ED008B06F5DC7000EBFD
:40020000C40080ED009B601CC4B2082C8DDBBDEC088B70BD70B504469C4890F82850022D14D19FED9B0A84ED000A9FED9A0A84ED010A9FED990A84ED020A9FED980A84EDF1
:40024000030A9FED970A84ED040A89E00D2D14D19FED8F0A84ED000A9FED8E0A84ED010A9FED8D0A84ED020A9FED8E0A84ED030A9FED8B0A84ED040A72E00C2D14D19FED1F
:40028000840A84ED000A9FED830A84ED010A9FED820A84ED020A9FED830A84ED030A9FED800A84ED040A5BE0032D14D19FED780A84ED000A9FED770A84ED010A9FED760A71
:4002C00084ED020A9FED780A84ED030A9FED740A84ED040A44E0012D14D19FED6D0A84ED000A9FED6C0A84ED010A9FED6B0A84ED020A9FED6C0A84ED030A9FED6C0A84EDC8
:40030000040A2DE00B2D17D127F06CF9A0B19FED600A84ED000A9FED5F0A84ED010A9FED5E0A84ED020A9FED5F0A84ED030A9FED600A84ED040A13E09FED550A84ED000A21
:400340009FED540A84ED010A9FED530A84ED020A9FED540A84ED030A9FED540A84ED040A70BD70B52DED028B04465248FFF752FF5048FFF7D4FE4F48FEF7C7FF4D48D0EDB8
:40038000550AB0EE600A204610F097FE4948D0ED550AB0EE600A204611F00BF84548D0ED590AB0EE600A204610F0E5FE4148D0ED590AB0EE600A204611F01FF83D4890ED8D
:4003C000000AFFEE000A20EE200AB0EE408A90ED5A0AD0ED530A30EE600AD0ED5C0A70EEC80A80EE801A80ED7E1AD0ED7E0A90ED531AB0EE480A00EEC10A80ED7F0A90ED2E
:40040000000AB0EE408A90ED5B0AD0ED560A30EE600AD0ED5D0A70EEC80A80EE801A80ED801AD0ED800A90ED561AB0EE480A00EEC10A80ED810A90ED040AD0ED7E0A80EE4D
:40044000201AB0EE418A9FED0D0A28EE000AB0EE408A9FED190AB4EEC08AF1EE10FA2DDD9FED150AB0EE408A33E00000000000000000F03F281100200000C8C20000C842DE
:400480000000000000000000880000202021002035FA0E3DC2B8323E00000000C2B8B23E8FDAA53B920A063F7CD9A03E88C3643B35FA0E3C1813002000007F43B7EE000AE9
:4004C000B4EEC08AF1EE10FA03D2B7EE000AB0EE408AB6EE000A38EE000ABCEEC00A10EE100AC5B22146284610F0C7FC2146284610F0A7FFFE4890ED040AD0ED800A80EEC1
:40050000201AB0EE418A1FED230A28EE000AB0EE408A1FED170AB4EEC08AF1EE10FA04DD1FED1B0AB0EE408A0AE0B7EE000AB4EEC08AF1EE10FA03D2B7EE000AB0EE408A81
:40054000B6EE000A38EE000ABCEEC00A10EE100AC5B22146284610F0C3FC2146284610F08EFFBDEC028B70BD2DE9F04F2DED088BC5B005468A4600241FED390AB0EE408AD4
:400580001FED3B0AF0EE408A1FED3D0AB0EE409A1FED3F0AF0EE409A032101A816F06BFFBAF1000F0DD1DFF84C8308F12C0905F1400605F16C0708F11C0B08F148004490E7
:4005C00024E0BAF1010F0FD1DFF8288308F1580808F12C0905F1980605F1C40708F11C0B08F14800449011E0BAF1020F0ED1DFF8048308F1B00808F12C0905F1F00605F51A
:400600008E7708F11C0B08F1480044901FED5E0A86ED000A1FED600A87ED000A1FED620A85ED050A032201A9584616F038FF032101A816F096FFF0EE409A032201A944982D
:4006400016F02DFF032101A816F08BFFB0EE409AB6EE080A29EE80AABEEE000A69EE80AAB6EE080A29EE00BABEEE000A69EE00BA012476E000EE104AB8EE400AF2EE040A56
:4006800020EE200A05F1140000EB840080ED000A601E08EB800090ED000AB5EEC00AF1EE10FA06DD1FED840A06EB840080ED000A08E0601E08EB800090ED000A06EB840006
:4006C00080ED000A601E09EB800090ED000AB5EEC00AF1EE10FA06D21FED910A07EB840080ED000A08E0601E09EB800090ED000A07EB840080ED000A06EB840090ED000AFE
:40070000601E06EB8000D0ED000A30EE600AB0EE408A07EB840090ED000A601E07EB8000D0ED000A30EE600AF0EE408AB4EECA8AF1EE10FA0ED3B4EEEA8AF1EE10FA09DC8B
:40074000F4EECB8AF1EE10FA04DCF4EEEB8AF1EE10FA04D223206749283981F8DA01601CC4B20B2C86DB45B0BDEC088BBDE8F08F10B500215E48FFF7F7FE10BD10B52DEDB9
:40078000028B5D4890F828400E2C35D2DFE804F0340C0807130B34341A1B1C230A0900BF00BF00BF00BF00BF9FED540A5148283880ED500A27E09FED520A4E48283880ED08
:4007C000500A20E000BF00BF9FED4C0A4948283880ED500A17E026F0EDFE30B1B3EE040A4448283880ED500A05E09FED450A4148283880ED500A06E01FEDD90A3D48283822
:4008000080ED500A00BF00BF08F003FC70B1FAF7D5FFB0EE408AFAF757FF00EE100AB8EE400AB4EEC08AF1EE10FA10DC08F0E2FB30B1FAF7D8FDB5EEC00AF1EE10FA06DC7A
:4008400015F082FFB5EEC00AF1EE10FA09DD2948283890ED500AFFEE000A20EE200A80ED500ABDEC028B10BD73B52DED020B04460D460A2C21D200BF05EB850221490968EF
:4008800001F5177101EBC20101EB8400042269460AF03EFE50B99DED000A05EB85011A4800EBC10000EB840080ED000A00BF1748C16B0220DFF858C000DF7FBD10B5FAF75D
:4008C00046FB10BD73B52DED020B04460D460A2C35D200BF05EB85020A49096801F59A7101EBC20101EB84000422694612E0000018130020501100202021002000008C42E5
:4009000000004842F00300207C23002068520020E12704080AF0FCFD50B99DED000A05EB8501F94800EBC10000EB840080ED000A00BFF648C16B0220DFF8D4C300DF7FBDC0
:4009400073B52DED020B04460D460A2C22D200BF05EB8502EF49096801F5037101EBC20101EB8400042269460AF0D2FD58B99DED000A05EB8501E448D83000EBC10000EB75
:40098000840080ED000A00BFE048C16B0220DFF880C300DF7FBD10B5FAF7D9FA10BD73B52DED020B04460D460A2C21D200BF05EB8502D8490968E43101EBC20101EB84006B
:4009C000042269460AF0A4FD58B99DED000A05EB8501CD48503800EBC10000EB840080ED000A00BFC948C16B0220DFF824C300DF7FBD70B50446C84890F828500E2D28D292
:400A0000DFE805F0270C0807120B2727272727180A0900BF00BF00BF00BF00BF1FED490ABE4880ED500A1AE01FED4B0ABB4880ED500A14E026F0BEFD28B19FEDB90AB748B5
:400A400080ED500A04E01FED530AB44880ED500A05E09FEDB30AB14880ED500A00BF00BF032C08D1AD4890ED500AFFEE000A20EE200A80ED500A70BDA74A92F8281006295A
:400A800005D19FEDA80AA54A82ED500A0CE0042905D11FED650AA14A82ED500A04E01FED690A9E4A82ED500A062808D19B4A92ED500AFFEE000A20EE200A82ED500A7047C4
:400AC000B5EEC00AF1EE10FA01D2012070470020FCE7B5EEC00AF1EE10FA01DD012070470020FCE72DE9F04106460C4615464FF00408894890F828702868A8B929F034F930
:400B00002860002088490870884890ED000A15F068FF20B1BFEE000A854880ED000A15F013FE844880ED000A0E2F38D2DFE807F0370C0807160B3737373737200A0900BF5F
:400B400000BF00BF00BF00BF794890ED000A5FED950A20EE200A84ED000A2AE0744890ED000A5FED990A20EE200A84ED000A20E026F020FD48B16E4890ED000ADFED680AFD
:400B800020EE200A84ED000A08E0694890ED000A5FEDA60A20EE200A84ED000A09E0644890ED000ADFED5E0A20EE200A84ED000A00BF00BF41F28831286829F0DBF828B1F1
:400BC000212030704FF00108002599E040F6C411286829F0CFF8F0B153480078D8B9564890ED000A15F0FDFE28B9534890ED000A15F09CFE78B101204B4908704C4890ED40
:400C0000000AFFEE000A20EE200A80ED000A29F0ABF8286074E0D4ED000AB0EE600AFFF758FF68B115F090FD4248D0ED000A30EE600ADFED420AB4EEE00AF1EE10FA14DC4B
:400C4000D4ED000AB0EE600AFFF73AFFB0B115F07BFD3848D0ED000A30EE600ADFED380AB4EEE00AF1EE10FA08D24FF003089FED2C0A84ED000A0020286041E0D4ED000A4D
:400C8000B0EE600AFFF725FF68B115F05DFD2948D0ED000A30EE600ADFED290AB4EEE00AF1EE10FA14D3D4ED000AB0EE600AFFF707FF28B315F048FD1E48D0ED000A30EE40
:400CC000600ADFED1E0AB4EEE00AF1EE10FA17DD114890F89C0018B90120F9F758FB07E00D4890F89C00012802D10020F9F74FFB4FF003089FED0A0A84ED000A00202860B8
:400D00004046BDE8F08100005422002068520020E1270408F003002020210020281100200000000000002042820300207C030020840300208803002074030020C2B8B23DCE
:400D4000C2B8B2BD70B52DED048B0425FE4890F8DC010A287DD2DFE800F00506EF477CEE487CEDEC00BFF84890F8DD0120B1102821D0112835D110E01120F34981F8DD0116
:400D800015F0E2FCF04880ED080AB6EE000A80ED500A0020EC49086024E0EB4A02F5A07101F19A00FFF79EFE032803D11020E64981F8DD0116E00620E34981F8DC01022093
:400DC00081F8DD010A2081F8E3010020086015F0BBFCDD4880ED080AB6EE000A80ED500A00E000BF00BF0AE300BFD74890F8DD01801E0B287BD2DFE800F0067AA0FC60C810
:400E00007A7A7A7A7B00D048006870B928F0ACFFCD490860084690F8E1010A2805DD084690F8E101C01F81F8E101C74991F8DC01FFF722FEC44908684FF47A6128F09AFFCF
:400E4000B0B115F081FCC048D0ED080A30EEC00A00E0F4E3B0EEC00ADFEDBC0AB4EEE00AF1EE10FA04D22120B74981F8DA0123E0B74890ED000A15F0B4FD20B1B24890F8AD
:400E8000DC0103280AD0B24890ED000A15F04EFD90B1AD4890F8DC0106280DD1B6EE000AA94880ED500A0620A74981F8DD010C2081F8DF0100200860A0E2B6EE000AA248DE
:400EC00080ED500A006818B928F04EFF9E4908609D490868C82128F04DFF38B19A4890F8DF01994981F8DD010020086086E284E2954991F8DC01FFF77CFD9348006818B912
:400F000028F032FF904908608F490868C82128F031FF68B1B6EE000A8B4880ED500A0620894981F8DD0100200860042081F8DF0164E2FDE3FDE363E263E215F005FCF0EE85
:400F4000409A4FF6FF71834816F0FBFB7E48006818B928F009FF7C4908607B4908684FF4FA7128F007FF78B1774890ED680A80ED080A0720744981F8DD010020086001F5C0
:400F8000C07000210162416238E26F48006818B928F0EAFE6C4908606B4890F8E30100EB8000400000EE100AB8EEC00A664880ED500A90F8DC01032808D1634890ED500A11
:400FC000FFEE000A20EE200A80ED500A604890ED000A15F006FD20B15B4890F8DC0106280CD05B4890ED000A15F0A0FCC0B1564800E030E090F8DC01032811D102205249E8
:4010000081F8DD0101F5C07000210162416215F09BFB4D4880ED080A00204B49086019E0494908684FF4FA7128F0A4FE90B1B6EE000A454880ED500A0620434981F8DD0192
:40104000086828F0B9FE4049C86100200860052081F8DF01D2E115F077FBF0EE409A4FF6FF713C4816F06DFB3748006818B928F07BFE35490860344908684FF4FA7128F00E
:4010800079FE00285FD0304890ED680AD0ED080A30EE608AB0EEC80AF0EE409A15F046FC20B1294890F8DC01032821D0284890ED000A15F03BFC20B1234890F8DC010328F3
:4010C00016D0B0EEC80AF0EE409A15F08AFC20B11D4890F8DC0106280AD01D4890ED000A15F07FFC98B1184890F8DC0106280ED10220154981F8DD01084690ED680A80EDAC
:40110000080A00F5C0700021016241620DE007200D4981F8DD01084690ED680A80ED080A00F5C070002101624162074890F8E301401E054981F8E301084690F8DC010328E6
:4011400062D1084608E057E12811002035FA0E3D74030020C812002090ED070AF8EE400A9FEDFE1A80EE810AC8EE000A90F8E311283000EB8100C0ED000AF94A92F8421039
:40118000F84A92F8E30192F8E331283202EB8302D2ED000AB0EE600AFFF701FCF14890F8E311283000EB8100D0ED000AB0EE600A0020FDF75EFEFFF7EEFBEA4890F8E3110C
:4011C000803000EB810080ED000AE54A92F84210E44A92F8E30192F8E331803202EB8302D2ED000AB0EE600AFFF7AAFBDD4890F8E311803000EB8100D0ED000AB0EE600AFB
:401200000020FDF7EBFD57E0D64890ED070AF8EE400A9FEDD21A80EE810AC8EE000A90F8E311543000EB8100C0ED000ACC4A92F84210CC4A92F8E30192F8E331543202EBC4
:401240008302D2ED000AB0EE600AFFF73BFBC54890F8E311543000EB8100D0ED000AB0EE600A0020FDF7E0FDFFF728FBBD4890F8E311AC3000EB810080ED000AB84A92F8CE
:401280004210B84A92F8E30192F8E331AC3202EB8302D2ED000AB0EE600AFFF7E5FAB14890F8E311AC3000EB8100D0ED000AB0EE600A0020FDF792FDAA4890F8E301002823
:4012C00013D1A84890F8DC0106280FD10320A54981F8DC01022081F8DD01B6EE000A084680ED500A0A2081F8E30182E0B7EE000A9C4880ED4E0A09209B49087026E0994857
:401300005430994991F9001000EB810090ED000A5FED720AB4EEE00AF1EE10FA10D2924890F9000000EE100AB8EEC00AF2EE040A20EE200A8B4880ED4E0AFF208A49087098
:4013400089480078401E40B287490870864890F900000028D3DAB7EE000A824880ED4D0A09208149087026E07E4828307E4991F9001000EB810090ED000ADFED7C0AB4EE4C
:40138000E00AF1EE10FA10DD774890F9000000EE100AB8EEC00AFAEE040A20EE200A714880ED4D0AFF20704908706F480078401E40B26D4908706C4890F900000028D3DAF3
:4013C000684890ED4E0A80ED4F0A0520654981F8DC010D2081F8DD01B6EE000A084680ED500A002081F8E3019FED610A084680ED4C0A00205B49086000E000BF00BFD9E169
:4014000000BF584890F8DD0106281DD00D2802D00E287DD132E0FFF7B1F9564890ED000A15F0B4FA78B1B6EE000A4E4880ED500A06204C4981F8DD010E2081F8DF0128F0D2
:4014400093FC484908608EE1B6EE000A454880ED500A014608684FF4FA7128F08BFC60B1404890F8DF013F4981F8DD010020086015F06AF93B4880ED080A74E1394890F83F
:40148000DC01052807D115F05FF93648D0ED080A70EE608A06E015F057F93248D0ED080A70EEC08A2F48006860B928F05DFC2D49086008460068C1F8E4019FED2D0A084680
:4014C00080ED7A0A264890F8430001282FD128F04BFC2449D1F8E411441A224890ED7A0A30EE280A80ED7A0AB4F57A7F1AD3D0ED7A0A00EE104AB8EE400A80EE801AF0EE17
:40150000418A9FED1B0A80ED7A0A28F02DFC00E028E11449C1F8E40115F016F9114880ED080A03E09FED120AF0EE408A00BF0C4890ED6E0AB4EEE80AF1EE10FA7ED20948D4
:4015400090ED4C0AD0ED500A30EE200A80ED4C0A90F8E301401C03490EE0000000007A4420210020281100208103002035FA0EBD000000007803002081F8E301B6EE000AB8
:40158000084680ED500A0D2081F8DD01086828F013FC00EE100AB8EE400A5FED100A80EE209AFE4890F8DC01052816D1FB4890ED4F0A30EE090AF1EE040A30EE600A80ED8A
:4015C0004F0A90ED4F0AB5EEC00AF1EE10FA1AD21FED190A80ED4F0A15E0F04890ED4F0A30EE490AF1EE040A30EE200A80ED4F0A90ED4F0AB5EEC00AF1EE10FA03DD1FEDFE
:40160000240A80ED4F0AE54890F8E30103283ADBE248D0ED4C0A90F8E30100EE100AB8EE400A80EE801ADD4880ED4C1A90F8DC01052829D1DA4991F8420001E03FE0B8E02A
:40164000D649D1ED4C0AB0EE600A0FF08EFE1FED380AD24880ED4C0AB6EE000A80ED500A0020CE4981F8E301022081F8DC010D2081F8DD0128F078FBC8490860084690EDA5
:401680004D0A80ED4F0A6CE0C54991F84200C349D1ED4C0AB0EE600A0FF043FE1FED4C0ABE4880ED4C0AB6EE000A80ED500A0820BA4981F8DC010F2081F8DD0151E0B748A9
:4016C00090ED500AB0EEC00ADFEDB60AB4EEE00AF1EE10FA07DA0146086828F06DFB4EF66021884207D92120AC4981F8DA01092081F8DC0135E0A94890F8DC01022819D19B
:40170000A649086828F058FB00EE100AB8EE400AFFEE000A20EE200A1FED701AC0EE010A9E4890ED4F0A30EE800A80ED500A18E01BE021E09949086828F03EFB00EE100A9F
:40174000B8EE400AF7EE000A20EE200A1FED7D1AC0EE010A914890ED4F0A30EE800A80ED500A00E000BF00BF24E002251FED800A8A4880ED500A1DE0FEF7FAFF874890F8DE
:40178000DA0120B10920854981F8DC0110E0844991F84200FEF7E5FD1020804981F8DD0103251FED8D0A084680ED500AFDF797FD00E000BF00BF794890F8DE01774991F84A
:4017C000DD11884214D0754890F8E101401C734981F8E101084690F8E101642802DD642081F8E1016D4890F8DD016C4981F8DE016A4890ED500AB5EEC00AF1EE10FA08D0D2
:40180000D0ED500AB0EE600A01210846F8F75FFE08E06248D0ED500AB0EE600A00210120F8F755FE2846BDEC048B70BD2DE9F0412DED048B042607F0ECFB10B1B3EE090A58
:4018400001E0B1EE040AB0EE409A07F0E2FB08B1554800E05548044607F0DBFB08B1544800E0544807464D4890F8DC010A2872D2DFE800F00506D77171D67171F9F800BF33
:40188000464890F8DD0120B110287DD011280ED000BF1120414981F8DD01B6EE000A084680ED500A28F060FA3C490860B6E03B49086828F081FAB0F5FA7F04D2A04737485D
:4018C00080ED090A89E03549086828F075FA40F6B831884205D29FED380A304880ED500A7BE02E49086828F067FA40F6AC51884217D2B6EE000A294880ED500AA0472748E0
:40190000D0ED090A30EE600AB4EEC90AF1EE10FA63DD1E20214981F8DA01092081F8DC015BE01E49086828F047FAB0F57A6F04D2A0471A4880ED090A4FE01849086828F086
:401940003BFA41F66411884206D29FED160A134880ED500A41E059E21049086828F02CFA41F6583188422CD2B6EE000A0B4880ED500AA0470948D0ED090A30EE600AF1EEF4
:40198000490AB4EEE00A00E028E0F1EE10FA24D21E20024981F8DA0109200FE0281100202021002000008C42BDB70008E7B30008C9B9000809B4000800008CC281F8DC01F3
:4019C0000BE0B6EE000AFE4880ED500A28F0CCF9FB490860102081F8DD011FE00520F84981F8DC010D2081F8DD01B6EE000A084680ED500A002081F8E30128F0B5F9F049B3
:401A000008609FEDF00A084680ED4C0A9FEDED0A80ED4F0A002081F8E10100BF00BFF6E100BFE74890F8DD0106282DD00D2802D00E287CD141E0FEF7A1FEB0EE000AB84729
:401A400090B1B6EE000ADE4880ED500A0620DC4981F8DD010E2081F8DF0128F085F9D849086010E068E16EE1D549086828F0A4F944F62061884206D92120D14981F8DA0164
:401A8000092081F8DC0155E1B6EE000ACC4880ED500A014608684FF4FA7128F06BF958B1C74890F8DF01C64981F8DD0100200860A047C34880ED090A3CE1C14890F8DC019C
:401AC000052806D1A047BE48D0ED090A70EE608A05E0A047BA48D0ED090A70EEC08AB848006818B928F040F9B5490860F4EEC98AF1EE10FA7EDDB24890F8E301002808DDBB
:401B0000AF4890ED4C0AD0ED500A30EE200A80ED4C0AAB4890F8E301401CA94981F8E301B6EE000A084680ED500A0D2000E000E181F8DD01086828F03FF900EE100AB8EE39
:401B4000400ADFEDA10A80EE208A9D4890F8E301012804D1B1EE040A28EE000A03E0B6EE000A28EE000AB0EE408A28F0FDF894490860084690F8DC01052816D1084690ED73
:401B80004F0A30EE080AF2EE040A30EE600A80ED4F0A90ED4F0AB5EEC00AF1EE10FA1AD29FED880A80ED4F0A15E0854890ED4F0A30EE480AF2EE040A30EE200A80ED4F0A60
:401BC00090ED4F0AB5EEC00AF1EE10FA03DD9FED7D0A80ED4F0A7A4890F8E30103283DDD7748D0ED4C0A90F8E30100EE100AB8EE400A00E04EE0B7EE001A30EE410A80EEB3
:401C0000801A6F4880ED4C1A90F8DC01052826D16E4991F842006A49D1ED4C0AB0EE600A0FF0A3FB9FED670A654880ED4C0AB6EE000A80ED500A0020614981F8E3010220DE
:401C400081F8DC010D2081F8DD0128F08DF85C4908609FED5C0A084680ED4F0A68E05B4991F842005649D1ED4C0AB0EE600A0FF058FB9FED540A524880ED4C0AB6EE000A21
:401C800080ED500A08204E4981F8DC010F2081F8DD014DE04A4890ED500AB0EEC00ADFED4C0AB4EEE00AF1EE10FA07DA0146086828F082F84EF66021884207D921204049CA
:401CC00081F8DA01092081F8DC0131E03C4890F8E30110B9B1EE040A01E0B6EE000AF0EE409A3749086828F067F800EE100AB8EE400A20EE290ADFED340A80EE201A304889
:401D000080ED501A90F8DC01022808D12C4890ED500AFFEE000A20EE200A80ED500A284890ED500AD0ED4F0A30EE200A80ED500A00E000BF00BF6AE002269FED220A2048C7
:401D400080ED500A63E01E4890F8DA0120B109201B4981F8DC0158E06425A8461B4991F84200694200EE101AB8EEC00A0FF0A5F9164991F84200694200EE101AB8EEC00AD1
:401D80000FF017FB114991F8420000EE105AB8EE400A0FF0F0F90D4991F8420000EE105AB8EE400A0FF029FB084890F8421040460FF063F8054890F8421040460AE0000090
:401DC000281100200000000000007A44202100200000A0420FF035FBFE4890F8421040460FF07EF8FB4890F8421040460FF047FB1020F94981F8DD0103261FED0E0A0846F7
:401E000080ED500AFDF76BFA00BF00E000BF00BFF14890F8DE01F04991F8DD11884214D0ED4890F8E101001DEB4981F8E101084690F8E101642802DD642081F8E101E648EC
:401E400090F8DD01E44981F8DE01E34890ED500AB5EEC00AF1EE10FA08D0D0ED500AB0EE600A01210846F8F732FB08E0DA48D0ED500AB0EE600A00210120F8F728FB3046A9
:401E8000BDEC048BBDE8F081002070471FED330AD14880ED720A1FED350A80ED740A1FED370A80ED6C0A1FED390A80ED6A0A1FED3B0A80ED700A1FED3D0A80ED6E0A7047F5
:401EC00070B52DED048B0446F0EE408AB0EE609AF0EE419A0D46BF4890F83000702804D0BC4890F8300093280CD1F7EE000A80EEA80A5FED4B0A89EE201A20EE010A20EE77
:401F0000298A6FE0B34890F8300091280ED0B14890F83000922809D0AE4890F83000712804D0AC4890F83000B8280CD1F0EE000A80EEA80A5FED5C0A89EE201A20EE010A09
:401F400020EE298A4EE0A81E0C283DD2DFE800F02D3C063C13203C3C3C3C2F2EF0EE080A80EEA80A5FED680A89EE201A20EE010A20EE298A35E0DFED990A80EEA80A5FED3E
:401F80006E0A89EE201A20EE010A20EE298A28E0DFED930A80EEA80A5FED750A89EE201A20EE010A20EE298A1BE000BF00BFDFED8D0A80EEA80A5FED7C0A89EE201A20EEAA
:401FC000010A20EE298A0CE0DFED870A80EEA80A5FED830A89EE201A20EE010A20EE298A00BF00BFB2EE040AB4EEC08AF1EE10FA04D2B2EE040AB0EE408A0AE09FED7B0A60
:40200000B4EEC08AF1EE10FA03DD9FED780AB0EE408A012C0AD16F4A92F84210BCEEC80A10EE102AD0B20FF00CFA09E0694A92F84210BCEEC80A10EE102AD0B20FF01FFAD7
:40204000BDEC048B70BD00B52DED028B95B0624890ED500A8DED140A27F086FE0E9004200C9014F017FB5C4880ED520AC0685A4948610846006988615D48007829F03BFE42
:402080005549C86027F070FE53490861084680690B9027F091FE4FF47A71B1FBF0F00F904D48C0684C494969401A00EE100AB8EEC00AF7EE000A20EE200A9FED4E1AC0EE60
:4020C000010A9DED0F0AB8EEC00A20EE800A8DED130A052148489DED130A15F032FB0521454808309DED140A15F02BFB1EF05CFB8DED0B0A1E21404818389DED0B0A15F097
:4021000020FB3E4890ED000A8DED0B0A1E213A4820389DED0B0A15F014FB384890ED000A2D4880ED510A3648007810F097FA8DED0B0A0521304808389DED0B0A15F001FB44
:402140003048007810F047FC8DED050A059832F02DF8CDE906019DED060B2EF001FC8DED080B9DED080B51EC100B31F0E3F905210B90214810389DED0B0A15F0E2FA15487E
:40218000B0F8BE014FF4967190FBF1F000EE100AB8EEC00A8DED0D0A0E4890F8280006284ED00C4890F82800072849D00A4890F8DC01042804D0084890F8DC0107283FD1B0
:4021C000054890ED740ADFED100AB4EEE00AF1EE10FA1BE02021002028110020CDCC4C406666A6408FC2753E9A99193F00007F435407002052EC2F45F01200209C550020FF
:402200000F070020600700200000484219DD90ED721A9DED0D0AF2EE040AF1EE041A41EEC00AB4EEE01AF1EE10FA79D20920FE4981F8DC01242081F8DA01002081F8DD012E
:402240006EE0F94890ED740ADFEDF80AB4EEE00AF1EE10FA19D290ED721A9DED0D0AFAEE040AF1EE041A41EE800AB4EEE01AF1EE10FA55DD0920EC4981F8DC01242081F828
:40228000DA01002081F8DD014AE0E748D0F8D001079031F08BFFCDE908019DED080B2EF05FFB8DED0A0B9FEDE20B53EC102B9DED0A0B51EC100B31F083FB31D1DDED0D0AC9
:4022C000B1EE040AB1EE041A01EE200A8DED070A079831F06BFFCDE90A01D348D0F8C801059031F063FFCDE906019DED060B2EF037FB8DED080B9DED0A0B53EC102B9DED49
:40230000080B51EC100B31F059FD09D20920C64981F8DC01242081F8DA01002081F8DD01C14890F8DD01062813D1BF48806801460B900E9827F04FFDBB494968884241F236
:40234000F283B94890F8DF01B74981F8DD0101F0EABBB54890F8DC010A2881F0E283DFE810F030000A0040006404E00B54024607E00BD60BC10BAC4890F8DB0180B1AA48DE
:4023800090F8DB01A84981F8DC01062081F8DD01002081F8DF01192048600E9888600EE00020A14981F8DC01062081F8DD01002081F8DF014FF47A7048600E98886001F075
:4023C000B1BB0220984981F8DC01062081F8DD01002081F8DF014FF47A7048600E988860EDE7914890F8DC018F4981F8DB01084690F8DD0108287CD003DC38B1052879D111
:4024000069E1092877D00B28F9D10BE00620864981F8DD010B2081F8DF01192048600E988860F0E18048806801460B900E9827F0D2FC41F28831884207D909207A4981F8CA
:40244000DC01262081F8DA0170E07B4890F8280006280ED0784890F82800072809D0724890ED520ADFED750AB4EEE00AF1EE10FA13DC714890F82800062804D06E4890F8B3
:40248000280007280FD1684890ED520ADFED6C0AB4EEE00AF1EE10FA05DDBBEE0E0A624880ED500A42E0644890F8280006280ED0614890F82800072809D05B4890ED520A2A
:4024C000DFED600AB4EEE00AF1EE10FA17D35A4890F82800062804D0574890F82800072813D1514890ED520ADFED570AB4EEE00A02E034E080E11AE0F1EE10FA05D2B3EEB4
:402500000E0A494880ED500A10E00620464981F8DD01092081F8DF014FF47A7048600E9888609FED4A0A084680ED500A6BE106203D4981F8DD01082081F8DF0119204860A4
:402540000E988860BAEE000A084680ED500A4048007829F0D0FB3449C1F8880153E1364890F82800062804D0334890F82800072810D12D48C0682C49D1F88811401A00EE08
:40258000100AB8EEC00ADFED330AB4EEE00AF1EE10FA40D3284890F8300091280FD0264890F8300092280AD0234890F83000712805D0214890F83000B82800D010E01A48D2
:4025C000C0681949D1F88811401A00EE100AB8EEC00ADFED210AB4EEE00AF1EE10FA1AD3154890F82800062851D0134890F8280007284CD00C48C0680B49D1F88811401A86
:4026000000EE100AB8EEC00ADFED120AB4EEE00AF1EE10FA3BD2084890F842000B909DED140A0EF07EFE19E028110020000048C2000000000000204020210020CDCCCC3C23
:40264000CDCC4C3DCDCCCCBCCDCC4CBD00000000540700206CE7DBC57390EAC40620FE4981F8DD01052081F8DF014FF47A7048600E9888609DED140A084680ED500AF748B5
:40268000007829F038FBF449C1F8880122E0F24890ED500A5FED1B0AB4EEE00AF1EE10FA0BD81FED160A80ED500A0920EA4981F8DC01272081F8DA010CE09DED140ADFED5B
:4026C000E80A30EE600A8DED140A9DED140AE24880ED500A97E0E048D0ED500A9FEDE11A80EE810A8DED010A019831F05FFDCDE902019DED020B2EF033F98DED060BD6481B
:40270000D0F8C001039031F051FDCDE904019DED060B53EC102B9DED040B51EC100B31F04FFA9FEDD10B53EC102BCDE908019DED080B51EC100B30F0EBFFCDE90A019DEDF8
:402740000A0B51EC100B30F0F5FEC349C1F85801084690ED6E0ADFEDC60A80EE201A80ED5A1AC44890F8300091280ED0C14890F83000922809D0BF4890F83000712804D078
:40278000BC4890F83000B82804D1B3EE090A8DED100A03E0B1EE040A8DED100A9DED100ADFEDB50A80EE201A9FEDB40A21EE000ABDEEC00AB8EEC00AA74880ED5E0AB0F8B1
:4027C000D80140F00400A449A1F8D8010521A24880F8DC110620A04981F8DD01002081F8DF014FF47A7048600E9888601FED690A084680ED500A06E000209749A1F8D801CA
:4028000081F8DC0100BF00BFD9E5934890F8DC01914981F8DB01084690F8DD0108287CD003DC38B1052879D167E1092877D00B28F9D10BE00620884981F8DD010B2081F88E
:40284000DF01192048600E988860ECE18248806801460B900E9827F0BEFA41F28831884207D909207C4981F8DC01282081F8DA0170E0804890F8280006280ED07D4890F89C
:402880002800072809D0744890ED520A5FED950AB4EEE00AF1EE10FA13DC764890F82800062804D0734890F8280007280FD16A4890ED520A5FED9E0AB4EEE00AF1EE10FA26
:4028C00005DDBBEE0E0A644880ED500A42E0694890F8280006280ED0664890F82800072809D05D4890ED520A5FEDAA0AB4EEE00AF1EE10FA17D35F4890F82800062804D097
:402900005C4890F82800072813D1534890ED520A5FEDB30AB4EEE00A02E034E07CE11AE0F1EE10FA05D2B3EE0E0A4B4880ED500A10E00620484981F8DD01092081F8DF0187
:402940004FF47A7048600E9888601FEDC00A084680ED500A67E106203F4981F8DD01082081F8DF01192048600E988860B2EE000A084680ED500A3948007829F0BCF93649C7
:40298000C1F888014FE13B4890F82800062804D0384890F82800072810D12F48C0682E49D1F88811401A00EE100AF8EEC00A9FED340AF4EEC00AF1EE10FA40DC2D4890F82E
:4029C000300091280FD02B4890F8300092280AD0284890F83000712805D0264890F83000B82800D010E01C48C0681B49D1F88811401A00EE100AB8EEC00ADFED220AB4EE36
:402A0000E00AF1EE10FA1ADC1A4890F8280006284FD0184890F8280007284AD00E48C0680D49D1F88811401A00EE100AB8EEC00ADFED130AB4EEE00AF1EE10FA39DD0D4844
:402A400090F842000B909DED140A0EF08EFC0620014981F8DD0117E02811002054070020CDCCCC3D0000C8420000000000408F4000007A4420210020000070428DED2448BD
:402A80006CE7DB457390EA44052081F8DF014FF47A7048600E9888609DED140A084680ED500AF948007829F026F9F849C1F8880122E0F64890ED500ADFEDF50AB4EEE00AF2
:402AC000F1EE10FA0BDB9FEDF30A80ED500A0920EE4981F8DC01292081F8DA010CE09DED140A5FED210A30EE200A8DED140A9DED140AE64880ED500A95E0E448D0ED500A24
:402B00001FED281A80EE810A8DED010A019831F04DFBCDE902019DED020B2DF021FF8DED060BDA48D0F8C001039031F03FFBCDE904019DED060B53EC102B9DED040B51EC70
:402B4000100B31F03DF81FED380B53EC102BCDE908019DED080B51EC100B30F0D9FDCDE90A019DED0A0B51EC100B30F0E3FCC749C1F86001084690ED6E0A5FED430A80EE46
:402B8000201A80ED5C1AC44890F8300091280ED0C14890F83000922809D0BF4890F83000712804D0BC4890F83000B82804D1B3EE090A8DED100A03E0B1EE040A8DED100A40
:402BC0009DED100A5FED540A80EE201A1FED550A21EE000ABDEEC00AB8EEC00AAB4880ED600AB0F8D80140F02000A849A1F8D801032081F8DC01062081F8DD01002081F8E9
:402C0000DF014FF47A7048600E9888609FEDA10A084680ED500A06E000209C49A1F8D80181F8DC0100BF00BFEEE5984890F8DC01964981F8DB01084690F8DD0130B10528C6
:402C40007ED007287DD00A287CD10BE006208F4981F8DD010A2081F8DF01192048600E988860C2E28948806801460B900E9827F0B2F842F21071884207D90920834981F866
:402C8000DC01262081F8DA01BCE0834890F8280006280ED0804890F82800072809D07B4890ED520A5FED920AB4EEE00AF1EE10FA13DC794890F82800062804D0764890F859
:402CC000280007282AD1714890ED520ADFED730AB4EEE00AF1EE10FA20DD6F4890F82800062804D06C4890F8280007280BD100BF694890ED300AF0EE040A30EE600A634817
:402D000080ED500A7EE0644890ED300AF2EE0E0A30EE600A5D4880ED500A73E05E4890F82800062812D05C4890F8280007280DD0564890ED520ADFED5A0AB4EEE00A02E0F1
:402D400061E0F5E14AE2F1EE10FA13D3524890F82800062804D0504890F8280007282AD14A4890ED520A5FEDC20AB4EEE00AF1EE10FA20D2484890F82800062804D04648C9
:402D800090F8280007280BD100BF434890ED320AF0EE040A30EE200A3C4880ED500A31E03D4890ED320AF2EE0E0A30EE200A374880ED500A26E00620344981F8DD010520DC
:402DC00081F8DF0140F6B83048600E988860324890F8280007280AD12F4890ED320ADFED310A20EE200A084680ED500A04E09FED290A264880ED500A00202449C1F88801C7
:402E0000C1F89401F1E12148D0F88801D0BB1E48007828F070FF1D49C1F88801084690ED6A0A80ED630A90ED6C0A80ED640A062081F8DD01072081F8DF01174890F828002D
:402E4000072803D14FF47A70486003E04FF47A700E4948600D490E9888600F4890F82800062804D00C4890F8280007281CD10A4890ED300AF2EE0E0A30EE600A034880ED1D
:402E8000500A54E11BE000005407002028110020000048420000000020210020CDCC4C3ECDCC4C3D9A99193FFE48D0ED300A1FED080A30EEC00AFC4880ED500A37E1FA4851
:402EC000D0F8940100287DD1F848007828F013FFF549C1F89401084690ED6A0A80ED660A90ED6C0A80ED670AD0F89401D1F88811401A0B9014F090FE00EE100AB8EE400A66
:402F0000DFEDEB0A20EE200ADFEDE90A80EE201AE54880ED5F1AD0F89401E349D1F88811401A00EE100AB8EEC00ADFEDE20AB4EEE00AF1EE10FA7DD2DA4890F828000628E5
:402F400004D0D84890F82800072804D19FEDDA0A8DED130A04E0D44890ED6C0A8DED130AD04890F82800072839D1CF4890F8E0010B90CC4890ED0F0A8DED0A0ACA4890ED35
:402F8000660A8DED090A0B989DED0A1ADDED130A9DED090A12F0CDFBC34880ED550A90F8E0010B90BF4890ED0F0A8DED0A0ABE4890ED630A8DED090A0B989DED0A1ADDEDD7
:402FC000130A00E0B3E09DED090A12F0B2FBB648D0ED550A30EEC00A80ED550A38E0B24890F8E0010B90AF4890ED0F0A8DED0A0AAD4890ED660A8DED090A0B989DED0A1A36
:40300000DDED130A9DED090A12F093FBA64880ED550A90F8E0010B90A24890ED0F0A8DED0A0AA14890ED630A8DED090A0B989DED0A1A00E06FE0DDED130A9DED090A12F04A
:4030400078FB9948D0ED550A30EEC00A80ED550A954890F8E0010B90934890ED570AB1EE400A8DED0A0A90ED550A8DED090A0B999DED0A1ADFED8E0A9DED090A0120FEF749
:403080001FFF894890ED550AF7EE000A80EE201A1FED800A31EE408A884800780FF0DEFADFED830A80EE201A7F4890ED570AB1EE400AC0EE010A7B4890ED300A9FED801A28
:4030C00010EE810AC8EE000A7748C0ED530AB0F8D80140F008007449A1F8D8010846B0F8D80140F01000A1F8D801062081F8DC0106216D4880F8DD11002180F8DF114FF4CB
:403100007A70694948600E9888601FED9E0A084680ED500A0BE01FEDA10A634880ED500A0920614981F8DC012B2081F8DA015CE006205D4981F8DD01052081F8DF010A2011
:4031400048600E9888600846D0ED500A9FED5C1A80EE810A8DED010A019831F027F8CDE902019DED020B2DF0FBFB8DED060B4E48D0F8C001039031F019F8CDE904019DED44
:40318000060B53EC102B9DED040B51EC100B30F017FD9FED4C0B53EC102BCDE908019DED080B51EC100B30F0B3FACDE90A019DED0A0B51EC100B30F0BDF93B49C1F85C0159
:4031C000084690ED6E0ADFED3A0A80EE201A80ED5B1ABAEE000A80ED500A06E000203249A1F8D80181F8DC0100BF00BFF0E32E4890F8DC012C4981F8DB01084690F8DD0186
:4032000030B105284DD0072879D00A2878D10BE00620254981F8DD010A2081F8DF01192048600E988860F1E31F48806801460B900E9826F0D0FD42F21071884207D9092092
:40324000194981F8DC01282081F8DA01D4E0154890F8280006280ED0124890F82800072809D0114890ED520ADFED180AB4EEE00AF1EE10FA13D30B4890F82800062804D09B
:40328000084890F82800072846D1074890ED520ADFED0F0AB4EEE00AF1EE10FA3CD2014818E0AAE020210020281100205407002000007A44FF4680C639B400400F0700208C
:4032C0000000C8420000000000408F40CDCCCCBDCDCC4CBE90F82800062804D0FE4890F8280007280DD100BFFB4890ED320AF0EE040A30EE200AF94880ED500A7CE093E372
:40330000E2E3F54890ED320AF2EE0E0A30EE200AF24880ED500A6FE0EF4890F8280006280ED0ED4890F82800072809D0EB4890ED520ADFEDEB0AB4EEE00AF1EE10FA13DC31
:40334000E54890F82800062804D0E34890F8280007282AD1E14890ED520A5FED240AB4EEE00AF1EE10FA20DDDB4890F82800062804D0D94890F8280007280BD100BFD648ED
:4033800090ED300AF0EE040A30EE600AD34880ED500A31E0D04890ED300AF2EE0E0A30EE600ACE4880ED500A26E00620CB4981F8DD01052081F8DF0140F6B83048600E9842
:4033C0008860C54890F8280007280AD1C24890ED300ADFEDC40A20EE200A084680ED500A04E09FEDC10ABD4880ED500A0020BB49C1F88801C1F8940172E3B848D0F8880115
:40340000D0BBBA48007828F076FCB449C1F88801084690ED6A0A80ED630A90ED6C0A80ED640A062081F8DD01072081F8DF01AA4890F82800072803D14FF47A70486003E07D
:403440004FF47A70A5494860A4490E988860A24890F82800062804D09F4890F8280007280BD19D4890ED320AF2EE0E0A30EE200A9A4880ED500AD6E20AE0974890ED320A0F
:40348000DFED9B0A30EE200A944880ED500ACAE29248D0F894010028EDD19448007828F02AFC8E49C1F89401084690ED6A0A80ED660A90ED6C0A80ED670AD0F89401D1F81D
:4034C0008811401A0B9014F0A7FB4FF47A71B0FBF1F000EE100AB8EE400A5FED8B0A20EE200A7E4880ED610AD0F894017B49D1F88811401A00EE100AB8EEC00ADFED7D0A87
:40350000B4EEE00AF1EE10FA7DDD734890F82800062804D0704890F82800072804D11FED9A0A8DED130A04E06C4890ED6C0A8DED130A694890F82800072837D1674890F8AB
:40354000E0010B90644890ED0F0A8DED0A0A634890ED660A8DED090A0B989DED0A1ADDED130A9DED090A12F0E4F85C4880ED550A90F8E0010B90584890ED0F0A8DED0A0AEF
:40358000564890ED630A8DED090A0B989DED0A1ADDED130A9DED090A12F0CBF84F48D0ED550A30EEC00A80ED550A38E04B4890F8E0010B90484890ED0F0A8DED0A0A474803
:4035C00090ED660A8DED090A0B989DED0A1ADDED130A9DED090A12F0ACF8404880ED550A90F8E0010B903C4890ED0F0A8DED0A0A3A4890ED630A8DED090A0B989DED0A1A8C
:40360000DDED130A00E002E29DED090A12F091F83248D0ED550A30EEC00A80ED550A2F4890F8E0010B902D4890ED590A8DED0A0A90ED550A8DED090A0B999DED0A1A5FED08
:40364000E40A9DED090A0220FEF73AFC234890ED550AF7EE000A80EE201A9FED230A31EE408A254800780EF0F9FF5FEDEF0A80EE201A1A4890ED590AC0EE010A164890ED54
:40368000320A1FEDF11A10EE810AC8EE000A1348C0ED540AB0F8D80140F040000F49A1F8D8010846B0F8D80140F08000A1F8D801084690ED560AD0ED580A30EE200A80ED5D
:4036C000560A90ED560AF0EE000A80EE201A80ED561A90ED570A11E02021002028110020CDCC4CBD9A99193F000000005407002000004842FF4680460F070020D0ED590A04
:4037000030EE200A80ED570A90ED570AF0EE000A80EE201A80ED571AD0ED5A0A90ED5C0A30EE800A80ED5A0A90ED5A0AF0EE000A80EE201A80ED5A1A90ED5B0AD0ED5D0A52
:4037400030EE200A80ED5B0A90ED5B0AF0EE000A80EE201A80ED5B1AD0ED5E0A90ED600A30EE800A80ED5E0A90ED5E0AF0EE000A80EE201A80ED5E1AD0ED5E0A9FEDFB0A42
:4037800020EE800A80ED5E0AD0ED5F0A90ED610A30EE800A80ED5F0A90ED5F0AF0EE000A80EE201A80ED5F1A90ED5F0ADFEDEF0A20EE200A80ED5F0A90ED5B0AD0ED5A0AF8
:4037C00070EE600A90ED570A90ED561A30EE411A80EE810A8DED0B0A9DED0B0A0AF0C7F8E34890ED5B0AE348D0ED700AE04890ED571A00EEC10A8DED0B0A9DED0B0A0AF077
:403800009CF8DB4890ED5F0AD0ED5E0A70EE600A90ED570A90ED561A30EE411A80EE810A8DED0B0A9DED0B0A0AF06DF8D04890ED5F0AD048D0ED720ACD4890ED571A00EEF4
:40384000C10A8DED0B0A9DED0B0A0AF042F8CA4800780EF003FFDFEDC90A80EE201AC54890ED700A21EE000AD0ED710AB2EE001A71EE600A80EE801A9FEDC10A21EE000AFA
:403880008DED130A90F82800062804D19FEDBD0A8DED110A1CE0B74890F8300091280ED0B44890F83000922809D0B24890F83000712804D0AF4890F83000B82804D19FED36
:4038C000B10A8DED110A03E09FEDAF0A8DED110AA748D0ED530A9DED110A80EE201AA54890ED300A31EE400A8DED120A9DED130ADFEDA30AB4EEE00AF1EE10FA10DD9DEDB6
:40390000120ADFED9F0AB4EEE00AF1EE10FA07DD90F842009FED9D0A0B900DF04AFD1DE09DED130ADDED120AB4EEE00AF1EE10FA0ADD904890F842000B909DED120AB1EE59
:40394000400A0DF036FD09E08A4890F842000B909DED130AB1EE400A0DF02BFD844890ED541A9DED110AC0EE010A824890ED320A30EE800A8DED120A9DED130ADFED800A25
:40398000B4EEE00AF1EE10FA10DD9DED120ADFED7C0AB4EEE00AF1EE10FA07DD90F842009FED770A0B900DF028FD1AE09DED130ADDED120AB4EEE00AF1EE10FA09DD6D4829
:4039C00090F842000B909DED120A0DF016FD08E0A8E0684890F842000B909DED130A0DF00CFD0820624981F8DC01062081F8DD01002081F8DF014FF47A7048600E988860F8
:403A00001FEDC70A084680ED500A0CE068E01FEDCA0A574880ED500A0920554981F8DC012B2081F8DA015BE00620514981F8DD01052081F8DF010A2048600E9888600846E0
:403A4000D0ED500A9FED4E1A80EE810A8DED030A039830F0ABFBCDE904019DED040B2CF07FFF8DED080B4248D0ED700A9FED431A80EE810A8DED050A059830F097FBCDE9AE
:403A800006019DED080B53EC102B9DED060B51EC100B30F095F8CDE90A019DED0A0B51EC100B2FF047FD3249C1F86401084690ED6E0ADFED320A80EE201A80ED5D1AB2EE1D
:403AC000000A80ED500A0BE000202949A1F8D80181F8DC011FEDFC0A084680ED500A00BF00BF1FE002200C900620214981F8DD01002081F8DF01192048600E9888609FEDF3
:403B0000240A084680ED500AFEF7C0F90AE003200C909FED1F0A164880ED500AFBF7DFFB00E000BF00BF124890ED500AB5EEC00AF1EE10FA0AD090ED500A8DED0B0A0121FE
:403B400008469DED0B0AF6F7C2FC0AE0084890ED500A8DED0B0A002101209DED0B0AF6F7B6FC0C9815B0BDEC028B00BD5F43BA3928110020202100200F07002000007A44EE
:403B80000000C8423333B33F3333B33E0000C8C20000000010B50124FB4890F8DA0170BB23F008FD68B1F94991F8300005F000FA18B1FDF73BFE04461FE0FEF744FA044630
:403BC0001BE023F00FFDC0B1F04890F82800072803D1FEF759F904460FE005F00BFA28B9EA4991F8300005F0E3F918B1FDF71EFE044602E0FDF7A6F80446FBF7F8F920460D
:403C000002F065FAE04890F8DA0120B1DE4991F8DA0102F065FF204610BD10B5DA4890F8DC010A284CD2DFE800F04C4D20054B21064B4B4E00BF0220D34981F8DD010020E8
:403C4000086012F081FDD04880ED080A90F8E301401CCD4981F8E301084690F8E3010A2802DD0A2081F8E30130E000BF0D20C64981F8DD0126F078F8C34908601FED3C0A8A
:403C8000084680ED4C0A002081F8E30105F0B2F970B1BD4890F8E101322804DD3220BA4981F8E1010BE00020B74981F8E10106E0B54890F8E101C01EB34981F8E10105E08E
:403CC00000BF00BF00BFFBF7F9F800BF00BFB0480021016241620020AB4981F8DA01B6EE000A084680ED500A10BD10B523F062FC10B302F0F1FE2B2802D1FBF7DFF81DE049
:403D0000A14890F8DB01A04981F8DC01062081F8DD01002081F8DF014FF47A70486026F023F8994988601FED660A084680ED500A002081F8DA0101E0FFF76FFF10BDB7EE75
:403D4000000A7047904890F8DA01704710B59148FCF760FA8F48FCF7E2F98E48FBF7D5FA10BD10B58B48FCF755FA8A48FCF7D7F98848FBF7CAFA10BD834890F8DC017047F3
:403D8000814890F8DD01704710B504247E4890F8DC01012804D106207B4981F8DC0186E04FF4FA717C48008825F0E4FF00287ED025F0DAFF78490880734890F8DC01801E04
:403DC000072872D2DFE800F0450571440471700000BF6D4890F8DD01801E0B2835D2DFE800F00634151F0B1A3434343410000620654981F8DD0129E00C20634981F8DD0176
:403E000024E00420604981F8DD011FE007205E4981F8DD011AE005205B4981F8DD0115E0594890F8DC01062807D10320564981F8DC01022081F8DD0106E00520524981F86B
:403E4000DC010D2081F8DD0100E000BF00BF2DE000BF4D4890F8DD01062804D00D2807D00E281ED109E00D20474981F8DD0119E00E20454981F8DD0114E0434890F8DC019C
:403E8000052809D10220404981F8DC01062081F8DD0105E00BE008E008203B4981F8DC0100E000BF00BF01E000E000BF00BF204610BD10B52DED088BB0EE408A05F0A9F883
:403EC00018B3F7F701FC00EE100AB8EE400A38EE400A10EE104A204630F068F941EC1B0BB0EE4B0AF0EE6B0A2CF03AFDB0EE40AAF0EE60AA9FED290B53EC102B51EC1A0B6D
:403F00002FF006FC41EC100B0BE018EE100A30F04DF941EC1A0BB0EE4A0AF0EE6A0A2CF01FFDB0EE409AF0EE609A51EC190B2FF001FB00EE100ABDEC088B10BD01B500BF87
:403F40000122694617480068433007F0E1FA20B99DF800000D4981F8430000BF08BD10B52DED020B00BF042269460E48006800F5DC7007F0CDFA20B99DED000A034880EDFD
:403F80006E0A00BF1CBD00002811002020210020A8120020181300208C0300200000000000005940F003002010B5044623F002FB00287DD0092C7CD005DC4CB1032C31D094
:403FC000062C77D158E00B2C75D00C2CF9D1E5E00120FE490870FA208861FA21FB48C16125F0C2FEF94948620121F84880F82810D0ED080AB0EE600AF548007827F020FFD4
:404000000020F24948604FF47A71F0488160416A0161002101759FEDEF0AEF48007827F00FFFF5E00120E9490870FA204860FA21E648816025F098FEE44908610121E3481F
:404040000175D0ED030AB0EE600AE348007827F0F7FE0020DD4988614FF47A71DB48C16101694162002180F828109FEDDA0AD848007827F0E5FECBE00120D44908704FF423
:404080007A7088610021D148C16125F06DFECF4948620121CD4880F82810D0ED080AB0EE600ACB48007827F0CBFE0020C74903E0AFE011E0ABE03AE048604FF47A71C3484D
:4040C0008160416A0161002101759FEDC20AC248007827F0B5FE9BE00120BC4908704FF47A7048600021B948816025F03DFEB74908610121B5480175D0ED030AB0EE600A86
:40410000B548007827F09CFE0020B04988614FF47A71AE48C16101694162002180F828109FEDAC0AAA48007827F08AFE70E00220A6490870642048600021A448816025F0E0
:4041400013FEA24908610121A0480175D0ED030AB0EE600AA048007827F072FE64209B49886100219948C16101694162002180F828109FED980A9648007827F061FE002034
:40418000924981F87C000121904880F87D10022180F88B10002180F88C1039E002208B4908704FF47A70486001468848816025F0DBFD86490861012184480175D0ED030A1E
:4041C000B0EE600A8448007827F03AFE4FF47A707E49886101467D48C16101694162002180F828109FED7B0A7948007827F028FE0020764981F87C000121744880F87D10FD
:40420000022180F88B10002180F88C1000E000BFDDE223F0E7F90028FAD0102C75D2DFE804F074083E75ABFA74E7E6E5E47474E3E2E10120654908704FF4FA70C8620146C1
:404240006248016325F090FD6049886301215F4880F83C106148007823F0EEF900205B4948604FF47A7159488160816B0161002101750020554908644FF47A7153484164B9
:40428000816BC164002180F850105348007823F0D3F900215248007823F0CEF996E201204A4908704FF4FA70086401464748416425F05AFD4549C8640121444880F8501011
:4042C0004748007823F0B8F90020404948604FF47A713E488160C16C01610021017500203A49C8624FF47A7138480163C16C8163002180F83C103848007823F09DF9002150
:404300003648007823F098F960E25EE201202F4908704FF4FA70486001462C48816025F023FD2A4908610121284801752A48007823F082F90020254908644FF47A7123483B
:4043400041640169C164002180F8501000201F49C8624FF47A711D48016301698163002180F83C101D48007823F066F900211C48007823F061F929E20120144908704FF437
:40438000FA70C86201461148016325F0EDFC0F49886301210D4880F83C101048007823F04BF94FF4FA700949086401460748416425F0DAFC0549C8640121044880F8501071
:4043C0000748007823F038F9002013E03816002029070020000000002A0700208107002078070020B5E172E129E1EEE0B7E080E049E010E0F74948600021F648816025F03B
:40440000B3FCF44908610021F2480175F248007823F012F9DAE10120EE4908703220C8623221EC48016325F09FFCEA4988630121E84880F83C10E948007823F0FDF83220AD
:40444000E44908643221E348416425F08DFCE149C8640121DF4880F85010E148007823F0EBF80020DB4948600021DA48816025F07BFCD84908610021D6480175D648007863
:4044800023F0DAF8A2E10120D24908704FF47A70C8620021CF48016325F066FCCD4988630121CC4880F83C10CC48007823F0C4F80020C84948604FF47A71C6488160816B3E
:4044C0000161002101750020C24908644FF47A71C0484164816BC164002180F85010BE48007823F0A9F80021BD48007823F0A4F86CE10120B74908704FF47A700864002128
:40450000B448416425F030FCB249C8640121B14880F85010B248007823F08EF80020AD4948604FF47A71AB488160C16C0161002101750020A749C8624FF47A71A5480163D5
:40454000C16C8163002180F83C10A348007823F073F80021A148007823F06EF836E101209C4908704FF47A70486000219948816025F0FAFB97490861012196480175964875
:40458000007823F059F80020924908644FF47A71904841640169C164002180F8501000208C49C8624FF47A718A48016301698163002180F83C108948007823F03DF800211D
:4045C0008748007823F038F800E10120814908704FF47A70C86200217E48016325F0C4FB7C49886301217B4880F83C107B48007823F022F84FF47A70764908640021754880
:40460000416425F0B1FB7349C8640121714880F850107348007823F00FF800206D49486000216C48816025F09FFB6A4908610021684801756848007822F0FEFFC6E00220E7
:40464000644908704FF47A70486000216148816025F08AFB5F49086101215E48017500215D48007822F0E8FF4FF47A705949C86200215848016301698163012180F83C1023
:4046800000215648007822F0D7FF4FF47A705149086400214F4841640169C164012180F8501000214E48007822F0C6FF0020494981F87C000221474880F87D10032180F8C2
:4046C0007E1080F88B10002180F88C107EE00220404908706420486000213E48816025F043FB3C49086101213A4801753A48007822F0A2FF64203749C86200213548016377
:4047000001698163012180F83C103448007822F093FF64202F49086400212E4841640169C164012180F850102D48007822F084FF0020284981F87C000221264880F87D10E2
:40474000032180F87E1080F88B10002180F88C103CE001201F4908704FF47A70486001461C48816025F000FB1A49086100211948017501211948007822F05EFF4FF47A70DE
:404780001449C86200211348016325F0EDFA1149886301210F4880F83C101048007822F04BFF00200B4908644FF47A710948416425F0DAFA0749C8640021064880F8501038
:4047C0000748007822F038FF00E000BF00BF0548047010BD381600202A07002081070020780700208E03002001B59DF8000000EE100AB8EE400AFE4880ED030A9DF800006E
:4048000000EE100AB8EE400AF94880ED080A00BF01226946F7480068403006F079FE20B99DF80000F44981F8400000BF0120F349087008BD08B506464FF4C8774FF000081C
:404840000121EF4880F8A8119421E9482AF003FF307818B94620FFF7C7FF11E0E64890F84050642D03DD6420FFF7BEFF08E00A2D03DA0A20FFF7B8FF02E02846FFF7B4FF66
:404880000020DB4981F88D0022F094FEE8B10020FFF78AFBDB48DFEDDC0A9FEDDC0A01230022DB490090DB48007826F02BFFD548DFEDD50A9FEDD50A01230022D649009092
:4048C000D648007826F01EFF05E022F08BFE10B10120FFF769FB0321C94880F8A81100BF012239464FF6FF70DFF834C300DF25F03BFA0446BE4890F88D00002874D10120CE
:4049000017F0D5FB18BB22F055FE68B1C548007818B9BA480078012805D10020FFF744FB0020B64908709EE022F05CFE0028FAD0BC480078052803D1B04800780128F2D1DF
:404940000520FFF731FB0020AC4908708BE001F0FAFA20BB22F02EFE70B1B2480078092803D1A648007801287DD10920FFF71CFB0020A249087076E022F034FE002872D0C8
:40498000A8480078022803D19C48007801286AD10220FFF709FB00209849087063E022F009FE70B19F480078062803D193480078012858D10620FFF7F7FA00208F4908703C
:4049C00051E022F00FFE28B396480078042803D18A480078012846D10420FFF7E5FA0020864908703FE0FFE7814890F88D00012823D122F0DFFD70B18A4800780C2803D1EB
:404A00007E48007801282ED10C20FFF7CDFA00207A49087027E022F0E5FD20B3814800780D2803D17548007801281CD10D20FFF7BBFA00207149087015E06D4890F88D0080
:404A4000022810D122F0CEFD68B1764800780F2803D16A480078012805D10F20FFF7A4FA00206649087062480078012802D002287ED115E15E48007D28BB5D48406810B31F
:404A80005B480169204625F0A6F95949896888423FD3012156480175046122F08BFD48B15348D0ED030AB0EE600A5C48007827F0C7F92EE022F096FD10B301215748007823
:404AC00022F0BAFD25E04A48007D012821D148488068A8B146480169204625F07CF944494968884215D3002141480175046122F061FD30B19FED4C0A4848007827F0A0F9A5
:404B000007E022F06FFD20B100214448007822F093FD374890F82800C8B935488069B0B13348416A204625F056F93149C96988422BD301212E4880F828104462D0ED080AE0
:404B4000B0EE600A3348007827F07AF91DE0284890F82800012818D12548C069A8B12448416A204625F037F921498969884200E0F6E10AD300211E4880F8281044629FEDAD
:404B80002A0A2448007827F05BF9194890F85000A8B91748006C90B11548C16C204625F01AF91349496C884245D30121104880F85010C4641D48007822F03EFD3BE00C48AE
:404BC00090F85000012836D10948406C80B30848C16C204625F0FFF80549096C88422AD30021034880F85010C4641048007820E038160020F0030020202100208F03002034
:404C00006852002070EC00200000FA4300247449001C004029070020002000402A070020412804088E030020000000007807002001E022F001FDD84890F83C00A8B9D6488A
:404C4000C06A90B1D448816B204625F0C4F8D249096B884223D30121CF4880F83C108463CE48007822F0E8FC19E0CB4890F83C00012814D1C848006B88B1C748816B2046E0
:404C800025F0A9F8C449C96A884208D30021C24880F83C108463C148007822F0CDFC5FE1BD4890F88C107C30405C78BBBA48007D01282CD1B8480169204625F08CF8B64936
:404CC0004968884221D30021B3480175046122F071FC30B11FED2C0AB148007827F0B0F80DE022F07FFC50B11FED310AAC48007827F0A6F80021AA48007822F09DFCA64875
:404D00008068002801D14FF00108C1E00BE0A2480169204625F05FF89F498968884201D34FF00108B4E09C4890F88C107C30405C01282BD1984890F8280001281AD196484D
:404D4000416A204625F047F893498969884210D30021914880F8281044621FED4D0A9148007827F06DF88C48C069002801D14FF001088DE08848416A204625F02CF886493E
:404D8000C969884201D34FF0010881E0824890F88C107C30405C022836D17F4890F83C00012825D17C48816B204625F014F87A49C96A88426CD30021774880F83C108463A8
:404DC0007648007822F038FC22F00CFC50B100217248007822F030FC1FED6D0A6F48007827F02EF86C48006B90BB4FF001084FE06948816B204624F0EEFF6749096B8842C9
:404E000046D34FF0010843E0634890F88C107C30405C03283CD1604890F8500001282CD15D48C16C204624F0D6FF5B49096C88422ED30021584880F85010C46422F0BAFB6C
:404E400038B11FED870A5748007826F0F9FF0EE01EE022F0C7FB50B11FED8D0A5248007826F0EEFF00215048007822F0E5FB4A48406C68B94FF001080AE04748C16C204638
:404E800024F0A9FF4449496C884201D34FF00108B8F1010F63D14FF000083F4890F88C00401CC1B23C4880F88C1090F88C1090F88B00814203DB0021374880F88C103648CE
:404EC00090F88C107C30405C022809D10121324880F83C1084633148007822F0ADFB3EE02D4890F88C107C30405C01280DD10121294880F828104462D0ED080AB0EE600A8A
:404F00002848007826F09CFF29E0234890F88C107C30405C032809D101211F4880F85010C4642148007822F087FB18E001211A480175046122F03EFB48B11748D0ED030A31
:404F4000B0EE600A1648007826F07AFF07E022F049FB20B101211248007822F06DFB00BFBEE42DE9F04106460C4617469846069D2078642803DD6420FFF736FC09E02078F3
:404F80000A2803DA0A20FFF72FFC02E02078FFF72BFCBDE8F081000038160020810700202A070020290700207807002070B544201CE0C41700EBD4646511CD4C54F82540D1
:404FC000C51700EBD5656D11A0EB45160125B5402C40C51700EBD5656D11A0EB45160125B540AC4200D103E0411EC8B20028E0DC00BF70BD30B5C31700EBD3635C11BC4BA6
:40500000183353F824300246C41700EBD4646411A0EB44150124AC4023430146C41700EBD4646511B24C183444F8253030BD13B50C4600BFAF49096801F5B0710819012250
:40504000694606F065FA18B99DF80010AA48015500BF1CBD13B50C4600BFA649096801F25F2108190122694606F052FA20B99DF80010A148FF30015500BF1CBD70B5044602
:405080009E480470E21704EBD2625311984A52F823202146E31704EBD3635B11A4EB43150123AB409A432046E31704EBD3635D118F4B43F82520E21704EBD26253118C4A3F
:4050C0000C3252F82320E31704EBD3635B11A4EB43150123AB409A43E31704EBD3635D11834B0C3343F82520E21704EBD26253117F4A183252F82320E31704EBD3635B11C2
:40510000A4EB43150123AB409A43E31704EBD3635D11774B183343F825200020FFF79AFF70BD30B50146CB1701EBD3635C11704B53F82430CC1701EBD4646411A1EB44154E
:405140000124AC4023400BB1012030BD0020FCE76B49087070476A480078704770B52DED048B04460025452C70D2DFE804F02324292E2F303139414951596169737C889112
:40518000ACB1FFFEFDFCFBFAF9F8F7F6F5F4F3F2F1F0EFEEEDECEBEAE9E8E7E6E5E4E3E2E1E0DFDEDDDCDBDAD9D8D7D6D5D4D3D2D19DD00003E30EF0D5FD80F00105FEE281
:4051C00022F0F0F980F00105F9E2F8E2F7E2F6E20FF09CFC18B1F8F7C1F800B10125EEE20FF094FC18B1F8F7B1F800B10125E6E20FF08CFC18B1F8F7B9F800B10125DEE213
:405200000FF084FC18B1F8F7C2F800B10125D6E20FF07CFC18B1F8F7B2F800B10125CEE20FF074FC18B1F8F7BAF800B10125C6E211F007FC012800D100E000200546BEE24D
:4052400011F0FFFB032802D1012001E0B6E200200546B4E22B4890F83800012800D100E000200546ABE20FF051FC38B1254890F8380008B9012000E0002005469FE221481C
:4052800090F89000012800D100E00020054696E20FF03CFC38B11B4890F8900008B9012000E0002005468AE2164890F83800022804D0144890F89000022801D1012000E058
:4052C000002005467BE209F09CFD80F0010576E20D48007DD0B90648001F006900F48020B0F5802F43D002F039FB78B101203FE0E4180020F8030020202700209803002072
:4053000099030020442900206C2A00202FE051E24CE23EE210E203E2FAE1EDE1E1E1D5E1CCE1C3E1B7E1AEE1A2E199E190E187E17EE175E16CE163E15AE151E148E13FE19C
:4053400036E12AE11EE10CE1E3E0D6E0C9E0BCE0AFE0A2E095E08BE080E075E05DE050E043E032E025E018E00FE00BE002E00020054624E2F748007D08B9012000E0002051
:4053800005461CE2F448057819E2F5F789F908B1012000E00020054611E20EF077FAB0EE408A9FEDEE1ADFEDEE0A0EF0EEF9054605E20EF06BFAB0EE408A9FEDEA1ADFEDFD
:4053C000EA0A0EF0E2F90546F9E102F0ADFFB0F57B4F07DB02F0A8FF4FF6FF71884201DA012000E000200546E9E102F05EFF28B1DE488078FE2801D0012000E000200546FA
:40540000DDE1DA488078FE2806D0F7F7C8FE18B101250020D6490872D1E1D4488078FE2805D0D448007810B103F06CFD20B101251C20FFF78DFE06E0FFF78DFE1C2802D198
:405440000020FFF785FEBAE1CB48007800F0A40008B1012000E000200546B0E1C648007800F0580008B1012000E000200546A6E1C2480088102801D0012000E000200546A2
:405480009DE10EF052FAB0EE408A9FEDB41ADFEDB60A0EF07AF9054691E10EF04EFAB0EE408A9FEDAE1ADFEDB00A0EF06EF9054685E10EF04AFAB0EE408A9FEDA81ADFED46
:4054C000AA0A0EF062F9054679E10EF007FAB0EE408A9FEDA21ADFEDA40A0EF056F905466DE10DF070FAB0EE408A9FED9C1ADFED9E0A0EF04AF9054661E10EF0F7F9B0EE0C
:40550000408A9FED961ADFED980A0EF03EF9054655E122F04FF818B3F5F719FDB0EE408AF5F7EAFC38EE400A10EE106A30462EF03DFE41EC190BB0EE490AF0EE690A2BF07C
:405540000FFAB0EE408AF0EE608A9FED8D0B53EC102B51EC180B2EF031FC00D2012500BF2DE1F5F7F4FCDFED880AB4EEE00AF1EE10FA04DDF4F7EFFA08B1012000E00020A6
:4055800005461CE102F0EAF920B903F04FF908B9012000E00020054611E102F0DFF920B108F0CEFC08B1012000E00020054606E10FF0ACFA18B103F0AFFD80F00105FEE0D1
:4055C000F5F779F808B1012000E000200546F6E0F5F790F808B1012000E000200546EEE0F5F715F908B1012000E000200546E6E0F5F74DF908B1012000E000200546DEE0F2
:40560000F5F782F908B1012000E000200546D6E0F5F7CEF908B1012000E000200546CEE0F5F706FA08B1012000E000200546C6E0F5F73AFA08B1012000E000200546BEE008
:40564000F5F76EFA08B1012000E000200546B6E0F5F7A6FA08B1012000E000200546AEE0F5F7DAFA08B1012000E000200546A6E00FF04CFA30B1F5F743FB08B1012000E067
:40568000002005469BE0F5F759FB08B1012000E00020054693E00FF039FA30B1F5F76CFB08B1012000E00020054688E0F5F78AFB08B1012000E00020054680E0F5F7A0FBBC
:4056C00008B1012000E00020054678E00FF01EFA30B1F5F7B3FB08B1012000E0002005466DE00FF013FA30B1F5F7C6FB08B1012000E00020054662E00EF0B3F906460EF034
:4057000033FA06430EB1012000E00020054656E00EF062FA08B1012000E0002005464EE00FF0F4F938B108F0A1FE012803D103F045FC00B9012542E0F4F751FF28B9F5F73F
:4057400040FC10B9F5F757FC00B303F037FCE8B901201CE0842A0020DD03002000FF7F4700A0254600007A460000000088DA0020583200203C050020ED030020BE0700206E
:40578000000000000070A7400000FA450020054615E00EF0C7FA20B9FE48007822F04EFB08B1012000E00020054608E003F07AF8054604E024F025FC054600E000BF00BFC3
:4057C00005B100BF3DB9F4480078002807DDF2480078844203D10120BDEC048B70BD0020FAE74FF00008C1464FF0010A4FF0500B0321EA4880F8B810002491E0E848005DC1
:4058000004EB840101EBC401E64A02EB810189680870E348FF30005D00287FD0E21704EBD2625311E04A52F82320E31704EBD3635B11A4EB431C012303FA0CF31A43E317E6
:4058400004EBD3634FEA631CD74B43F82C20E21704EBD2625311D44A0C3252F82320E31704EBD3635B11A4EB431C012303FA0CF31A43E31704EBD3634FEA631CCA4B0C3318
:4058800043F82C2004EB840000EBC400C54901EB8000007BE0B1E21704EBD2625311C24A183252F823202146E31704EBD3635B11A4EB431C012303FA0CF31A432046E31799
:4058C00004EBD3634FEA631CB74B183343F82C2024F04AFAB54941F8240000BFE21704EBD2625311B04A243252F823202146E31704EBD3635B11A4EB431C012303FA0CF328
:405900009A432046E31704EBD3634FEA631CA64B243343F82C2000E000E000BF601CC4B2452CFFF66BAF4FF47A60DFF884C200DF9A48D0F8DC100120DFF878C200DF4FF48A
:405940007A60DFF86CC200DF00BF002259460320DFF864C200DF0646022E21D1DFF85CC200DF074607F00200D0B1002416E0002004EB840101EBC4018A4A02EB810189684E
:40598000087004EB840101EBC40102EB8101896808782146FFF74BFB601CC4B2452CE6DB0024A9E22046FFF7D9FB05462046FFF7B8FBA8427ED0002D7DD1A946E31704EBDF
:4059C000D3634FEA631C784B0C3353F82C304FEAE47C04EBDC6C4FEA6C1CA4EB4C1E4FF0010C0CFA0EFC03EA0C034FEAE47C04EBDC6C4FEA6C1CA4EB4C1E4FF0010C0CFA52
:405A00000EFC634501D04FF0010904EB840000EBC400644901EB800090F8330000F0010008B14FF0010904EB840000EBC4005D4901EB800090F8330000F0020020B109F006
:405A40009CF808B14FF0010904EB840000EBC400544901EB800090F8330000F0040038B108F076FA10B921F0D0FD08B14FF0010904EB840000EBC4004A4901EB800090F813
:405A8000330000F0080020B1BAF1000F01D04FF0010904EB840000EBC400424901EB800090F8330000F0100038B14548005D012803D101E00FE00FE08146B9F1010F0AD157
:405AC00000203F4908554FF001082046FFF7D6FA3720F7F745FD02E1E31704EBD3634FEA631C314B53F82C304FEAE47C04EBDC6C4FEA6C1CA4EB4C1E4FF0010C0CFA0EFCE3
:405B000003EA0C034FEAE47C04EBDC6C4FEA6C1CA4EB4C1E4FF0010C0CFA0EFC6345DAD000202749085500BF01F018FFE8B1E21704EBD26253111C4A243252F823202146B4
:405B4000E31704EBD3635B11A4EB431C012303FA0CF31A432046E31704EBD3634FEA631C114B243343F82C2034E0E21704EBD26253110D4A243252F823202146E31704EB9A
:405B8000D3635B11A4EB431C012303FA0CF39A43204617E08E0700209A030020685200202027002094430408E4180020CC17002081270408E127040841280408892704084D
:405BC00085170020E31704EBD3634FEA631CF84B43F82C20E21704EBD2625311F44A243A52F82320E31704EBD3635B11A4EB431C012303FA0CF31A43E31704EBD3634FEA51
:405C0000631CEB4B243B43F82C2024F0ADF8E94941F8240004EB840000EBC400E64901EB800080680078401C04EB840101EBC401E14A02EB81018968087004EB840000EB82
:405C4000C400114601EB8000806800787E2808DD7E2004EB840101EBC40102EB81018968087000BF00BF01F079FE01281BD1E21704EBD2625311CE4A52F823202146E31796
:405C800004EBD3635B11A4EB431C012303FA0CF31A432046E31704EBD3634FEA631CC44B43F82C201AE0E21704EBD2625311C04A52F823202146E31704EBD3635B11A4EB83
:405CC000431C012303FA0CF39A432046E31704EBD3634FEA631CB64B43F82C2000BF002D7DD0E21704EBD2625311B14A183A52F82320E31704EBD3635B11A4EB431C012353
:405D000003FA0CF31A40002A53D104EB840000EBC400A94901EB8000406AE8BBE21704EBD2625311A24A183A52F82320E31704EBD3635B11A4EB431C012303FA0CF31A43B1
:405D4000E31704EBD3634FEA631C994B183B43F82C204FF0010804EB840000EBC40001EB8000806800787E2811DA04EB840000EBC40001EB800080680078401C04EB840109
:405D800001EBC4018C4A02EB81018968087021460120FFF75FF900E00CE004EB840101EBC401854A02EB8101896808782146FFF73EF95BE004EB840202EBC4027E4B03EB60
:405DC0008202516A7B4A52F8240023F0D3FFE8B3E21704EBD2625311754A183A00E083E052F82320E31704EBD3635B11A4EB431C012303FA0CF31A43E31704EBD3634FEA02
:405E0000631C6B4B183B43F82C204FF0010804EB840000EBC400684901EB8000806800787E2811DA04EB840000EBC40001EB800080680078401C04EB840101EBC4015E4AC4
:405E400002EB810189680870214600E00EE00120FFF700F904EB840101EBC401564A02EB8101896808782146FFF7E1F804EB840202EBC402504B03EB8202127BA2B3E2171A
:405E800004EBD26253114A4A0C3A52F82320E31704EBD3635B11A4EB431C012303FA0CF31A400ABB01F05AFD10B901F00CFCE0B104EB840000EBC4003F4901EB8000806AA1
:405EC00068B104EB840202EBC4020B4603EB8202916A384A52F8240023F04CFF20B12046FFF788F84FF0010804E02046FFF782F84FF00108601CC4B2452CFFF653ADB8F15D
:405F0000010F0BD12D48D0F8DC100120DFF8B0C000DF4FF000083720F7F722FB4FF0000AFFF744F8044610E5002108E02048243850F8210008B101207047481CC1B20329D8
:405F4000F4DB0020F8E7002108E019480C3850F8210008B101207047481CC1B20329F4DB0020F8E770B544201DE0C41700EBD46465110F4C0C3C54F82540C51700EBD5658B
:405F80006D11A0EB45160125B5402C40C51700EBD5656D11A0EB45160125B540AC4200D103E0411EC8B20028DFDC00BF70BD000008190020CC17002094430408685200202B
:405FC000E127040870B5002401F0C8FC78B344242AE0E31704EBD3635D11364B53F82530E51704EBD5656D11A4EB45160125B5402B40E51704EBD5656D11A4EB451601257E
:40600000B540AB420ED104EB840303EBC4032A4D05EB830393F83330102B03D1274B1B5D03B903E0601EC4B2002CD2DC00BF204670BD0121214A1154704701460020FF29A9
:4060400006DA1E4A525C0AB1012200E000221046704700B5002304E01846FFF7EAFF581CC3B2452BF8DB00BD0EB5154A07CA8DE807001CF0F9FB1DF08BFC0C226946FF205C
:406080001CF0BEFB0EBD014601EB810000EBC100094A52F820007047014601EB810000EBC100054A02EB8000007970477047054908707047F0180020944304088517002035
:4060C000985104089A030020FE48007B7047FD490873704770B52DED068B04460D46284623F06AFE00EE100AB8EE400AB0EE408A9FEDF50AC8EE000AB0EE608A94ED000AEA
:40610000D4ED020A00EE880ADFEDF00A68EE200A20EE200A10EE101A08462EF047F841EC1A0BB0EE4A0AF0EE6A0A2BF0D9FAB0EE409AF0EE609A51EC190B2DF0FBF908EE85
:40614000100A94ED040A20EE080AB0EE408AB0EE480ABDEC068B70BD10B52DED088BF0EE409AF0EE608A04469FEDD90AF0EE40AA9FEDD50AC0EE290AB0EE608AB1EE000AA7
:4061800028EE800AC0EE080AB0EE60AA9FEDD00AB0EE40BA204623F00FFEBCEEC80A10EE101AB0FBF1F201FB120000EE100AB8EE400AB0EE409AB5EE000A28EE000AB4EE34
:4061C000C90AF1EE10FA15D8B6EE080A28EE000AB4EEC90AF1EE10FA0CDDBFEE000A2AEE000AB0EE40AAB0EE000A28EE800AB0EE40BA0EE0B6EE080A28EE000AB4EEC90A5F
:40620000F1EE10FA05D8B9EE000A28EE800AB0EE40BAB0EE4B0A0AEE090AF0EE40AAB0EE6A0ABDEC088B10BD2DE9F0412DED028B05460F4690460024002600BF32E03221FC
:4062400008FB01F000EE100AB8EEC00ADFED9E0A80EE201A05F1300000EB840090ED000A30EE410A05F1300000EB840080ED000A08FB01F000EE100AB8EEC00ADFED920A31
:4062800080EE201A05F1700000EB840090ED000A30EE410A05F1700000EB840080ED000A601CC4B2082CCADB0024D8E007F1300000EB840090ED000A07F1700000EB840089
:4062C000D0ED000A30EE600AF0EE000A20EE200AB0EE408A05F1300000EB840090ED000A07F1300000EB8400D0ED000A30EE600A05F1900000EB860080ED000A05F19000D1
:4063000000EB860090ED000AC0EE080A9FED710A20EE800A05F1CC0000EB860080ED000A05F1500000EB840090ED000A05F1100000EB8400D0ED000A30EE600A07F1500014
:4063400000EB8400D0ED000A07F1100000EB840090ED001A70EEC10A80EE201A05F5847000EB860080ED001AB7EE000AC0EE080A05F5A27000EB8600C0ED000A701CC6B27B
:406380000F2E6ADA07F17000611C00EB810090ED000A07F1300000EB8400D0ED000A30EE600AF0EE000A20EE200AB0EE408A05F1700000EB810090ED000A07F1700000EB6A
:4063C0008100D0ED000A30EE600A05F1900000EB860080ED000A05F1900000EB860090ED000AC0EE080A9FED3B0A20EE800A05F1CC0000EB860080ED000A05F1500000EBDD
:40640000810090ED000A05F1100000EB8400D0ED000A30EE600A07F1500000EB8100D0ED000A07F1100000EB840090ED001A70EEC10A80EE201A05F5847000EB860080ED6A
:40644000001AB7EE000AC0EE080A05F5A27000EB8600C0ED000A701CC6B2601CC4B2082CFFF624AF1C4B0F221C4901F13C0013F0C8FA1B4B0F2219493C3901F1780013F0A2
:40648000C0FA154890ED010A0E4880ED1D0A124890ED000A0B4880ED230A114890ED010ADFED100A30EEC00AD0ED000A80EE201A044880ED261A0F210848783813F087FABA
:4064C000004811E02819002000007A44DB0FC940000000000000B443A0030020D81A0020A80300200000344380ED200ABDEC028BBDE8F08170B52DED028B0446B0EE408AE2
:406500000D46207800F0100000280AD094ED020A84ED030A84ED028AA078082802D10420208086E0207800F00100D8B394ED020AD4ED030AB4EEE00AF1EE10FA20DD94EDBF
:40654000020AFE48817804F1500000EB810080ED000AFB49486823F02FFC00EE100AB8EE400A5FED270A80EE201AF448817804F1700000EB810080ED001A0020E07002E07A
:40658000E078401CE070E0782179884251DD208840F002002080208820F0010020800020E07046E0FFE7207800F00200F0B394ED020AD4ED030AB4EEE00AF1EE10FA1ED2B1
:4065C00094ED020AA17804F1100000EB810080ED000ADB49486823F0EFFB00EE100AB8EE400A5FED470A80EE201AA17804F1300000EB810080ED001A0020E07002E0E07824
:40660000401CE070E0782179884212DD208840F001002080208820F002002080A078401CA0700020E0700DB1207900E001E0401E2071BDEC028B70BD10B52DED028BF0EE88
:40664000408AB0EE608ABE49486823F0B5FBB0F57A7F0BD90121B0EE480ABA48FFF74AFF0021B0EE680AB548FFF744FFB548008804280DD1B1480088042809D10222AF49E0
:40668000B048FFF7D1FD2020AE490880AB490880BDEC028B10BD70B52DED0C8B044602F074FD60B1F6F7B8FEB0EE408AD4ED098AF1EE009AB1EE00AAB0EE009A57E002F0CA
:4066C0009DFD40B3F5F704F80546F5F705F8281A00EE100AB8EEC00ADFED9B0A20EE200AB0EE40BAF5F76AF8DFED980A20EE208A94ED090ADFED950A60EE208AB1EE000AE2
:406700006BEE009AB1EE000A2BEE00AAB0EE000A2BEE009A2BE00FF0BDFFB0EE408A8C4991F8280091ED0F0AF0EE400AB0EE480A0FF0B4FEDFED870A20EE200AB0EE408A8E
:40674000834991F8280091ED0F1AF0EE410A94ED091AB0EE410A0FF0A1FEDFED7E0A60EE208AF0EE009AB0EE00AAB7EE009A4020005D40B994ED0B0A38EEC00A84ED0E0A91
:4067800001214020015519EE900A2DF00FFD41EC1B0B94ED0B0A30EE480A10EE101A08462DF004FD41EC1D0BB0EE4D0AF0EE6D0A2AF0D6F8B0EE40CAF0EE60CA53EC1B2B8E
:4067C00051EC1C0B2DF0FAFA0ED24C20005D58B9606823F0F1FA00EE100AB8EE400A84ED110A01214C2001551AEE100A2DF0DEFC41EC1B0B38EEC80A10EE101A08462DF045
:40680000D5FC41EC1C0BB0EE4C0AF0EE6C0A2AF0A7F8B0EE40DAF0EE60DA53EC1B2B51EC1D0B2DF091F90ED25820005D58B9606823F0C2FA00EE100AB8EE400A84ED140AED
:4068400001215820015519EE100A2DF0AFFC41EC1B0B38EEC80A10EE101A08462DF0A6FC41EC1C0BB0EE4C0AF0EE6C0A2AF078F8B0EE40DAF0EE60DA53EC1B2B51EC1D0BDF
:406880002DF09CFA0DD8002164200155607B324951F8200000EE100AB8EE400A84ED170A31E019EE100A2DF081FC41EC1B0B38EEC80A10EE101A08462DF078FC41EC1C0B8A
:4068C000B0EE4C0AF0EE6C0A2AF04AF8B0EE40DAF0EE60DA53EC1B2B51EC1D0B2DF034F911D26420005D70B9012164200155606823F062FA00EE100AB8EE400A84ED170A46
:4069000023F032FAA06078EEC8AA94ED0E0AB5EEC00AF1EE10FA0BD2B4EEE88AF1EE10FA06D294ED1B0AB4EEEA0AF1EE10FA24D394ED0E0AB5EEC00A10E00000501B002002
:4069400028190020D019002017B7D1380AD7233C20210020E02E6542A4510408F1EE10FA25DDB4EEE88AF1EE10FA20DD94ED1B0AB4EEEA0AF1EE10FA19DDC4ED1BAA94ED88
:406980001B0A10EE101A08462DF010FC41EC1C0BB0EE4C0AF0EE6C0A29F0E2FFB0EE40BAF0EE60BA51EC1B0B2CF0C4FDA066BDEC0C8B70BD00200022002100BF33E0FE4BBC
:4069C00003EB820393ED000AB5EEC00AF1EE10FA01D14B1C99B2F84B403303EB820393ED000AB5EEC00AF1EE10FA01D14B1C99B2F24B03EB820393ED000AB5EEC00AF1EEAD
:406A000010FA01D14B1C99B2EC4B403303EB820393ED000AB5EEC00AF1EE10FA01D14B1C99B2531CDAB2082AC9DB00224FE0E44B93ED1D0ADFEDE30AB4EEE00AF1EE10FA21
:406A400006DC93ED1D0AB5EEC00AF1EE10FA01D24B1C99B2DA4B93ED230ADFEDDA0AB4EEE00AF1EE10FA08DC93ED230ADFEDD60AB4EEE00AF1EE10FA01D24B1C99B2D04B69
:406A800093ED260ADFEDCF0AB4EEE00AF1EE10FA06DC93ED260AB5EEC00AF1EE10FA01D24B1C99B2C64B93ED200ADFEDC60AB4EEE00AF1EE10FA06DC93ED200AB5EEC00ADA
:406AC000F1EE10FA01D24B1C99B2531CDAB20F2AADDB01B901207047B94890F8A4007047B74981F8A4007047B548407B0C2823D0B348407B0B281FD0B148407B07281BD09D
:406B0000AF48407B112817D0AD48407B082813D0AB48407B0A280FD0A948407B04280BD0A748407B052807D0A548407B0F2803D0A348407B102801D1012070470020FCE763
:406B40009F48407B08281BD09D48407B042817D09B48407B052813D09948407B0A280FD09748407B0B280BD09548407B0F2807D09348407B102803D09148407B112801D1BC
:406B8000012070470020FCE78D48407B082817D08B48407B042813D08948407B05280FD08748407B0A280BD08548407B0B2807D08348407B102803D08148407B0F2801D1D7
:406BC000012070470020FCE77D48407B082803D07B48407B0A2801D1012070470020FCE770B5002428F000FA002872D101F05DFB18B10720FFF774FF80E008F002F930B936
:406C0000FFF7E2FF18B90220FFF76AFF76E019F0EBFDB5EEC00AF1EE10FA06D2FFF7B4FF18B90920FFF75CFF68E019F0DDFDDFED670AB4EEE00AF1EE10FA02D2FFF780FF9C
:406C400060B15F48407B0F280CD119F0D1FDDFED5F0AB4EEE00AF1EE10FA03D20420FFF73FFF4BE019F0C0FDDFED590AB4EEE00AF1EE10FA06DDFFF763FF18B90520FFF723
:406C80002FFF3BE05348007D18B90120FFF728FF34E0F3F7A4FC50B102F090F938B94848407B0F2803D10D20FFF71AFF26E007F04FFA28B107F04CFA0546FFF711FF1DE01D
:406CC000F6F776FB30B1F6F773FB0546FFF708FF14E01AE007F034F938B13948407B0B2803D02420FFF7FCFE08E0FFF72CF928B1FFF7FAFE10B90A20FFF7F2FEFFF7ECFEBE
:406D000018B10120FFF7E3F90124204670BDC9B1DFED310AC0ED000ADFED300AC0ED010A2F4AD2ED060AB8EE601ADFED2E1AC1EE210A9FED2D1AC1EE201AC0ED021A80EDA1
:406D4000040A1CE0DFED290AC0ED000ADFED280AC0ED010A224AD2ED0D0AB8EE601ADFED211AC1EE210ADFED231A81EEA01AF6EE000A61EE200AC0ED020A80ED040A7047D6
:406D800010B501219FED1C0A0D481030FFF7BFFF4FF4C0710848303828F05DFC4FF4C0710648303828F057FC0A2003493039087102493039087121E0001A0020801B002044
:406DC0002819002000409C4500409CC52FDDE43E2FDDE43F842A0020CDCCCC3D14AE473FA451040800007A447A142E3FCDCC4C3E0000204233331F42C2B8B23E1120FC4975
:406E00000880FC49088010BD2DED028B84B04FF47A66A821F84828F01EFC1421F74828F01AFC00BF002231460320DFF8D4C300DF0546022D70D1DFF8CCC300DF0446022C15
:406E40006BD1EE480078002867D0EC480078122863DC0120EC490870E8480078E649487322F082FFE4494860E44890ED010A084680ED090A407BE54908700020DE498860CA
:406E8000084600218166C1660167C165016641668163C163016441648164C1640165416581650020D44981F8A4000846407BD84951F82000D04908600846407B122877D2B1
:406EC000DFE800F0A5505354555609454D4E4CA0412C3A515246C848002141678167C1678030C160016141618161C1610162016041608160FFF744FF04208DF8040003201E
:406F00008DF8050005208DF80600022201A9FF201BF076FC04267BE0B0E07DE000219FEDBD0AB5481030FFF7F2FE9FEDBB0AB24880ED090A04266BE09FEDB80AAE4880EDB3
:406F4000090A042664E0F7F7ECFFC82660E000BFF7F7E7FFFCF7C9FEC82659E000BF00BF042655E000BF00BF00BF00BF00BF00BF02F00BF950B1F6F74FFAB0EE408A9E4843
:406F800080ED0B8A012180F834102BE002F036F978B1F4F713FCDFEDA20A20EE200AB0EE408A954880ED0B8A012180F8341019E02DE00FF06FFBB0EE408A9A4991F8280062
:406FC00091ED0F0AF0EE400AB0EE480A0FF066FADFED950A20EE200A874880ED0B0A012180F8341004208DF8040003208DF8050005208DF80600032201A9FF201BF000FCB2
:40700000042605E04FF4C87607F09BF900E000BF00BF042078490873012C2FD1002076494873002101209FED7C0AF3F750FA0020754908709FED780A704880ED010A9FED08
:40704000760A6D4880ED090A012180F864104FF47A665820F6F784FA5920F6F781FAFFF733F8042802D10020FFF731F811201AF0F1F8002201A9FF201BF0C2FB5E48407BCF
:4070800000287DD05C4A1168506822F073FE18BBFFF71AF804280FD05748407B07281BD05548407B112817D05348407B0B2813D05148407B0C280FD0FFF792FD60B94E4828
:4070C00090F8640001286DD14B49886840F6C41122F050FE002865D04748407B022807D04548407B012803D04348407B032819D1414890F8640030B93F4890ED000AB8EEF5
:40710000400A80ED170A3C4890F8580030B93A4890ED000AB8EE400A80ED140A5920F6F71FFA1FE03448407B06281BD1FFF742FC80B99FED3E0A304880ED1D0A9FED3B0AB9
:4071400080ED230A9FED390A80ED260A9FED370A80ED200A002026490880264908805820F6F7FEF911201AF075F8002022494873FEF7AAFF042802D10020FEF7A8FF00E014
:4071800010E0002101209FED240AF3F7A0F900201D4908709FED200A184880ED010A4FF47A663FE61448407B122879D2DFE800F0095279F5F3F2F1F0EFEEEDECEBEAE90A2C
:4071C0000BE81CE200BF02F019F888B3F4F794FB00EE100AB8EE400A074880ED090AD0ED090AB0EE600A0121032009F086FC2DE0D0190020501B0020281900201419002079
:4072000041280408892704089C030020B8030020A45104080000A04200000000000070420AD7233C20210020E02E6542003C1C46FFE71FED070AFC4880ED090AD0ED090A63
:40724000B0EE600A0121032009F0CDFAF648FFF722FAD4E101F0D2FF88B1F4F735FA00EE100AB8EE400AF04880ED090AD0ED090AB0EE600A0121032009F03FFC0CE01FEDEE
:407280001A0AE94880ED090AD0ED090AB0EE600A0121032009F0A7FAE348FFF7FCF9AEE193E101F072FF68B19FEDE00ADE4880ED090AD0ED090AB0EE600A0121032009F07C
:4072C00076FB59E001F09AFF00B3F4F7FDF900EE100AF8EE408AF4F7F7F98046F4F7FCF9A8EB000000EE100AB8EEC00ADFEDD00A40EEC08ACC48C0ED098AD0ED090AB0EEA2
:40730000600A0121032009F0F8FB35E020F07DF9D8B1C84890ED640ADFEDC70A20EE200A5FED410A20EE200AB0EE408A014691F8280091ED0F0AF0EE400AB0EE480A0EF0E2
:40734000C9FAB94880ED090A0DE0BA4991F8280091ED0F0AF0EE400A9FEDB80A0EF0BAFAB14880ED090AB048D0ED090AB0EE600A0121032009F037FAAB48FFF78CF93EE124
:40738000F9E0D0E0E5E00BE104E1F7E001E1F6E0F0E08FE07FE06FE0FFE701F0F6FE68B19FEDA50AA04880ED090AD0ED090AB0EE600A0121032009F0FAFA59E001F01EFF5A
:4073C00000B3F4F781F900EE100AF8EE408AF4F77FF98046F4F778F9A8EB000000EE100AB8EEC00ADFED920A40EE808A8E48C0ED098AD0ED090AB0EE600A0121032009F061
:407400007CFB35E020F001F9D8B18A4890ED650ADFED890A20EE200A5FED7F0A20EE200AB0EE408A014691F8280091ED0F0AF0EE400AB0EE480A0EF04DFA7B4880ED090A34
:407440000DE07C4991F8280091ED0F0AF0EE400A9FED7B0A0EF03EFA734880ED090A7248D0ED090AB0EE600A0121032009F0BBF96D48FFF710F9C2E06E4890F84210D030FE
:4074800000EB8100D0ED000AB0EE600A01210846F3F71DF8B3E0674890F84210D83000EB8100D0ED000AB0EE600A01210846F3F70EF8A4E05C4841681030FEF70BFE5A48B2
:4074C00080ED090A5B4991F8280091ED0F1AF0EE410A554991ED091AB0EE410A0EF0FAF9F0EE408A0121032009F07DF94E4890F82900B8B100204C4981F829000FF020F953
:40750000F0EE408A03214F4810F01BF94D4890ED001AF0EE410A444890ED091AB0EE410AFFF78AF86BE0404948684749D1ED000A464991ED000AFEF70FFE3B4880ED090AFA
:40754000D0ED090AB0EE600A01210846F2F7BFFF55E0354841681030FEF7BCFD324880ED090AD0ED090AB0EE600A01210846F2F7AEFF44E000BFFCF70DFB40E000BF2A48CC
:40758000D0ED090AB0EE600A01210846F2F79FFF35E034E006F0F7FD8046FEF798FD2EE0214A083202F11C0101F18000F9F79AFA8046FEF78CFD1C48D0ED090AB0EE600A60
:4075C00001210846F2F783FF19E00020164948730873002101201FEDF00AF2F778FF00201B4908701FEDF40A1A4880ED010A002201A9FF201BF004F94FF47A6600BF00BFE6
:40760000FEF762FD04287FF4CCAD4FF4FA71384622F0B0FB00283FF4C4AD22F0A5FB0746112019F017FEBCE52819002000008CC23333333F2021002000008C42C2B8B2BE9A
:40764000C2B8B23EB0030020C0030020BC0300209C0300201419002070B52DED028B0446B0EE408A0025B5EEC08AF1EE10FA0AD04CB1122C07DCAF4890ED010AB4EE480A1B
:40768000F1EE10FA0DD1AC48D0F890110120DFF8ACC200DF9FEDAA0AA64880ED010A00250DE00CB1A3480470A24880ED018AA248D0F890110220DFF884C200DF01252846A6
:4076C000BDEC028B70BD9F480078704701209E4981F8290070477A2303709B4BD3ED0E0A9FED9A0AB2EE041A00EE810ABDEEC00A10EE103A1AB24270130A8370924B93EDD3
:40770000110ABCEEC00A10EE103A99B2C1700B0A03718D4B93ED140ABCEEC00A10EE103A99B241710B0A8371874B93ED170ABCEEC00A10EE103A99B2C1710B0A0372824B32
:40774000D3ED1A0A9FED810AB2EE041A00EE810ABDEEC00A10EE103A1AB24272130A837270477B230370784BD3ED1D0A9FED781A9FED760A00EE810ABDEEC00A10EE103AB6
:4077800019B241700B0A83706F4BD3ED230A9FED701A9FED6E0A00EE810ABDEEC00A10EE103A19B2C1700B0A0371674BD3ED260A9FED671A9FED650A00EE810ABDEEC00A31
:4077C00010EE103A19B241710B0A83715E4B93ED200ADFED600A20EE200ABCEEC00A10EE103A9AB2C271130A0372704710B500245548407B122813D2DFE800F01314171809
:40780000191A1B091E1F1D0E121C1215160A00BFFCF7B2FA044611E006F08DFD04460DE000BF00BF00BF00BF00BF00BF00BF00BF00BF00BF00BF00BF00BF00BF00BF20462D
:4078400010BD10B500244048407B122813D2DFE800F013141718191A1B091E1F1D0E121C1215160A00BFFCF78BFA044611E006F062FD04460DE000BF00BF00BF00BF00BFF6
:4078800000BF00BF00BF00BF00BF00BF00BF00BF00BF00BF204610BD2B48407B70472A4890F86400704710B500242748407B122816D2DFE800F01718191A1B1C1D09202139
:4078C0001F16151E150E0F0A00BFF7F75AFB044613E000BFFFF7E3FF642110FB01F40CE000BF00BF00BF00BF00BF00BF00BF00BF00BF00BF00BF00BF00BF00BF204610BDF8
:40790000002011490873704713480078704710B500F0DBFF044644F6206122F02BFA38B900F0D3FF40F2DC51884201D9012010BD0020FCE71419002068520020E127040864
:40794000000000009C03002028190020000000470000C84200007A44B8030020FE490979042901D1012100E000210846704770B50023012113E0CC1701EBD4646511F74CF0
:4079800054F82540CD1701EBD5656D11A1EB45160125B5402C4004B10B46481CC1B24029E9DB184670BD70B504460D46E21704EBD2625311E94A52F823202146E31704EB39
:4079C000D3635B11A4EB43160123B3401A432046E31704EBD3635E11E04B43F826202846FDF7B6FB002C37D00821DD48DFF874C300DF012813D0DA482038817F807F401C87
:407A0000D74A203A907710464454807F1E2802DB002011468877D248DFF84CC300DF0821D248DFF840C300DF012815D022F09CF9CF4901EBC4014860CD4810F83400FF28C5
:407A400006DACB4810F83400401CC94901F83400C648DFF814C300DF70BDC6490870704710B5BD48007905287BD2DFE800F003152581DE00FEF767FA10B90220B64908716D
:407A8000BD48007838B10120BC490870FFF7E5FF0020B94908701AE1FEF755FA10B90220AD490871B448007828B10120B34908700020B14908700AE1FEF745FA18B1002039
:407AC000A549087153E0AC48007898B30120AB490870FEF738FA50B1FEF744FA044621460920FFF760FF0120FFF7B7FF3FE006F027FA38B129210320FFF755FF0120FFF764
:407B0000ACFF34E09E48007800F0080038B91A213120FFF748FF0120FFF79FFF27E003208D49087122F020F9964908600020FDF70FFB1CE0FFE7FFF7B2FEC0B909F04EFD73
:407B4000A8B1FFF7C0FD90B9FFF7E1FE78B118F04FFEDFED8D0AB4EEE00AF1EE10FA06DD00E0B3E09FED890A0F20FFF775FDAEE08148007800284DD006F0E2F950B1292149
:407B80000320FFF710FF0120FFF767FF01207B49087049E0FEF7D7F968B10120FFF75DFF012076490870FEF7DDF9044621460920FFF7F9FE38E04FF47A717248006822F0E5
:407BC000D9F890B16E48007800F0020008BB0120FFF743FF1A213120FFF7E5FE01206749087000205C4908711EE06548007800F00B0070B1FFF767FD30B16548D0F89011BB
:407C00000120DFF890C100DF04205349087106F0D8FF09E01A210220FFF7C5FE01205749087002204C49087151E05348007850B91A210220FFF7B7FE012050490870022005
:407C40004549087137E006F07BF968B129210320FFF7A9FE0220404908710120FFF7FDFE01204649087026E0FEF76DF980B10020394908710120FFF7F0FEFEF773F904469E
:407C800021460920FFF78FFE01203C49087012E0F5F79BFB78B100202F4908710120FFF7DCFEF5F792FB044621460920FFF77BFE01203249087028480079042805D022F022
:407CC00053F82549086006F07BFF00E000BF00BF214800792049487110BD2048001F0021016041608160C16070472B490870704710B52A4991F8300001F02AF930B10022B6
:407D000013466421264813F03FFD11E0234991F8300001F03FF928B9204991F8300001F041F928B10022134631211D4813F02CFD10BD10B50024194991F8300001F008F951
:407D400048B9164991F8300001F024F918B9134991F8300026E028E0C8030020701F00205C1F0020A92C0408C52B0408F81C00203C1D0020D2030020D3030020D403002047
:407D8000DC030020D80300202FDDE43E0000C84268520020E1270408D003002020210020C8DF002001F0FEF800B10124204610BDFE480078704710B50446FD480078844291
:407DC00004D0FB480470162019F044FA10BD00EE900AB8EE601ADFEDF70AF5EE001A51EE210AB0EE600ADFEDF40A80EE201AB0EE410A7047F1480078704710B52DED028BE4
:407E0000FFF7F8FF022807D0FFF7F4FF032803D0FFF7F0FF052812D10CF063FE30B10CF05AFE022802D19FEDE68A0AE00CF059FE10B19FEDE48A04E01FED2D8A01E01FED61
:407E40002E8AB0EE480ABDEC028B10BD10B52DED028B18F0ADFCB0EE408AFFF7CEFFB4EEC08AF1EE10FA03DB0120BDEC028B10BD0020FAE710B52DED048BF0EE408AB0EE83
:407E8000609A0446F0EE689AFFF7E0FF00EE100AB8EE400AB4EEC90AF1EE10FA07DDFFF7D5FF00EE100AB8EE400AB0EE409A29EE090ADFEDC50A80EE808AECB1F4EEC88A47
:407EC000F1EE10FA05DDF0EE489A0120BF49087015E0B1EE480AF4EEC08AF1EE10FA07D2B1EE480AF0EE409A0120B849087006E00020B649087002E00020B4490870B0EEAD
:407F0000690ABDEC048B10BD10B504460020206060606071207121F027FF206010BD2DED048B92B04FF05008002405E04FF6FF702DF81400601CC4B2022CF7DB0020FFF7F4
:407F4000D4FE00208DF80400A1490870FFF785FD0020A0490870A048DFF880C200DFA048DFF878C200DF9F48DFF870C200DF00209949183908759C48FFF7C6FF03219B482E
:407F800080F8441100BF002241460720DFF860C200DF0746022F7AD1DFF858C200DF054605F00200002873D010218B48DFF848C200DF012809D028228749183908A827F04F
:407FC00010FB8548DFF834C200DFBDF82060FFF7C5FC08B1012000E00020814618F0E8FBF0EE408A3046FFF7F2FEB0EE409A4846F0EE680AFFF73EFFB0EE408AFFF7AEFCF0
:4080000000B375481838007D01280BD1DDED0A0AB0EE600A0121042008F05CFC8146FFF7CAFE2FE06C481838007D02280BD1DDED090AB0EE600A0121052008F0B8FC8146C8
:40804000FFF7B9FE1EE064481838007D03280BD1DDED0B0AB0EE600A0121062008F04DFD8146FFF7A8FE0DE05B481838007D042808D101210220B0EE480A08F0B4FB8146FD
:40808000FFF799FE9DF83500012802D102E047E032E000205A4908709DF8350040B95948007840F00800574908700020FFF7D5FC4FF6FF7086421FD05248007800F0020095
:4080C000D0B95048007800F00800A8B1002410E03DF81410711A08B20FF097FD022806DC4848007840F002004649087003E0601CC4B2022CECDB00BF05F0040080B14248C7
:4081000001889DF80420501CC0B28DF804002DF812109DF80400022802DB00208DF804001CF017FA88B10BF01DFE70B1FFF740FE58B9364813F06AFB38B1FFF7FAFD08B1BF
:40814000FFF7D6FD0120FFF7D0FD9DF8360090B10C9821F031FEB0F5C87F0CD301201C4908702248D0F8B4100120DFF8A4C000DF0CF0D8FC02E00020154908702548007DD6
:40818000012854D19DF81C0028B900201D49087021F0EAFD824640F2E241504621F0EAFDD0B31FF032FAB8BB012036E0D0030020C60300200000FB4500007A44C403002015
:4081C0000AD7A33C9A99193ED222FB3FD5030020D1030020DD030020201D0020B52B04085C1F0020F81C0020C8030020685200204128040889270408A92C0408C52B040830
:40820000D3030020DC030020301D002070E10020E1270408542A002028E0FE490870FE48D0F8B4100120DFF8F4C300DF1EE09DF81C0001281AD1FA48007DB8B90020F54941
:408240000870FFF74AFDF448D0F8B4100120DFF8CCC300DFF348007840F00100F14908700120F149087021F07FFD82461822EC4902A827F0B6F9FFF7F3FBEB4800780128C6
:4082800009D1FFF774FBE94908700020E6490870172018F0DFFFFFF761FB08B1012000E000208146F3F72BFC6DE6E14800787047E04800787047E0480078704770B500254A
:4082C000DE48007D012801D1002405E0DB48007D08B9012400E002242543D948C472FDF732FE08B9012400E0002445EA8400C5B2D3484472D348007D08B9012406E0D14806
:40830000007D012801D1002400E0022445EA0410C5B2CB488472FFF7CEFF044645EA8415C7480472284670BDC748008870472DE9F04105460C4617469846069EB5F52D4FAC
:4083400028D12821C0481830DFF800C300DF012820D0A078BC49C875A07800F0030048752078617840EA0120B749088021F0FCFCB54908610120887504200875A648D0F88E
:4083800040110220DFF894C200DFAF481830DFF8C0C200DFBDE8F081F0EE400A9FEDAD0A30EEC01ADFEDAC1A81EE210A70472DE9F0412DED028B04460D4616461F46207887
:4083C000AD2833D12821A0481830DFF880C200DF01282AD0E0789C49C875E07800F0030048756078A17840EA012000EE100AB8EEC00AB0EE408AB0EE480AFFF7CDFF9248E6
:4084000080ED020A21F0B0FC8F4908610120887508758148D0F840110220DFF800C200DF89481830DFF828C200DF6BE02078A92834D1282184481830DFF810C200DF01282E
:4084400060D0E0788049C875E07800F0030048756078A17840EA012000EE100AB8EEC00AB0EE408AB0EE480AFFF796FF764880ED010A21F079FC74490861012088750220AD
:4084800008756548D0F840110220DFF890C100DF6D481830DFF8B8C100DF33E02078AF2830D1282168481830DFF8A0C100DF012828D0E0786449C875E07800F003004875DE
:4084C0006078A17840EA012000EE100AB8EEC00AB0EE408A5C4880ED038A21F045FC5A49086101208875032008754B48D0F840110220DFF828C100DF53481830DFF850C16E
:4085000000DF00BFBDEC028BBDE8F0811FEDD61A5FEDD80A40EE010AF1EE001AB6EE001A00EEA11AFCEEC10A10EE901A88B2704710B52DED028B0EF0ADF8B0EE408A9FED3D
:40854000470AB4EE408AF1EE10FA06D0B0EE480AFFF7DCFF3A49088003E04FF6FF70384908802D48D0F840110420DFF8B0C000DF33480088BDEC028B10BD70B58CB0064688
:408580000025002E6ED01FF040F8002878D040F2B240012102220023CDE90532CDE90710042017210193CDE902310490972013460022114600900AA812F0E8FE0AA93046E3
:4085C00012F0C7FB044640F292400440844204D11DB9042022490870012540F2B240012102220023CDE90532CDE90710042017210193CDE90231049097200123002211467F
:4086000000900AA812F0C2FE0AA9304612F0A1FB044629E0DD03002068520020E1270408542A0020DC030020D4030020C5030020D1030020C6030020D2030020842A002012
:40864000301D0020002A0020081D0020A92C0408C52B040800401C460000C84200FF7F47C40300200BE00BE040F292400440844205D1002DFCD10520954908700125B7E0DD
:4086800040F2B240012102220023CDE90532CDE9071017210193CDE902319720049300900123002211460AA812F070FE0AA9304612F04FFB044640F292400440844204D17F
:4086C0001DB9032082490870012540F2B240012102220023CDE90532CDE9071017210193CDE902319720049300901346002211460AA812F04BFE0AA9304612F02AFB0446D5
:4087000040F292400440844204D11DB9022070490870012540F2B240012102220023CDE90532CDE9071017210193CDE902319720049300900323002211460AA812F026FEB6
:408740000AA9304612F005FB044640F292400440844204D11DB903205D490870012540F2B240012102220023CDE90532CDE9071017210193CDE90231972004930090042363
:40878000002211460AA812F001FE0AA9304612F0E0FA044640F292400440844204D11DB902204B490870012540F2B240012102220023CDE90532CDE9071017210193CDE968
:4087C000023197201A461946049300900AA812F0DDFD0AA9304612F0BCFA044640F292400440844204D11DB9012039490870012515B15620F4F7B4FE28460CB070BD10B501
:40880000344890F8280007280DD117F0D1FFDFED320AB4EEE00AF1EE10FA01DB012000E00020044600E00124204610BD10B517F0BFFFDFED2A0AB4EEE00AF1EE10FA01D854
:40884000012010BD0020FCE710B5FFF7FFFA20B9204890F8FF01032801D1012010BD0020FCE79FED1F0A70479FED1E0A70471848007803280FD01648007802280BD01448AC
:408880000078012807D012480078042803D010480078052801D1012070470020FCE712480079704710B500F05AFC10B10F48047800E00024204610BDF0EE400A1FED9A1A7D
:4088C0001FED9C0A00EE810A7047074800687047C4030020202100202FDDE43E83C00041B81E4141A2454841C8030020D503002010B5044600BF28222146FE48006802F064
:4089000007FE20B928222146FB4826F025FE00BF10BD10B504462822F749204626F01CFE10BD01B500BF04226946F2480068283002F0EEFD18B99DF80000EF49886200BF3C
:40894000EE48C16B0220DFF8B8C300DF08BD01B500BF04226946E74800682C3002F0D8FD18B99DF80000E449C86200BF08BD01B5E14890F830000099884219D000BF042270
:408980006946DC480068303002F0C2FD10B9DA490098086300BFD84890F83000922804D0D54890F83000932802D101201BF008F808BD10B52DED020B00BF04226946CD486E
:4089C00000683C3002F0A4FD20B99DED000ACA4880ED0F0A00BF04F028F8C848C16B0220DFF81CC300DF0220F4F7BAFD5020F4F7B7FD1CBD01B500BF01226946BD480068E5
:408A0000483002F085FD20B99DF80000BA4981F8480000BF08BD08B5002000901EF0E2FDA0B10021B74800781EF006FEB64800781FF004FA28B10220FFF7DCFF012000903F
:408A400004E00120FFF7D6FF0220009000BF01226946A8480068493002F05AFD20B99DF80000A54981F8490000BFA448016D0120DFF88CC200DF08BD01B500BF042269465E
:408A80009C480068443002F043FD10B99A490098486400BF08BD01B5974890F841009DF80010884215D000BF0122694691480068413002F02DFD20B99DF800008E4981F881
:408AC000410000BF19F0D0FE08F097FD1F20F4F747FD08BD01B500BF0122694685480068423002F015FD20B99DF80000824981F8420000BF19F0B8FE2620F4F731FD7F4856
:408B0000C16B0220DFF8F8C100DF08F076FD08BD01B500BF042269467C480068AC3002F0F7FC18B974480099C0F89C1400BF08BD70B52DED028B04460D4616461EF03AFDF5
:408B4000F8B16D49E0314A5D891C495D501800EBD071491000EE101AB8EEC00AB0EE408ABCEEC80A10EE101AC8B2294608F085F9BCEEC80A10EE101AC8B2294608F0B0F985
:408B80000EE01EF02FFD58B15B49E031485D294608F073F95849E231485D294608F0A0F95B4800EB8400D0ED000AB0EE600A2946204608F01AF856490831085D2A4621462A
:408BC00008F064F852490A31085D2A46214608F0D9F84F490C31085D2A46214608F00FF946B11D2018F036FB4448016D0120DFF810C100DFBDEC028B70BD70B500240CE08E
:408C0000002506E0002229462046FFF791FF681CC5B2022DF6DB601CC4B2022CF0DB1D2018F018FB3548016D0120DFF8D4C000DF70BD70B52DED028B04460D461EF0BAFCBE
:408C400000B32D48D03000EB840090ED000AB1EE400A2948D83000EB8400D0ED000A30EE200AF0EE000A80EE201AB0EE418A2046B1EE480A08F021FA2046B0EE480A08F045
:408C80007AFA18E01EF0AEFCA8B11B48D03000EB8400D0ED000AB0EE600A204608F00DFA1548D83000EB8400D0ED000AB0EE600A204608F060FA1048C03000EB8400D0ED62
:408CC000000AB0EE600A204608F03DF90A48C83000EB8400D0ED000AB0EE600A204608F090F9FDB1192018F0B5FA1D2018F0B2FA19200FE0F003002020210020685200205A
:408D0000E12704087307002093070020F40300200423002018F09EFAF748016D0120DFF8DCC300DFBDEC028B70BD10B5002405E000212046FFF77DFF601CC4B2022CF7DB8E
:408D4000192018F087FA1D2018F084FA192018F081FAE948016D0120DFF8A0C300DF10BD70B505460C4600212046FFF762FF002221462846FFF7DCFE70BD70B52DED028BAC
:408D800005460024A1E0DE4890F8491005F1380000EB81100E3030F9140000EE900AF8EEE00AB0EE600A204608F0BBFAD44890F8491005F1380000EB8110123030F91400FE
:408DC00000EE900AF8EEE00AB0EE600A204608F0CCFACB4890F8491005F1380000EB8110163030F9140000EE900AF8EEE00AB0EE600A204608F0DDFAC14890F8491005F159
:408E0000380000EB81101A3030F9140000EE900AF8EEE00AB0EE600A204608F0EEFAB84991F8492005F1380101EB82110A31085D214608F006FBB24991F8492005F1380194
:408E400001EB82110C31085D214608F018FBAC4890F8491005F1380000EB8110401C005D00EE100AB8EE400ADFEDA60A80EE201AB0EE418A2046B0EE480A08F01EFBA04952
:408E800091F8492005F1380101EB8211091D085D214608F02BFB9A4991F8492005F1380101EB8211891D085D214608F033FB944991F8492005F1380101EB82110831085DCC
:408EC000214608F03BFB601CC4B2022CFFF65BAF8B4890F8491005F1380000EB8110D0ED080AB0EE600A08F0E0F9854991F8492005F1380101EB8211C87807F003FFBDEC68
:408F0000028B70BD7E4890F8280008B9012070470020FCE710B501201AF091FD01467A4880F8391000201AF08AFD7749487401201AF085FD04462146012011F0FBFE002057
:408F40001AF07DFD04462146002011F0F3FE10BD01460020282901D1012200E00022402901D1012300E000231A43492901D1012300E000231A434A2901D1012300E000233B
:408F80001A434B2901D1012300E000231A4302B10120704701460020562901D0782900D10120704701460020592900D10120704701460020712900D10120704710B50024D9
:408FC0004F4890F8300091280ED04D4890F83000922809D04A4890F83000712804D0484890F83000B82803D11EF0FCFA00B10124204610BD424890F82810082905D0092969
:4090000003D00A2901D00E2901D1012070470020FCE73B4890F828100A2901D1012070470020FCE7364890F82810082901D1012070470020FCE7324890F82810092901D1F8
:40904000012070470020FCE72D4890F828100E2901D1012070470020FCE710B504461EF0C1FA70B11EF0D1FA00B92CB90121274800781EF0E1FA04E00021244800781EF0A3
:40908000DBFA10BD1E4890F8300000EBC00101EB00101F4901EB0010408E70470246012109E001EB01101B4B13F81000904201D1C8B27047491C2229F3DB0020F9E71048E3
:4090C00090ED0F0A70470E4890F84900022801D1012070470020FCE7094890F84900012800D170470020FCE7054890F8490008B9012070470020FCE768520020E1270408A7
:40910000202100200000C84248E100206E07002070560408EC51040810B50024FFF7E4FF08B1012419E01EF05DFAB0B1FFF7D4FF20B1634800781EF081FE68B9FFF7C3FF49
:4091400058B1F1F759FA38B9F1F756FA28B95C4800781EF073FE00B90124204610BD594890F8970020B1574890F89700012801D1012070470020FCE7524890F82800072857
:4091800001D1012070470020FCE74E4890F89700022804D04B4890F89700032801D1012070470020FCE7474890F89700032801D1012070470020FCE7424890F8970002286C
:4091C00001D1012070470020FCE73E4890F8970008B9012070470020FCE73A4890F89700012800D170470020FCE7364890F89700042801D1012070470020FCE7314890F8B5
:409200009700042801D1012070470020FCE701B500BF012269462C480068973002F078F920B99DF80000274981F8970000BF08BD01B500BF012269462348006800F285303E
:4092400002F066F920B99DF800001E4981F8850300BF08BD10B500241A4890F83000282827D0184890F83000402822D0154890F8300049281DD0134890F830004A2818D0A7
:40928000104890F830004B2813D00E4890F8300059280ED00B4890F830005C2809D0094890F83000782804D0064890F830001D2800D101242046FFF7BBFF204610BD00006C
:4092C0009307002020210020F00300201FB51EF0B0F9062808D01EF0ACF9072804D01EF0A8F9082841F077821EF08FF900287DD0002000900190029003460122FE490390CC
:409300001EF071FA002000900190029003460322FA49039001201EF066FA002000900190029003460322F649039002201EF05BFA002000900190029003460322F149039068
:4093400010461EF050FA002000900190029003460322ED49039004201EF045FA002000900190029003460422E849039005201EF03AFA002002220123CDE9012000930390F2
:4093800003460322E24906201EF02DFA002000900190029003460246DE49039007201EF022FA002000900190029003460322DA49039008201EF017FA002000900190029039
:4093C00003460122D549039009201EF00CFA002000900190029003460122D14903900A201EF001FA00200090019000E0E0E3029003460122CB4903900B201EF0F4F9002025
:4094000001210090CDE9010103460A46C64903900C201EF0E8F9002000900190029003460246C249039011201EF0DDF9002000900190029003460322BD49039012201EF03B
:40944000D2F900200222CDE9000202900346B949039016201EF0C7F9002001210090CDE9010103460A46B449039017201EF0BBF9002000900190029003460222AF4903903A
:4094800019201EF0B0F900200222CDE9000202900346AB4903901A201EF0A5F9002000900190029001230222A64903901B201EF09AF9002000900190029001230222A249F9
:4094C00003901C201EF08FF900200222CDE90002029003469D4903901E201EF084F900200222CDE90002029003460246984903901F201EF078F90020009001900290034681
:4095000003229449039021201EF06DF90020009001900290034603228F49039022201EF062F90020009001900290034603228B49039023201EF057F900200090019002906E
:40954000034603228649039024201EF04CF90020009001900290034603228249039025201EF041F90020009001900290034603227D49039026201EF036F9002000900190FA
:409580000290034601227949039027201EF02BF90020009001900290034601227449039028201EF020F90020009001900290034601227049039029201EF015F90020009041
:4095C00001900290034602226B4903902B201EF00AF9002000900190029003460222674903902C201EF0FFF8002000900190029003460122624903902D201EF0F4F8002080
:40960000009001900290034601225E4903902E201EF0E9F8002000900190029003460122594903902F201EF0DEF80020009001900290034601225549039031201EF0D3F853
:409640000020009001900290034601225049039032201EF0C8F800200121CDE9000103460A46CDE902104B4936201EF0BCF8002000900190029003460122474903903B209C
:409680001EF0B1F8002000900190029003460122424903903C201EF0A6F800200122CDE90002029003463E4903903D201EF09BF800200122CDE900020290034639490390B5
:4096C0003E201EF090F8002001210090CDE9010103460A463449039041201EF084F80020009001900290034601223049039042201EF079F800205BE03707002054070020F8
:409700005307002097070020980700205707002058070020A3070020550700206B0700206A070020690700208B070020200700205D070020130700202A07002014070020F9
:4097400019070020990700209A070020180700201D0700200D0700200F07002060070020610700206207002063070020650700206407002066070020670700206807002058
:40978000590700205B0700205A0700206C0700206D0700206E07002070070020710700207207002073070020740700203E07002000900190029003460122FE4903904320AC
:4097C0001EF011F8002000900190029003460122F949039044201EF006F8002001210090CDE9010103460A46F449039048201DF0FAFF002001210090CDE9010103460A464A
:40980000EF4903904B201DF0EEFF002001210090CDE9010103460A46EA4903904D201DF0E2FF002000900190029003460322E64903904F201DF0D7FF012000220092CDE9D4
:40984000012013460246E149039050201DF0CBFF002001210090CDE9010103460A46DC49039051201DF0BFFF002000900190029003460122D749039052201DF0B4FF0020C7
:4098800000900190029003460322D349039054201DF0A9FF002000900190029003460322CE49039055201DF09EFF002000900190029003460322CA49039056201DF093FFA9
:4098C000002000900190029003460322C549039057201DF088FF00200222CDE90002029003460246C049039057201DF07CFF002000900190029003460322BC490390582070
:409900001DF071FF002000900190029003460322B749039059201DF066FF002000900190029003460322B34903905A201DF05BFF002000900190029003460322AE4903906F
:409940005B201DF050FF002001210090CDE9010103460A46A94903905C201DF044FF002000900190029003460122A54903905D201DF039FF002000900190029003460122DB
:40998000A04903905E201DF02EFF0020009001900290034601229C4903905F201DF023FF00200222CDE900020290034601229749039061201DF017FF00200222CDE9000201
:4099C0000290034601229249039062201DF00BFF0020009001900290034601228D49039064201DF000FF0020009001900290034601228949039065201DF0F5FE00200121BF
:409A00000090CDE9010103460A468449039067201DF0E9FE002001210090CDE9010103460A467F49039069201DF0DDFE00200222CDE900020290034602467A4903906A207C
:409A40001DF0D1FE01200021009101910B460246CDE9021074496B201DF0C5FE00200222CDE9000202900346704903906D201DF0BAFE00200222CDE90002029003466C492B
:409A800003906E201DF0AFFE00200222CDE9000202900346674903906F201DF0A4FE002001210090CDE9010103460A466249039073201DF098FE00200222CDE9000202904E
:409AC000034602465D49039079201DF08CFE002000900190029003460222594903907A201DF081FE002000900190029003460122544903907B201DF076FE00200090019005
:409B0000029003460122504903907C201DF06BFE0020009001900290034601224B4903907D201DF060FE002001210090CDE9010103460A46464903907E201DF054FE002019
:409B400000900190029003460122424903907F201DF049FE002001210090CDE90101034602223D49039082201DF03DFE002001210090CDE90101034602223849039083200D
:409B80001DF031FE002001210090CDE90101034602223349039084201DF025FE01200021009101910B460222CDE902102D495BE0DAE0000075070020760700209B07002087
:409BC0009C0700208A07002056070020770700207807002079070020A0070020A1070020A2070020A4070020250700207E0700207F070020800700201B070020810700204C
:409C00008307002084070020820700205F0700205E070020850700208607002087070020890700204B070020380700209D0700209E0700209F0700208C0700208E070020DC
:409C40008F070020310700203207002090070020910700208D0700203B0700203C0700203D0700209307002086201DF0BCFD01200021009101910B460222CDE90210FE4922
:409C800087201DF0B0FD01200021009101910B460246CDE90210F94988201DF0A4FD002000900190029003460322F54903908E201DF099FD00200090019002900346032241
:409CC000F04903908F201DF08EFD002000900190029003460322EC4903908F201DF083FD012009F060FD0021E84800781DF0A4FC0021E74800781DF09FFC0021E5480078E9
:409D00001DF09AFC0021E44800781DF095FC01200021009101910B460222CDE90210DF4986201DF060FD01200021009101910B460222CDE90210DA4987201DF054FD012157
:409D4000D84800781EF0FDF80121D74800781EF0F8F80121D54800781EF0F3F80121D44800781EF0EEF8E1E3002000900190029003460122CF4903901DF035FD002000909A
:409D80000190029003460322C649039001201DF02AFD002000900190029003460322C249039002201DF01FFD002000900190029003460322C049039010461DF014FD002080
:409DC00000900190029003460322BC49039004201DF009FD002000900190029003460422B749039005201DF0FEFC002002220123CDE901200093039003460322B14906207F
:409E00001DF0F1FC002000900190029003460322A749039007201DF0E6FC002000900190029003460322A149039008201DF0DBFC002000900190029003460122A2490390C7
:409E400009201DF0D0FC0020009001900290034601229E4903900A201DF0C5FC002000900190029003460122994903900B201DF0BAFC002001210090CDE9010103460A466A
:409E8000944903900C201DF0AEFC0020009001900290034603229049039011201DF0A3FC0020009001900290034603228B49039012201DF098FC00200222CDE900020290BC
:409EC00003468749039016201DF08DFC002001210090CDE9010103460A466E49039017201DF081FC0020009001900290034602227C49039019201DF076FC00200222CDE972
:409F0000000202900346784903901A201DF06BFC002000900190029001230222734903901B201DF060FC0020009001900290012302226F4903901C201DF055FC00200222F0
:409F4000CDE90002029003466A4903901E201DF04AFC00200222CDE90002029003460246654903901F201DF03EFC00200222CDE900020290034602466049039020201DF0E9
:409F800032FC0020009001900290034603225C49039021201DF027FC0020009001900290034603225749039022201DF01CFC002000900190029003460322534903902320FB
:409FC0001DF011FC0020009001900290034603224E49039024201DF006FC0020009001900290034603224A49039025201DF0FBFB0020009001900290034603224549039078
:40A0000026201DF0F0FB0020009001900290034601224149039027201DF0E5FB0020009001900290034601223C49039028201DF0DAFB002000900190029003460122384911
:40A04000039029201DF0CFFB002000900190029003460222334903902B201DF0C4FB0020009001900290034602222F4903902C201DF0B9FB002059E094070020950700209F
:40A0800044070020450700204307002081070020780700202A0700206D070020270700202607002054070020530700205507002052070020370700209707002098070020D3
:40A0C00057070020580700206B0700206A070020690700208B070020210700205D070020130700201407002019070020990700209A070020180700201D070020240700202E
:40A100000D0700200F07002060070020610700206207002063070020650700206407002066070020670700206807002000900190029003460122FE4903902D201DF053FB31
:40A14000002000900190029003460122F94903902E201DF048FB002000900190029003460122F54903902F201DF03DFB002000900190029003460122F049039031201DF020
:40A1800032FB002000900190029003460122EC49039032201DF027FB00200121CDE9000103460A46CDE90210E64936201DF01BFB002000900190029003460122E2490390EB
:40A1C0003B201DF010FB002000900190029003460122DE4903903C201DF005FB00200122CDE9000202900346D94903903D201DF0FAFA00200122CDE9000202900346D549AD
:40A2000003903E201DF0EFFA002001210090CDE9010103460A46D049039041201DF0E3FA002000900190029003460122CB49039042201DF0D8FA00200090019002900346DA
:40A240000122C749039043201DF0CDFA002000900190029003460122C249039044201DF0C2FA002001210090CDE9010103460A46BD49039048201DF0B6FA00200121009024
:40A28000CDE9010103460A46B84903904B201DF0AAFA002001210090CDE9010103460A46B34903904D201DF09EFA002000900190029003460322AF4903904F201DF093FA04
:40A2C000012000220092CDE9012013460246AA49039050201DF087FA002001210090CDE9010103460A46A549039051201DF07BFA002000900190029003460122A04903903B
:40A3000052201DF070FA0020009001900290034603229C49039054201DF065FA0020009001900290034603229749039055201DF05AFA0020009001900290034603229349F4
:40A34000039056201DF04FFA0020009001900290034603228E49039057201DF044FA0020009001900290034603228A49039058201DF039FA00200090019002900346032271
:40A380008549039059201DF02EFA002000900190029003460322814903905A201DF023FA0020009001900290034603227C4903905B201DF018FA002001210090CDE901018F
:40A3C00003460A46774903905C201DF00CFA002000900190029003460122734903905D201DF001FA0020009001900290034601226E4903905E201DF0F6F90020009001908B
:40A400000290034601226A4903905F201DF0EBF900200222CDE900020290034601226549039061201DF0DFF900200222CDE900020290034601226049039062201DF0D3F936
:40A440000020009001900290034601225B49039064201DF0C8F90020009001900290034601225749039065201DF0BDF9002001210090CDE9010103460A4652490390672082
:40A480001DF0B1F9002001210090CDE9010103460A464D49039069201DF0A5F900200222CDE90002029003460246484903906A201DF099F901200021009101910B460246FB
:40A4C000CDE9021042496B201DF08DF900200222CDE90002029003463E4903906D201DF082F900200222CDE90002029003463A4903906E201DF077F900200222CDE90002F1
:40A5000002900346354903906F201DF06CF9002001210090CDE9010103460A463049039073201DF060F9002002225BE053E10000590700205B0700205A0700206C0700203D
:40A540006D0700206E07002070070020710700207207002073070020740700203E07002075070020760700209B0700209C0700208A07002056070020770700207807002027
:40A5800079070020A0070020A1070020A2070020A40700207E0700207F070020800700201B070020810700208307002084070020820700205F0700205E0700208507002047
:40A5C0008607002087070020890700204B070020380700209D0700209E0700209F0700208C070020CDE90002029003460246FE49039079201DF0F7F8002000900190029060
:40A6000003460222F94903907A201DF0ECF8002000900190029003460122F54903907B201DF0E1F8002000900190029003460122F04903907C201DF0D6F8002000900190F9
:40A64000029003460122EC4903907D201DF0CBF8002001210090CDE9010103460A46E74903907E201DF0BFF8002000900190029003460122E24903907F201DF0B4F80020EA
:40A6800001210090CDE9010103460222DD49039082201DF0A8F8002001210090CDE9010103460222D849039083201DF09CF8002001210090CDE9010103460222D349039026
:40A6C00084201DF090F801200021009101910B460222CDE90210CE4986201DF084F801200021009101910B460222CDE90210C94987201DF078F801200021009101910B46AB
:40A700000246CDE90210C44988201DF06CF8002000900190029003460322C04903908E201DF061F8002000900190029003460322BB4903908F201DF056F8002000900190CF
:40A74000029003460322B74903908F201DF04BF8012009F028F80021B34800781CF06CFF0021B24800781CF067FF0021B04800781CF062FF0021AF4800781CF05DFF0120E6
:40A780000021009101910B460222CDE90210AA4986201DF028F801200021009101910B460222CDE90210A54987201DF01CF80121A34800781DF0C5FB0121A24800781DF017
:40A7C000C0FB0121A04800781DF0BBFB01219F4800781DF0B6FB1FBD1FB50020009001900290034603229A49039001201CF0FBFF00200090019002900346032295490390DA
:40A8000002201CF0F0FF0020009001900290034603229149039010461CF0E5FF0020009001900290034603228C49039004201CF0DAFF002000900190029003460422884942
:40A84000039005201CF0CFFF0020009001900290034603228349039006201CF0C4FF0020009001900290034603227F49039007201CF0B9FF002000900190029003460322E9
:40A880007A49039008201CF0AEFF0020009001900290034602225549039009201CF0A3FF0020009001900290034602227049039017201CF098FF0020009001900290034697
:40A8C00002466C49039019201CF08DFF0020009001900290034603226749039021201CF082FF0020009001900290034603226349039022201CF077FF00200090019002908E
:40A90000034602224D49039027201CF06CFF0020009001900290034602224749039028201CF061FF0020009001900290034602465349039029201CF056FF0120002100919C
:40A9400001910B460A46CDE902104E492A201CF04AFF0020009001900290034602464A4903902B201CF03FFF002000900190029003460122454903902D201CF034FF00207B
:40A9800000900190029003460246414903902E201CF029FF0020009001900290034602463C4903902F201CF01EFF0020009001900290034602463849039030201CF013FFDA
:40A9C0000020009001900290034602463349039046201CF008FF0020009001900290034602462F4903905DE08E0700208F0700203107002032070020900700209107002034
:40AA00008D0700203B0700203C0700203D07002093070020940700209507002044070020450700204307002081070020780700202A0700206D070020270700202607002000
:40AA400054070020530700205507002052070020600700200D0700200E0700200F070020100700206307002011070020120700203F070020170700201A0700201B0700206D
:40AA800028070020210700201E07002048070020490700204A0700204B0700201C0700204D07002047201CF09EFE002000900190029003460246F649039048201CF093FEF7
:40AAC000002000900190029003460122F149039057201CF088FE002000900190029003460222ED49039059201CF07DFE002000900190029003460222E84903905A201CF0AE
:40AB000072FE002000900190029003460122E44903905B201CF067FE002000900190029003460122DF4903905C201CF05CFE002000900190029003460122DB4903905D206B
:40AB40001CF051FE002000900190029003460122D64903905E201CF046FE002000900190029003460122D24903905F201CF03BFE002000900190029003460122CD49039022
:40AB800060201CF030FE002000900190029003460122C949039061201CF025FE002000900190029003460122C449039064201CF01AFE002000900190029003460122C04978
:40ABC000039065201CF00FFE002000900190029003460122BB49039066201CF004FE002000900190029003460122B749039067201CF0F9FD00200090019002900346012220
:40AC0000B249039068201CF0EEFD002000900190029003460122AE49039069201CF0E3FD002000900190029001231A46A94903906A201CF0D8FD0020009001900290034666
:40AC40000122A54903906C201CF0CDFD002000900190029003460122A04903906D201CF0C2FD0020009001900290034601229C4903906E201CF0B7FD012000210091019151
:40AC80000B460A46CDE9021096497C201CF0ABFD01200021009101910B460A46CDE9021091497D201CF09FFD002001210090CDE9010103460A468D49039081201CF093FD46
:40ACC0000020009001900290034602228849039082201CF088FD0020009001900290034602228449039083201CF07DFD0020009001900290034602227F49039084201CF069
:40AD000072FD0020009001900290034602227B49039086201CF067FD0020009001900290034602227649039087201CF05CFD002000900190029003460246724903908820FF
:40AD40001CF051FD0020009001900290034603226D4903908D201CF046FD002000900190029003460322694903908E201CF03BFD00200090019002900346032264490390FA
:40AD80008F201CF030FD0121584800781CF054FC0121604800781CF04FFC01215E4800781CF04AFC1FBD1FB500240CE000205B4901EB041189680870584901EB0411C96829
:40ADC0000870601CC4B2902CF0DB1CF087FB1DF025FA20F0B9FD0121022023F02EF90020009001900290034601224D49039016201CF0F9FC002001210090CDE901010346F2
:40AE00000A46484903901E201CF0EDFC002000900190029003460122434903906B201CF0E2FC1CF006FCFF2831D00121084623F004F90121042023F000F90121082023F033
:40AE4000FCF80121102023F0F8F80121202023F0F4F80121402023F0F0F80121802023F0ECF80121080223F0E8F81CF0E2FB0A2862D2DFE800F06105060708095B5C5D5ED7
:40AE800000BF00BF00BF00BFFFF7A6FC55E055E01D07002051070020290700202A0700202B0700202C0700202D0700204E0700204F070020500700202E07002071070020EF
:40AEC00072070020310700203207002033070020340700203507002038070020390700203A07002024070020230700203E0700203B0700203C0700203D0700205407002039
:40AF000053070020400700204307002044070020450700204107002042070020F87C040813070020180700203707002000BF00BF00BFFEF7CBF900E000BF00BF1FBD10B5D2
:40AF40000120FE4908701EF00FFFFC494860012022F024FF1CE0612022F0C2FE78B145F25550F74908600120486040F6B83088604CF6CC4008600220F049087008E0EF491E
:40AF800048681EF019FF642802D90320EB490870EA4800780128DED010BD10B50020E74908704FF4FA701EF0B3FEFA201EF0F6FEFFF7C5FFFFF7F7FE1CF0FCFAC8B1E148D9
:40AFC00000781CF03BFF40B90121DF4800781CF033FB0020DD4908700BE0DD4800781CF02DFF18B10220D949087002E00120D74908701BF051FDEDF765F900221146D548D0
:40B00000DFF854C300DF002010BD10B572B66FF0040000F059FA6FF0010000F055FA4FF0FF3000F051FA042000F04EFA052000F04BFA062000F048FA072000F045FA0820EF
:40B0400000F042FA092000F03FFA0A2000F03CFA0B2000F039FA0C2000F036FA0D2000F033FA0E2000F030FA0F2000F02DFA102000F02AFA112000F027FA122000F024FACA
:40B08000132000F021FA142000F01EFA152000F01BFA162000F018FA172000F015FA182000F012FA192000F00FFA1A2000F00CFA1B2000F009FA1C2000F006FA1D2000F051
:40B0C00003FA1E2000F000FA1F2000F0FDF9202000F0FAF9212000F0F7F9222000F0F4F9232000F0F1F9242000F0EEF9252000F0EBF9262000F0E8F9272000F0E5F92820DE
:40B1000000F0E2F9292000F0DFF92A2000F0DCF92B2000F0D9F92C2000F0D6F92D2000F0D3F92E2000F0D0F92F2000F0CDF9302000F0CAF9312000F0C7F9322000F0C4F9F4
:40B14000332000F0C1F9342000F0BEF9352000F0BBF9362000F0B8F9372000F0B5F9382000F0B2F9392000F0AFF93A2000F0ACF93B2000F0A9F93C2000F0A6F93D2000F0FA
:40B18000A3F93E2000F0A0F93F2000F09DF9402000F09AF9412000F097F9422000F094F9432000F091F9442000F08EF9452000F08BF9462000F088F9472000F085F94820DF
:40B1C00000F082F9492000F07FF94A2000F07CF94B2000F079F94C2000F076F94D2000F073F94E2000F070F94F2000F06DF9502000F06AF9512000F067F96FF0040000F080
:40B200006CF96FF0010000F068F94FF0FF3000F064F9042000F061F9052000F05EF9062000F05BF9072000F058F9082000F055F9092000F052F90A2000F04FF90B2000F04A
:40B240004CF90C2000F049F90D2000F046F90E2000F043F90F2000F040F9102000F03DF9112000F03AF9122000F037F9132000F034F9142000F031F9152000F02EF9162001
:40B2800000F02BF9172000F028F9182000F025F9192000F022F91A2000F01FF91B2000F01CF91C2000F019F91D2000F016F91E2000F013F91F2000F010F9202000F00DF904
:40B2C000212000F00AF9222000F007F9232000F004F9242000F001F9252000F0FEF8262000F0FBF8272000F0F8F8282000F0F5F8292000F0F2F82A2000F0EFF82B2000F06B
:40B30000ECF82C2000F0E9F82D2000F0E6F82E2000F0E3F82F2000F0E0F8302000F0DDF8312000F0DAF8322000F0D7F8332000F0D4F8342000F0D1F835200FE0E403002021
:40B34000003000401E0700203A070020E00300204B0700207B4C0208F52F040800F0BDF8362000F0BAF8372000F0B7F8382000F0B4F8392000F0B1F83A2000F0AEF83B207D
:40B3800000F0ABF83C2000F0A8F83D2000F0A5F83E2000F0A2F83F2000F09FF8402000F09CF8412000F099F8422000F096F8432000F093F8442000F090F8452000F08DF81C
:40B3C000462000F08AF8472000F087F8482000F084F8492000F081F84A2000F07EF84B2000F07BF84C2000F078F84D2000F075F84E2000F072F84F2000F06FF8502000F0D7
:40B400006CF8512000F069F862B610BD38B5044660680090009D206880F3088800BFA84738BD00BFBFF34F8F3048006800F4E0602F490843001D2D490860BFF34F8F00BF37
:40B4400000BFFEE710B500212A4800781CF0F4F80021294800781CF0EFF80021274800781CF0EAF801DF10BD01B500BF04226946234800688C3000F04BF818B921480099E1
:40B48000C0F87C1400BF08BD01B500BF042269461B480068903000F03BF818B919480099C0F8801400BF08BD01B500BF0422694613480068943000F02BF818B91148009986
:40B4C000C0F8841400BF08BD00F01F02012191400D4A430942F82310704700F01F02012191400A4A430942F8231070470CED00E00000FA0572070020700700207107002045
:40B50000F40300202021002080E100E080E200E070B504460D461646324629462046EDF77AFC70BD2DE9F34F82B0844600BF00210A460B460E460F46002001908046009099
:40B5400064E09CF80000A0F13004E5179CF800002E2838D1B8F1000F0CD1FA494FF00009A2FB010A03FB01A102FB0919861949EB07071FE0B8F1010F0CD1F3494FF00009BE
:40B58000A2FB010A03FB01A102FB0919861949EB07070FE0B8F1020F0CD14FF47A714FF00009A2FB010A03FB01A102FB0919861949EB070708F1010000F0FF08002000905E
:40B5C000002213461CE09CF80000C8B1009810B922462B4610E0009801280DDB4FF00A0A4FF0000B1146A1FB0A1E03FB0AE902FB0B900A1940EB05030098401CC0B2009067
:40B600000CF1010C0198401CC0B2019003990198884296DBB6185F413046394604B0BDE8F08F2DE9F04F83468946924600BF00BF51465846FFF776FF05460E4651464846B6
:40B64000FFF770FF07468846781B78EB060001DA012407E0E81B76EB080002DA4FF0FF3400E000242046BDE8F08F70B586B00546B6A2B9A102A823F089FE1022294602A838
:40B68000FFF7CFFF00283EDD0026002001900090012435E0062C0CD2DFE804F00B0C09070503AE4E08E0AE4E06E0AE4E04E0AE4E02E000BFAD4E00BF00BF912001902120A9
:40B6C0000090AB4890F830000A2817D1042201A906F13000FFF71CFF0422694606F12C00FFF716FFA24890F82404A04206D19DF804009F4908639DF80000C862601CC4B2FA
:40B70000052CC7DD00BF06B070BD70B586B0054698A291A102A823F039FE1022294602A8FFF77FFF00282DDD002600200190012425E0062C0CD2DFE804F00B0C09070503A0
:40B74000864E08E0864E06E0864E04E0864E02E000BF864E00BF00BFFF200190012201A906F2FF10FFF7D4FE814890F82404A04203D19DF80400F0F7A0FA601CC4B2052C1C
:40B78000D7DD00BF06B070BD70B586B005467CA271A102A823F0FAFD1022294602A8FFF740FF00283FDD0026002001909FED770A8DED000A012433E0062C0CD2DFE804F07A
:40B7C0000B0C09070503654E08E0654E06E0654E04E0654E02E000BF644E00BF00BF002001909FED6A0A8DED000A012201A906F14300FFF78DFE0422694606F5DC70FFF7FC
:40B8000087FE5B4890F82404A04207D19DF80400F8F794FB9DED000AF8F7A1FB601CC4B2052CC9DD00BF06B070BD70B586B0054657A249A102A823F0A9FD1022294602A89E
:40B84000FFF7EFFE00282DDD002664200190012425E0062C0CD2DFE804F00B0C090705033E4E08E03E4E06E03E4E04E03E4E02E000BF3E4E00BF00BF64200190012201A9E5
:40B8800006F56970FFF744FE394890F82404A04203D19DF8040005F035FA601CC4B2052CD7DD00BF06B070BDF0B585B005463BA229A101A823F06AFD1022294601A8FFF730
:40B8C000B0FE00283CDD2A4890F82464012434E0062C0CD2DFE804F00B0C090705031F4F08E01F4F06E01F4F04E01F4F02E000BF1E4F00BF00BF40F6C41000900222694641
:40B9000007F56070FFF704FEB44204D1BDF800001749A1F880034FF47A5000900222694607F28230FFF7F4FDB44204D1BDF800000F49A1F88203601CC4B2052CC8DD00BFC8
:40B9400005B0F0BD00CA9A3B40420F0032312E322E302E313000000025730000581B00687017006888130068A00F0068B80B00682021002032312E322E302E3600000000F8
:40B9800032312E322E302E350000000035FA8E3C32312E312E302E3900000000322E342E302E3533000000002DE9F04105460E4617463A4631462846EDF7A4FA044604B1D2
:40B9C00003DF2046BDE8F081F0B585B00546F7A2AFF27C0101A823F0D9FC1022294601A8FFF71FFE00282FDDF34890F82474012427E0062C0CD2DFE804F00B0C090705036A
:40BA0000EE4E08E0EE4E06E0EE4E04E0EE4E02E000BFEE4E00BF00BF042206F5C6716846FFF7C2FF0422694606F56270FFF770FDBC4204D19DED000ADF4880EDE20A601CE4
:40BA4000C4B2052CD5DD00BF05B0F0BDF0B585B00546DFA2AFF2001101A823F097FC1022294601A8FFF7DDFD00282BDDD24890F82464012423E0062C0CD2DFE804F00B0C27
:40BA800009070503CD4F08E0CD4F06E0CD4F04E0CD4F02E000BFCD4F00BF00BF002000900122694607F19700FFF732FDB44204D19DF80000C04981F89700601CC4B2052C3F
:40BAC000D9DD00BF05B0F0BD2DE9F04186B00546C2A2AFF27C1102A823F058FC1022294602A8FFF79EFD002836DD002001900026B14890F8247400242BE0062C13D2DFE8F0
:40BB000004F0130F0C090603DFF8B0820FE0DFF8B0820CE0DFF8AC8209E0DFF8AC8206E0DFF8A88203E000BFDFF8BC8200BF00BF042201A908F1B400FFF7EAFCBC4206D1A7
:40BB40009D490198C1F8B4000846C0F89860601CC4B2052CD1DD00BF06B0BDE8F081F0B587B00646A1A2AFF2102103A823F00EFC1022314603A8FFF754FD002857DD8E48AD
:40BB800090F8247400244FE0062C0ED2DFE804F00E0B09070503894D0AE0894D08E0894D06E0894D04E0894D02E000BF8E4D00BF00BF042205F1300101A8FFF7F5FE13203E
:40BBC0008DF809000198FDF7C3F918B90198FDF7E9F918B190208DF808000AE00198FDF7D9F918B113208DF8080002E0FF208DF8080001220DF1090105F1B300FFF788FC7A
:40BC0000012202A905F1B200FFF782FCBC4209D19DF80910684880F8B3109DF80800664981F8B200601CC4B2052CADDD00BF07B0F0BDF0B585B005466FA2AFF2E42101A8DD
:40BC400023F0A4FB1022294601A8FFF7EAFC00282DDD594890F8246401200090002423E0062C0ED2DFE804F00E0B09070503534F0AE0534F08E0534F06E0534F04E0534F6D
:40BC800002E000BF584F00BF00BF0122694607F14B00FFF73DFCB44204D19DF80000464981F84B00601CC4B2052CD9DD00BF05B0F0BDF0B587B0054651A2AFF2643103A8D2
:40BCC00023F064FB1022294603A8FFF7AAFC002839DD394890F82474002431E0062C0ED2DFE804F00E0B09070503344E0AE0344E08E0344E06E0344E04E0344E02E000BF11
:40BD0000394E00BF00BF012206F1280102A8FFF74BFE9DF80800042810D0B2EE040A8DED010A042201A906F5FC70FFF7F1FBBC4204D19DED010A204880ED7E0A601CC4B226
:40BD4000052CCBDD00BF07B0F0BDF0B585B006462DA2AFF2FC3101A823F018FB1022314601A8FFF75EFC00287EDD072729A2AFF2184101A823F00AFB1022314601A8FFF714
:40BD800050FC002800DD092700200090002468E0062C49D2DFE804F0494644070503074D45E0074D43E0074D41E00000322E342E302E34340000000020210020581B0068D3
:40BDC0007017006888130068A00F0068B80B0068322E332E302E333000000000322E322E302E343600000000D0070068322E322E302E313800000000322E322E302E3200EF
:40BE0000322E322E302E3100322E312E302E373300000000322E312E302E353400000000F64D04E0F64D02E000BFF64D00BF00BF042205F130016846FFF7B6FD0098384422
:40BE40000090009814280BD30422694605F13000FFF75EFBEB48854202D1EB4900980863641C062C94D300E000E000BF05B0F0BD2DE9F3410D46E449ADEB01040846071963
:40BE8000DF482618AAB239463046FFF741FBDE480719DA482618AAB239463046FFF738FBD9480719D9482618AAB239463046FFF72FFBD5480719D6482618AAB2394630467F
:40BEC000FFF726FBD0480719D2482618AAB239463046FFF71DFBBDE8FC812DE9FE4F81468A46174698460020009000262D2200233846414623F0BFF905462D220023384692
:40BF0000414623F0B8F9934615B9BBF1000F35D0D5B1002416E0C4EB041000EB400048440290C4EB041000EB4000504401902D22DDE90110FFF7ECFA0646009931430091A4
:40BF4000601CC4B2AC42E6D3BBF1000F18D0C5EB051000EB400048440290C5EB051000EB4000504401901FFA8BF2DDE90110FFF7CFFA064600993143009101E0402000907B
:40BF80000098BDE8FE8F01B500BF01226946A24800682D30FFF7BCFA20B99DF800109A4880F81D1400BF08BD2DE9FE4F81468A46174698460020009000262D22002338468D
:40BFC000414623F058F905462D2200233846414623F051F9934615B9BBF1000F35D0D5B1002416E0C4EB041000EB400048440290C4EB041000EB4000504401902D22DDE9FC
:40C000000110FFF7D1FC0646009931430091601CC4B2AC42E6D3BBF1000F18D0C5EB051000EB400048440290C5EB051000EB4000504401901FFA8BF2DDE90110FFF7B4FCD0
:40C04000064600993143009101E0402000900098BDE8FE8F3EB5002002900A200190002000904FF47C71684823F0F5FAB0216B4823F0F1FA4FF458716848B03023F0EBFA33
:40C08000012201A9644800689830FFF741FA012261480168983102A8FFF786FC9DF80800401CC0B20190012201A95B4800689830FFF72EFA012258480168983102A8FFF737
:40C0C00073FC9DF808009DF80410884207D05448007840F080005249087001248CE001224D4801682E316846FFF75EFC9DF8000044284CD0FF224FF47C71434823F0A3FA5B
:40C100004FF47C72002340493E48FFF7E6FE4FF47C7200233C493A48FFF7DFFE4FF47C72002339493548FFF7D8FE4FF47C72002335493648FFF7D1FE4FF47C720023324991
:40C140003348FFF7CAFE4FF47C7200232E493148FFF7C3FE4FF47C712B4823F07CFAB02200232E494FF0D040FFF7B7FE4FF4587200232A49B0312B48FFF7AFFE442000906B
:40C1800001226946244800682E30FFF7C1F9B02200234FF0D0412148FFF706FF4FF45872002320491D48B030FFF7FEFE01221A4801682D3119482D30FFF7F6FB124890F87F
:40C1C0001D04672810D001246720FFF7DCFE4FF47C710D4823F03FFA4FF47C7200230A490848FFF77AFE07E002244FF47C72002304490548FFF7D8FE20463EBDA00F0068BE
:40C20000B80B0068D0070068202100208813006870170068581B0068F403002010250020ED030020F401006810B5FA48ECF7A2FD0446204610BD70B58CB00024002008904A
:40C2400009900A900B9004900590069007900090019002900390F0490870F049087001200870FFF7E1FFFFF7F5FEED490870ED4AAFF61C1108A823F089F804A81BF0C6FF23
:40C28000E9A104A823F00EFA08B1012000E00020054645B1E6A01BF0A5FFE3A01BF0A2FFE7A01BF085FF04A81BF094FF102204A908A8FFF7B6F90446D9480078012806D137
:40C2C0000020D649087008A81BF072FFCFE0002CFCD0002006F0B0F8002006F000F908A81BF066FF002C39DA0020FFF74CFEFF224FF47C71D44823F0A6F94FF47C720023B5
:40C30000D149D248FFF7E9FD4FF47C720023CE49CF48FFF7E2FD4FF47C720023CA49CD48FFF7DBFD4FF47C720023C749CA48FFF7D4FD4FF47C720023C349C848FFF7CDFDDF
:40C340004FF47C720023C049C548FFF7C6FD4FF47C71BD4823F07FF903DF88E0C1A2AFF60821684623F012F8102204A96846FFF758F9002838DD0020FFF705FEFF224FF406
:40C380007C71B14823F05FF94FF47C720023AE49AE48FFF7A2FD4FF47C720023AA49AC48FFF79BFD4FF47C720023A749A948FFF794FD4FF47C720023A349A748FFF78DFD22
:40C3C0004FF47C720023A049A448FFF786FD4FF47C7200239C49A248FFF77FFD4FF47C71994823F038F903DFA1A2AFF69421684622F0CCFF102204A96846FFF712F90028F1
:40C4000011DD012008F07DF901218F48B130FFF72FFD1BF0CFF830B10320EFF709FE01219648FFF725FD04A8FFF78FFC04A8FFF740FC04A8FFF7FDFB04A8FFF790FB04A82A
:40C44000FFF742FB04A8FFF701FB04A8FFF7BCFA04A8FFF729FA04A8FFF7E7F904A8FFF793F904A8FFF751F904A8FFF7FEF80020FCF74EFBFCF7EEFE0646FCF7EEFD674886
:40C4800000780CB070BD65480078704701B500BF012269467A4800683430FFF739F820B99DF80010684880F8241400BF7548C16B0220DFF8D4C100DF08BD2DE9FC470746E5
:40C4C000884615461E46714890F84200C006C10A6E4890F8410041EA00206C4991F8401040EA010908F01EF910B907F03BFC00B3FDB1F6B14D4504D1012E02D10120BDE8D2
:40C50000FC874D4503D1022E01D10220F7E74D4503D1032E01D10320F1E74D4503D1042E01D10420EBE74D4573D1052E71D10520E5E7002D6DD1464C042204F1340101A81A
:40C54000FFF732FA012204F1B1016846FFF72CFA0198874205D19DF80000404501D10120CDE73C4C042204F1340101A8FFF71CFA012204F1B1016846FFF716FA019887429F
:40C5800005D19DF80000404501D10220B7E7324C042204F1340101A8FFF706FA012204F1B1016846FFF700FA0198874205D19DF80000404501D10320A1E7284C042204F1C6
:40C5C000340101A8FFF7F0F9012204F1B1016846FFF7EAF90198874205D19DF80000404501D104208BE71E4C042204F1340101A8FFF7DAF9012204F1B1016846FFF7D4F90C
:40C600000198874244D19DF80000404540D1052075E73DE000380040ED030020EE030020EC0300209CBE0008322E302E310000003030303030303030303030300000000081
:40C64000322E302E302E310020210020D0070068B80B0068A00F00688813006870170068581B0068322E302E302E363500000000322E312E302E333900000000D322002099
:40C68000F403002068520020E127040848E10020002034E738B5F84C042204F5EC716846FFF782F940F2FD110098884201D0012038BDF24C042204F5EC716846FFF774F9D1
:40C6C00040F2FD110098884201D00220F0E7EC4C042204F5EC716846FFF766F940F2FD110098884201D00320E2E7E64C042204F5EC716846FFF758F940F2FD110098884273
:40C7000001D00420D4E7E04C042204F5EC716846FFF74AF940F2FD110098884201D00520C6E70020C4E710B54FF47C71D74822F092FF4FF47C720023D449D548FFF7CDFBA7
:40C7400010BD10B54FF47C71D04822F084FF4FF47C720023CD49CE48FFF7BFFB4FF47C720023CA49C448FFF7B8FB4FF47C720023C649C248FFF7B1FB4FF47C720023C3498F
:40C78000BF48FFF7AAFB4FF47C720023BF49BD48FFF7A3FB4FF47C720023BC49BA48FFF79CFB4FF47C71B94822F055FF10BD2DE9F0410446884615461F463CB9B4482E1840
:40C7C0003A4641463046FEF7A3FE30E0012C07D1A9482E183A4641463046FEF799FE26E0022C07D1A5482E183A4641463046FEF78FFE1CE0032C07D1A1482E183A4641465A
:40C800003046FEF785FE12E0042C07D19D482E183A4641463046FEF77BFE08E0052C06D199482E183A4641463046FEF771FEBDE8F0812DE9F04104460F46154698463CB9D8
:40C8400093482E18424631463846FFF7ADF830E0012C07D188482E18424631463846FFF7A3F826E0022C07D184482E18424631463846FFF799F81CE0032C07D180482E1813
:40C88000424631463846FFF78FF812E0042C07D17C482E18424631463846FFF785F808E0052C06D178482E18424631463846FFF77BF8BDE8F08110B5744890F82444062CF5
:40C8C0002CD2DFE804F02C030B131B234FF47C7200236E496848FFF700FB21E04FF47C7200236A496548FFF7F8FA19E04FF47C72002366496248FFF7F0FA11E04FF47C7203
:40C90000002362495F48FFF7E8FA09E04FF47C7200235E495C48FFF7E0FA01E000BF00BF00BF10BD2DE9F04105460E461746984643463A4631462846FFF7BFFD0446062C2A
:40C940005ED2DFE804F05E031527394B4FF47C72002349494D48FFF727FB4FF47C7200234A494B48FFF7B9FA0120FFF78FFD54E04FF47C72002341494448FFF715FB4FF46B
:40C980007C72002341494248FFF7A7FA0220FFF77DFD42E04FF47C72002339493B48FFF703FB4FF47C72002338493948FFF795FA0320FFF76BFD30E04FF47C720023314980
:40C9C0003248FFF7F1FA4FF47C7200232F493048FFF783FA0420FFF759FD1EE04FF47C72002329492948FFF7DFFA4FF47C72002326492748FFF771FA0520FFF747FD0CE0D3
:40CA000000BFFFF790FE0020FFF740FD002021494860272014F01EFC00BF00BF04B103DFBDE8F0814FF40050704710B5174890F82404062840D2DFE800F040030C152F37BF
:40CA40000D4C042211493C3104F13C00FEF760FD34E00A4C04220D493C3104F13C00FEF757FD2BE0064C042208493C3104F13C00FEF74EFD22E00000B80B0068A00F00682A
:40CA80008813006870170068581B006820210020D0070068583200200B4C04220B4904F13C00FEF735FD09E0094C0422074904F13C00FEF72DFD01E000BF00BF00BF10BD47
:40CAC0000448042170470000701700685C210020581B00683E9BEFE310B51DF045F9FE49086009F031FEFC4880ED010A10BD10B5FA4890F84A00022824D1F84890F8BD010E
:40CB000002281FD1F64890ED020ADFEDF60AB4EEE00AF1EE10FA0ADBFAF720FFC4B223467D22ED490C3101200DF0A2F82EE0FAF715FFC4B223467D22E7490C3100200DF01A
:40CB400097F823E0E648D0ED010AE448B0F8BE0100EE100AB8EE400AF4EEC00AF1EE10FA0ADBFAF7FBFEC4B22346FA22DA490C3101200DF07DF809E0FAF7F0FEC4B22346A9
:40CB8000FA22D5490C3100200DF072F810BD10B52DED048B1AF026FD002867D0FFF7A7FFEDF72AFD18B10020CB49087261E0CA48007A60B9C84890F82000002859D1012081
:40CBC000C54908721DF0D0F8C349086051E0C248007A01280CD1C049C86947F230511DF0C9F8A0B30220BC490872FFF775FF40E0B948007A02283CD109F0A6FDB648D0ED60
:40CC0000010A30EEC00A10EE104A204627F0CEFA41EC190BB0EE490AF0EE690A23F0A0FEB0EE408AF0EE608A9FEDAF0B53EC102B51EC180B27F0C2F80ED2A74890F8200088
:40CC4000012805D10020A44948720120087210E00120A14948720CE09F4908684FF4FA611DF088F828B1FFF737FF02E000209A494872BDEC048B10BD994981F890007047E4
:40CC8000974981F838007047F0EE400A9FED980A20EE800A704770B52DED0A8B82B004468E4890F8BD010F287ED2DFE800F07D365EFC37FBFAF97D7D087DF8F7F600EDF763
:40CCC00096FC10EE105A284627F070FA41EC1A0BB0EE4A0AF0EE6A0A23F042FEB0EE409AF0EE609A51EC190B26F024FCA0619FED810A84ED1C0A94ED060A84ED010AEDF7DB
:40CD0000C0FC18B10020FFF7BBFF02E00420FFF7B7FF0420FFF7B0FF6AE200BF764800781BF08CF820B19FED750A84ED060A03E09FED700A84ED060A714800781BF07EF8DA
:40CD400020B19FED6E0A84ED1C0A03E09FED690A84ED1C0A0420FFF793FF0420FFF78CFF94ED060A84ED010AEEE3634800781AF029FE00EE100AF8EE400A9FED621A9FED7F
:40CD8000620A10EE810A84ED0C0AE16821611CF0EBFFE060D4E90310091A6161D4ED0C0AB0EE600A0A2100E0BFE304F118000AF0C8FC94ED060ADFED550AB4EEE00AF1EEC3
:40CDC00010FA03D20020FFF75BFF0FE094ED060AF0EE040AB4EEE00AF1EE10FA03DD0120FFF74EFF02E00420FFF74AFF0420FFF743FF94ED0C0AB5EEC00AF1EE10FA02D25D
:40CE00009FED3C8A01E094ED068A94ED0F0A84ED100A84ED0F8A94ED050AB8EE400ADFED370A80EE201A11EE105A284627F0BEF941EC1A0B94ED0F0AD4ED100A30EE600A56
:40CE400010EE101A084627F0B1F941EC1C0BB0EE4C0AF0EE6C0A23F083FDB0EE40BAF0EE60BA53EC1A2B51EC1B0B26F051FC41EC190B26F05FFB60639FED1E0A84ED1C0AA3
:40CE8000B0EE480AFFF700FF84ED010AD4ED0D0AB0EE600AFFF7F8FE06E0D9E2A9E1E6E2FBE112E103E069E084ED020A4CE3124800781AF087FD00EE100AB8EE400ADFED87
:40CEC000110A20EE200ADFED120A80EE201A84ED0C1AD4ED0C0A1DE020290020202100204429002000C0DA44000000401857B63FC0A90646000000005207002000007A441F
:40CF0000560700203333533A9A99193FCDCCCCBE0CAC233FB0EE600A0A2104F118000AF010FC94ED060ADFEDFE0AB4EEE00AF1EE10FA03D20020FFF7A3FE0FE094ED060A8D
:40CF4000DFEDF80AB4EEE00AF1EE10FA03DD0120FFF796FE02E00420FFF792FE0420FFF78BFE1FED1C0A84ED1C0AD4ED060AB0EE600AFFF789FE84ED010AE5E2EA480078A8
:40CF80001AF020FD00EE100AF8EE400A1FED231A1FED230A10EE810A84ED0C0AD4ED0C0AB0EE600A0A2104F118000AF0CAFB94ED060A5FED2A0AB4EEE00AF1EE10FA03D24F
:40CFC0000020FFF75DFE0FE094ED060AF0EE040AB4EEE00AF1EE10FA03DD0120FFF750FE02E00420FFF74CFE94ED0C0AB5EEC00AF1EE10FA02D21FED418A01E094ED068ACA
:40D00000CA4800781AF0DEFC00EE100AF8EE400A1FED441A1FED440A10EE810A84ED220AD4ED220AB0EE600A0A2104F170000AF088FB94ED1C0A5FED4B0AB4EEE00AF1EEAB
:40D0400010FA03D20020FFF717FE0FE094ED1C0AF0EE040AB4EEE00AF1EE10FA03DD0120FFF70AFE02E00420FFF706FE94ED220AB5EEC00AF1EE10FA02D25FED628A01E0C0
:40D08000D4ED1C8AB0EE480AFFF7FEFDB0EE401AB0EE680AFFF7F8FD31EE400A10EE105A284627F083F841EC1A0BB0EE4A0AF0EE6A0A23F055FCB0EE409AF0EE609A51ECDD
:40D0C000190B26F037FA60603EE2974800781AF079FC00EE100AB8EE400A5FED760A20EE200A5FED750A80EE201A84ED0C1AD4ED0C0AB0EE600A0A2104F118000AF021FBDC
:40D1000094ED060ADFED860AB4EEE00AF1EE10FA03D20020FFF7B4FD0FE094ED060ADFED810AB4EEE00AF1EE10FA03DD0120FFF7A7FD02E00420FFF7A3FD7C4800781AF028
:40D1400041FC00EE100AB8EE400A5FED920A20EE200A5FED910A80EE201A84ED221AD4ED220AB0EE600A0A2104F170000AF0E9FA94ED1C0ADFED6A0AB4EEE00AF1EE10FA60
:40D1800003D20020FFF778FD0FE094ED1C0ADFED650AB4EEE00AF1EE10FA03DD0120FFF76BFD02E00420FFF767FD94ED060AD4ED1C0A30EE600A10EE101A084626F0F6FF89
:40D1C00041EC1B0BB0EE4B0AF0EE6B0A23F0C8FBB0EE40AAF0EE60AA51EC1A0B26F0AAF909EE100AB0EE490AFFF74EFD84ED010AAAE16421E0681CF0BDFDE8B31CF0B4FD00
:40D20000E06094ED0F0A84ED100A494800781EF072FD00EE100AB8EEC00A84ED0F0A94ED0F0AD4ED100A30EE600A10EE101A084626F0BCFF41EC1A0BB0EE4A0AF0EE6A0A27
:40D2400023F08EFBB0EE409AF0EE609A51EC190B26F070F92063D4ED0C0A9FED361A80EE810AF2EE040A80EE201A84ED0C1AD4ED0C0AB0EE600A00E00EE0032104F11800A8
:40D280000AF05FFA94ED060A84ED010A0420FFF7F7FC0420FFF7F0FC56E16421E0681CF069FD00287DD01CF05FFDE06094ED0F0A84ED100A1C4800781EF01DFD00EE100A37
:40D2C000B8EEC00A84ED0F0A94ED0F0AD4ED100A30EE600A10EE101A084626F067FF41EC1A0BB0EE4A0AF0EE6A0A23F039FBB0EE409AF0EE609A51EC190B26F01BF920630A
:40D3000094ED0C0ADFED0B0A80EE201A84ED0C1A94ED250A84ED260A074800780EE00000CDCCCC3C33339F40520700205507002054070020CDCCCC3D560700201EF0DBFCD6
:40D3400000EE100AB8EEC00A84ED250A94ED250AD4ED260A30EE600A10EE101A084626F025FF41EC1A0BB0EE4A0AF0EE6A0A23F0F7FAB0EE409AF0EE609A51EC190B26F05B
:40D38000D9F88821085194ED220A5FED160A80EE201A84ED221AD4ED0C0AB0EE600A032100E054E004F118000AF0CBF9D4ED220AB0EE600A032104F170000AF0C2F994ED96
:40D3C000060AD4ED1C0AB4EEE00AF1EE10FA04DD94ED060A84ED010A03E094ED1C0A84ED010AEDF74EF918B10020FFF749FC13E094ED1C0AD4ED060A30EE600AF3EE090A97
:40D40000B4EEE00AF1EE10FA03DD0220FFF738FC02E00420FFF734FCEDF740F918B10020FFF72AFC13E094ED060AD4ED1C0A30EE600AF3EE090AB4EEE00AF1EE10FA03DDC1
:40D440000220FFF719FC02E00420FFF715FC7BE09FEDFB0A84ED0C0A9FEDF90A84ED010A0420FFF70DFC0420FFF706FC6CE0FA21E0681CF07FFCE8B36A4601A9F1480078D9
:40D480001EF08CFD05461CF06FFCE06094ED0F0A84ED100A9DED000A84ED0F0A94ED0F0AD4ED100A30EE600A84ED0C0A94ED0C0AF5EE000A80EE201A11EE106A304626F0DB
:40D4C00075FE41EC1A0BB0EE4A0AF0EE6A0A23F047FAB0EE409AF0EE609A51EC190B26F029F82063D4ED0C0AB0EE600A022104F1180000E018E00AF024F994ED060A84ED64
:40D50000010A012D06D19DED010AB5EEC00AF1EE10FA03D10020FFF7B3FB02E00420FFF7AFFB0420FFF7A8FB0EE09FEDC50A84ED0C0A9FEDC30A84ED010A0020FFF7A0FB9F
:40D540000020FFF799FB00BF00BF02B0BDEC0A8B70BD10B51AF059F8D0B1FAF7FFF9C4B22346FA22B84900200CF082FB9FEDB40AB64880ED060A9FEDB20A80ED060A042198
:40D5800080F8381080F890100020B14948722EE0AE48FFF780FBAF48B0F8BE0118B90220A949087521E0A948D0ED010AA948B0F8BE0100EE100AB8EE400AF4EEC00AF1EEF5
:40D5C00010FA09DBFAF7CAF9C4B22346FA229E4901200CF04DFB08E0FAF7C0F9C4B22346FA22994900200CF043FBFFF7D0FA10BD97494872704731B50024BDF80000C828EC
:40D6000003DDC8200090022406E0BDF80000012802DA01200090032400BF022269468E48006800F5DF70FDF773FF20B9BDF800008849A1F8BE0100BF204638BD31B500249F
:40D64000BDF80000642803DD64200090022406E0BDF80000012802DA01200090032400BF022269467C48006800F5DF70FDF750FF20B9BDF800007749A1F8BE0100BF2046C7
:40D6800038BD31B50024BDF80000B0F5FA7F04DD4FF4FA700090022406E0BDF80000012802DA01200090032400BF022269466A48006800F5DF70FDF72BFF20B9BDF8000040
:40D6C0006449A1F8BE0100BF204638BD31B50024BDF80000322803DD32200090022406E0BDF80000012802DA01200090032400BF022269465848006800F5DF70FDF708FFB9
:40D7000020B9BDF800005349A1F8BE0100BF204638BD31B50024BDF80000C82803DDC8200090022406E0BDF80000012802DA01200090032400BF022269464748006800F52A
:40D74000DF70FDF7E5FE20B9BDF800004149A1F8BE0100BF204638BD31B50024BDF8000040F26351884203DD08460090022406E0BDF80000012802DA01200090032400BF6F
:40D78000022269463448006800F5DF70FDF7C0FE20B9BDF800002F49A1F8BE0100BF204638BD31B50024BDF8000045F2CC01884203DD08460090022406E0BDF8000001280F
:40D7C00002DA01200090032400BF022269462248006800F5DF70FDF79BFE20B9BDF800001C49A1F8BE0100BF204638BD10B52DED028BB0EE408A0024164890F8BD010E2809
:40D8000053D2DFE800F0072B08122C091336522D4052493700BF00BFBCEEC80A10EE101A88B2FFF7BEFF044648E000BFBCEEC80A10EE101A88B2FFF78FFF04463EE00000A7
:40D840000000000052070020002A0020442900202029002020210020F003002000BF00BFBCEEC80A10EE101A88B2FFF752FF044624E000BFBCEEC80A10EE101A88B2FFF7F7
:40D8800025FF04461AE0BCEEC80A10EE101A88B2FFF7F7FE044611E0BCEEC80A10EE101A88B2FFF7CBFE044608E0BCEEC80A10EE101A88B2FFF79FFE044600BF00BF412093
:40D8C000EFF74EFE0020FFF793FE2046BDEC028B10BD10B52DED020B00BF04226946FC48006800F5E670FDF713FE20B99DED000AF84880ED730A00BFF748016D0120DFF86F
:40D90000DCC300DF1CBD10B52DED020B00BF04226946EF48006800F5E470FDF7F9FD20B99DED000AEB4880ED720A00BFEA48016D0120DFF8A8C300DF1CBD10B52DED020B4F
:40D9400000BF04226946E248006800F5E270FDF7DFFD20B99DED000ADE4880ED710A00BFDD48016D0120DFF874C300DF1CBD10B52DED020B00BF04226946D548006800F5BC
:40D98000E070FDF7C5FD20B99DED000AD14880ED700A00BFD048016D0120DFF840C300DF1CBD10B5CB4890F8300091280ED0C94890F83000922809D0C64890F8300071281A
:40D9C00004D0C44890F83000B82818D1C14890F8BD010A2813D19FEDC20AFFF707FF9FEDC10AFFF7C4FF9FEDC00AFFF7A6FF9FEDBF0AFFF788FF9FEDBE0AFFF76AFFB5488A
:40DA000090F83000702804D0B24890F83000932819D1B04890F8BD010A2814D19FEDB50AFFF7E4FE9FEDB40AFFF7A1FF9FEDB30AFFF783FF9FEDB20AFFF765FF9FEDB10A69
:40DA4000FFF747FF18E0A34890F8BD010A2813D19FEDA80AFFF7CAFE9FEDA20AFFF787FF9FEDA10AFFF769FF9FEDA70AFFF74BFFBBEE040AFFF72DFF964890F8BD01012843
:40DA800004D1B7EE000AFFF7B1FE53E0914890F8BD01022804D19FED9D0AFFF7A7FE49E08C4890F8BD01032804D1B3EE040AFFF79DFE3FE0874890F8BD01042804D11FED5A
:40DAC000A00AFFF793FE35E0824890F8BD01052804D19FED8F0AFFF789FE2BE07D4890F8BD01062804D19FED8B0AFFF77FFE21E0784890F8BD01072804D0764890F8BD0171
:40DB00000D2804D1B1EE040AFFF770FE12E0714890F8BD01092804D19FED7E0AFFF766FE08E06C4890F8BD010C2803D1B2EE040AFFF75CFE10BD10B5664890F8BD010A28C5
:40DB40001CD1644890F8300091280ED0614890F83000922809D05F4890F83000712804D05C4890F83000B82803D1FA20FFF789FD03E04FF49670FFF784FD00E000BF00BF56
:40DB800010BD00B589B019F02DFD002879D0514890F8BD010E2875D2DFE800F074072A2B4E7576C274FDFCFBFAF9002000900190029003460246584903900846007819F066
:40DBC00012FE002000900190029003460246534903900846007819F006FE01214E4800781AF0AFF901214D4800781AF0AAF999E100BF0020009001900290034603224649E8
:40DC000003900846007819F0EEFD002000900190029003460322414903900846007819F0E2FD03213C4800781AF08BF903213B4800781AF086F975E101200021009101917A
:40DC40000B460A46CDE9021033490846007819F0CAFD01200021009101910B460A46CDE902102E490846007819F0BDFD01212A4800781AF066F90121284800781AF061F978
:40DC800050E150E129E100BF002000900190029003460322204903900846007819F0A3FD0020009001900290034603221B4903900846007819F097FD0021174800781AF0F0
:40DCC00040F90021154800781AF03BF92AE10000F00300202021002068520020E127040800007A43C6DCB53DB8AF833E52B8444114AE4740000096436744293EE5F25F3E9A
:40DD000052B862416666E6C133331B41000016430080BB440000C8425207002055070020002000900190029003460222F84903900846007819F057FD002000900190029020
:40DD400003460322F34903900846007819F04BFD002000900190029003460222EE4903900846007819F03FFD0221E94800781AF0E8F80221E84800781AF0E3F80020009024
:40DD80000190034614220121029004A804E092E072E01EE0A3E0A1E01DF0CCFD04A8DFEDDF0A9FEDDF0A02230022DE490090D84800781DF0A7FC04A8DFEDD80A9FEDD80A8F
:40DDC00002230322D8490090D34800781DF09AFCA8E0002000900190029003460222CC4903900846007819F0FEFC002000900190029003460322C74903900846007819F006
:40DE0000F2FC002000900190029003460222C24903900846007819F0E6FC0621BC4800781AF08FF80621BC4800781AF08AF8002000900190034614220121029004A81DF0D5
:40DE400079FD04A8DFEDB50A9FEDB50A02230022B4490090AE4800781DF054FC04A8DFEDAF0A9FEDAF0A02230322AF490090AA4800781DF047FC55E0002000900190029001
:40DE800003460222A24903900846007819F0ABFC01219F4800781AF054F8A448DFED9F0A9FEDA30A052300229E490090984800781DF028FC36E00020009001900290034614
:40DEC0000322944903900846007819F08CFC0021904800781AF035F824E000BF00BF002000900190029003460322894903900846007819F078FC0020009001900290034607
:40DF00000322844903900846007819F06CFC01217F4800781AF015F801217E4800781AF010F800BF00BF834890F8BD01824908700020FFF75DFB00208049087209B000BD22
:40DF40007F49097D012900D100E00021084670477B48407D70477A48007D08B9012070470020FCE7774909880143764A11807047F7EE000AB0EE600A7C2202706D4A92F85B
:40DF8000BD210E2A22D2DFE802F007120809130A0B1721141B211E1800BF00BF00BF00BF01224270DFED680AB0EE600A0FE000BF00BF022242700AE000BF0422427006E0CD
:40DFC0000522427003E00622427000E000BF00BF594AD2ED060A60EE800AFCEEE00A10EE902A91B281700A0AC270534AD2ED1C0A60EE800AFCEEE00A10EE902A91B2017142
:40E000000A0A42714B4AB2F8BE1181710A0AC2717047494890ED010A704701B500BF012269464A48006800F2BD10FDF771FA20B99DF800003F4981F8BD0100BFFFF7B1FC5D
:40E04000012000F0DDFC1E20EFF78AFA08BD01B500BF022269463D48006800F5E870FDF757FA20B9BDF800003249A1F8D00100BF08BD00202F4991F8BD110E291AD2DFE8B2
:40E0800001F01A0D0A070E0B0810131B1519171100BF012011E000BF01200EE000BF01200BE000BF012008E0012006E0012004E0012002E000BF00BF00BF00BF704700206E
:40E0C0001C4991F8BD110E291DD2DFE801F01D0F0B07100C0812151E171C1A1300BF40F2635013E000BF45F2CC000FE000BFC8200CE000BF322009E0C82007E04FF4FA702E
:40E1000004E0642002E000BF00BF00BF00BF70475207002055070020560700200000000000504347000400400000014070EC0020002474492021002044290020202900205D
:40E14000002A0020FC030020C0A90646F00300200020C84991F8381009B9142012E0C54991F83810012901D116200BE0C14991F8901009B9152005E0BE4991F8901001291F
:40E1800000D11720704770B50424BB4880780A2876D2DFE800F0051376C5C5C5C5BFC1C30020B5490870C8808860FFF750FFB2488078B149487001208870B2E0FFF7C8FF2B
:40E1C000AD4908700846007810B10720887056E0A948806820B91BF0C7FDA74988604EE0A54988684FF47A711BF0C4FD002846D0FFF70FFFBCEEC00A10EE100A85B2284603
:40E20000FFF725FF9D48B0F8AC0068B19B48B0F8AC009A49B1F8D011884205DD9748B0F8AC009549C88021E09448B0F8D001002803DC01209049C88018E0904890F8BD0114
:40E24000032804D08D4890F8BD01062805D18B48B0F8D00100F5FA7006E08848B0F8D0018000032190FBF1F08349C8800220824988701BF079FD804988600020087350E0A0
:40E280004EE0FFF7C6FE7C48C08800EE900AF8EE600AB4EEE00AF1EE10FA05DB7648007B401C7549087302E0002073490873FFF74FFF714908700846007810B1072088701A
:40E2C00027E06D48007B04280DDB6B48C08800EE900AF8EE600AB0EE600AFFF787FA09206549887015E06449886841F288311BF041FD70B16048C08800EE900AF8EE600A02
:40E30000B0EE600AFFF772FA07205B4988701820087006E0012404E0022402E0032400E000BF00BF5448007818B153490878F8F7D7FB204670BD5048807870474E480078E2
:40E34000704700204C498870C870704701B500BF022269464A480068AC30FDF7D9F820B9BDF800004549A1F8AC0000BF08BD10B52DED028B414890F8BD0103280ED03F48B7
:40E3800090F8BD01062809D03C4890F8BD01022804D03A4890F8BD0105280CD114F0B2FA10B1012806D102E0B7EE008A02E09FED358A00BF01E0B7EE008AB0EE480ABDEC5F
:40E3C000028B10BDB7EE000AF0EE400A2B4890F8BD010E2818D2DFE800F007100809110A0B1317121417151600BF00BF00BF00BF1FEDAB0AF0EE400A07E000BF00BF00BF73
:40E4000000BF00BF00BF00E000BF00BF194890ED060A20EE200A7047B7EE000AF0EE400A164890F8BD010E2818D2DFE800F007100809110A0B1317121417151600BF00BFB4
:40E4400000BF00BF1FEDC00AF0EE400A07E000BF00BF00BF00BF00BF00BF00E000BF00BF044890ED1C0A20EE200A70470648407A7047000044290020182A00202021002074
